:020000020000FC
:100000000C945C4F0C9446000C9446000C944600F3
:100010000C9446000C9446000C9446000C94460048
:100020000C9446000C9446000C94703B0C944600D3
:100030000C9446000C9446000C9446000C947B50A3
:100040000C9446000C9446000C94A2030C944600B9
:100050000C9446000C9446000C9446000C94460008
:100060000C9446000C9446000C9446000C944600F8
:100070000C9446000C9446000C94C0030C9446006B
:100080000C9446000C9446000C94460018952032BF
:100090003030352D31302D32302000000D0D2A2A20
:1000A0002A2A2A2A2A2A2A2A2A2A2A2A2A2A2A2AB0
:1000B0002A2A2A2A2A2A2A2A2A2A2A2A2A2A2A2AA0
:1000C0002A2A2A2A2A2A2A0D2A204D6963726F7346
:1000D00074657070696E672054656C6573636F70CA
:1000E0006520436F6E74726F6C6C657220202020E7
:1000F0002A0D2A204D617274696E20436962756C05
:10010000736B6920202020202863292020200000F4
:100110002A0D2A2A2A2A2A2A2A2A2A2A2A2A2A2A5C
:100120002A2A2A2A2A2A2A2A2A2A2A2A2A2A2A2A2F
:100130002A2A2A2A2A2A2A2A2A2A2A0D0000524D45
:1001400053206572726F723A200066696C6C20737E
:10015000696E65207461626C6520666F72206D6FD8
:10016000746F722063757272656E7473202E2E2EFA
:100170000D006C6F61642064656661756C7420703D
:10018000726F66696C65202E2E2E0D006D6F746F78
:100190007220636F6E74726F6C6C657273202E2E9A
:1001A0002E0D00007374617274206D6F746F722075
:1001B00074696D65722032202E2E2E0D000073742E
:1001C00061727420636C6F636B2074696D6572205B
:1001D00030202873796E633F29202E2E2E0D0000CB
:1001E000737461727420636C6F636B2074696D65E6
:1001F000722030202E2E2E0D0000696E697420634F
:100200006F6D706C657465642C20737461727420FA
:1002100063616C63756C6174696F6E206C6F6F7075
:10022000202E2E2E200D0000656E61626C652074FC
:10023000696D657220696E74657272757074732071
:100240002E2E2E200D006F70656E206F626A656322
:1002500074206461746162617365202E2E2E0D001E
:100260006D61746820283129202E2E2E200D00006B
:100270006D61746820283229202E2E2E200D00005A
:1002800068616E64626F7820646973706C61792054
:10029000286E657729202E2E2E0D00006D61746862
:1002A00020283329202E2E2E200D00007374617219
:1002B000742074776F207769726520696E74657237
:1002C00066616365202E2E2E200D000068616E642D
:1002D000626F7820646973706C6179202E2E2E0D08
:1002E000000068616E64626F78206D656E75202E07
:1002F0002E2E200D00006D6F6E69746F72202E2EF1
:100300002E0D0000585920706F736974696F6E6507
:1003100072206D6F6465202E2E2E200D000020208F
:10032000204F4B2020202D2D2D2D2D2D2D2D206FBC
:1003300066342020202050726F66696C6520202072
:100340004255535920202D2D2D2D2D2D2D2D45522B
:10035000524F520D00000D0D436F6D6D616E647351
:100360003A0D6462203C6164727C6C626C3E2020B9
:1003700020202020202020202020646973706C61C0
:10038000792062797465200D6477203C6164727C09
:100390006C626C3E20202020202020202020202065
:1003A000646973706C617920776F7264200D646C7E
:1003B000203C6164727C6C626C3E202020202020F6
:1003C000202020202020646973706C6179206C6F7C
:1003D0006E67200D6466203C6164727C6C626C3ECA
:1003E00020202020202020202020202064697370DD
:1003F0006C617920666C6F61740D6461203C61648E
:10040000727C6C626C3E2020202020202020202046
:100410002020646973706C61792061647265737304
:10042000200D6D62203C6164727C6C626C3E203CED
:1004300076616C75653E202020206D6F6469667959
:10044000202062797465200D6D77203C6164727C98
:100450006C626C3E203C76616C75653E20202020ED
:100460006D6F646966792020776F7264200D6D6C02
:10047000203C6164727C6C626C3E203C76616C75E1
:10048000653E202020206D6F6469667920206C6FA6
:100490006E67200D6D66203C6164727C6C626C3E00
:1004A000203C76616C75653E202020206D6F64696C
:1004B00066792020666C6F61740D706F72747320A2
:1004C000202020202020202020202020202020202C
:1004D0002020646973706C617920706F7274730D81
:1004E0006C6162656C73203C67726F75705F6E6FD4
:1004F0003E202020202020206C697374206C6162D3
:10050000656C206E616D6573200D72657365742076
:1005100020202020202020202020202020202020DB
:10052000202072657374617274206170706C6963ED
:100530006174696F6E0D6C6F616470726F66203CE0
:100540006E6F3E20202020202020202020206C6F55
:1005500061642070726F66696C652066726F6D20D1
:10056000656570726F6D200D7361766570726F6670
:10057000203C6E6F3E2020202020202020202020A4
:10058000736176652070726F66696C6520746F2088
:10059000656570726F6D200D00006E6F7420616C68
:1005A00069676E656420210D000070726F66696C6A
:1005B00065206E6F2E200000206C6F616465640DF5
:1005C000000070726F66696C65206E6F2E200000EF
:1005D0002073617665640D000F930081002319F08C
:1005E00010D03196FACF0F9108950F920F93C895BE
:1005F000002021F0002D05D03196F9CF0F910F90FA
:1006000008955D9BFECF0CB9089500909B0005FEF8
:10061000FCCF00939C0008950F931F932F93AF93EB
:10062000BF93109107080024A4E6B1E0A10FB01D0C
:100630003DD006F5033211F4112311F40D3021F4ED
:1006400000270C93139516C0083029F4112319F0D4
:100650001A951197EDCF173259F3003248F3002362
:100660003AF3013618F00B370CF400520C93119644
:100670001395DECF10930708BF91AF912F911F9173
:100680000F9108950F931F932F93E8942FB7F89429
:100690000091400101500F731091410101136894C2
:1006A00027FD78942F911F910F9108951F932F93F9
:1006B000AF93BF932FB7F894E89400914001015095
:1006C0000F7310914101011759F013951F73109387
:1006D0004101A0E0B1E0A10F10E0B11F0C916894BE
:1006E00027FD7894BF91AF912F911F910895109895
:1006F000119A00E019E10093900019B900E00BB9DC
:1007000008E90AB906E00093950001E00093400172
:100710000093620100E0009341010093630108959A
:100720008A988B9A00E017E600939800109399003E
:1007300000E000939B0008E900939A0006E0009314
:100740009D0008950F930FB70F931F93AF93BF931F
:100750000091400110914101011759F0A0E0B1E072
:10076000A00F10E0B11F1CB11C9303950F730093F1
:100770004001BF91AF911F910F910FBF0F9118953D
:100780000F930FB70F9300919C000F910FBF0F9124
:10079000189511E0E894043040F008951127E8948A
:1007A000043008F0089500938F01F0E0E1E026E7BF
:1007B000029FE00DF11D0F93B8E0A5E501E00E9456
:1007C000CE04B5E0AAE208E00E94CE04B5E0A2E3C0
:1007D00008E00E94CE04B5E0AAE308E00E94CE043F
:1007E000B5E0A2E408E00E94CE04B5E0AAE408E087
:1007F0000E94CE04B5E0A9E201E00E94CE04B4E07C
:10080000A7E401E00E94CE04B2E0A9E601E00E9464
:10081000CE04B6E0A9EB01E00E94CE04B6E0A0EF62
:1008200001E00E94CE04B6E0A3E704E00E94CE04FB
:10083000B6E0AAEB04E00E94CE04B6E0A7E704E02D
:100840000E94CE04B6E0AEEB04E00E94CE04B6E017
:10085000ABE704E00E94CE04B6E0A2EC04E00E9404
:10086000CE04B6E0AFE704E00E94CE04B6E0A6EC0A
:1008700004E00E94CE04B6E0A3E904E00E94CE04A6
:10088000B6E0AAEC04E00E94CE04B6E0AFE904E0D2
:100890000E94CE04B6E0A6ED04E00E94CE04B6E0CD
:1008A000ABEA04E00E94CE04B6E0A2EE04E00E94AF
:1008B000CE04B6E0A3EF01E00E94CE04B6E0A4EFC0
:1008C00001E00E94CE04B6E0A9EF01E00E94CE0450
:1008D000B6E0AAEF01E00E94CE04B6E0ABEF01E083
:1008E0000E94CE04B6E0ACEF01E00E94CE04B6E078
:1008F000AFEF01E00E94CE04B7E0A0E001E00E946B
:10090000CE04B6E0A7EF01E00E94CE04B6E0A8EF67
:1009100001E00E94CE04B7E0A1E002E00E94CE0414
:10092000B7E0A3E002E00E94CE04B7E0A5E002E059
:100930000E94CE04112371F0E2ECF5E00E94F50272
:100940000F910F5C0E940103E0EDF5E00E94F502BB
:100950006894089500270E941237EAEAF5E00E94A1
:10096000F5020F910F5C0E940103E8EBF5E00E9495
:10097000F5020E94A12068940895E199FECFFFBB83
:10098000EEBB0DBBF894E29AE19A78940895E19950
:10099000FECFFFBBEEBBE09A0DB308950C90E1993A
:1009A000FECFFFBBEEBBE09A1DB2112311F41C92E7
:1009B00007C0011429F00DBAF894E29AE19A7894EC
:1009C000319611960A9551F70895E199FECFFFBB34
:1009D000EEBBE09A0DB20D9231960A95B1F70895EB
:1009E0000F931F9305900D9201501040D9F71F915E
:1009F0000F91E01BF10BA01BB10B08951ED005E574
:100A000090E080E021D0DEF790E080E071D0E6F762
:100A10000E944C420DE00E9401030AEA90E080E04F
:100A200013D0DEF790E080E063D0E6F70E944C42FE
:100A30000DE00E940103689408950CE0009370009B
:100A400000E00093710008951F932F93E89424EA27
:100A5000209374002091740027FFFCCF2091710037
:100A6000287F18E021133EC020EA2093730024E879
:100A7000209374002091740027FFFCCF2091710017
:100A8000287F18E121132EC08093730024E820935F
:100A900074002091740027FFFCCF20917100287F03
:100AA00018E221131FC09093730024E82093740070
:100AB0002091740027FFFCCF20917100287F18E25D
:100AC000211310C00093730024E820937400209138
:100AD000740027FFFCCF20917100287F18E22113BA
:100AE00001C0689414E9109374002F911F91089528
:100AF0001F93E89404EA009374000091740007FFC8
:100B0000FCCF00917100087F18E001135BC000EA80
:100B10000093730004E8009374000091740007FFD1
:100B2000FCCF00917100087F18E101134BC0809346
:100B3000730004E8009374000091740007FFFCCF79
:100B400000917100087F18E201133CC0909373007C
:100B500004E8009374000091740007FFFCCF00913B
:100B60007100087F18E201132DC004EA009374009D
:100B70000091740007FFFCCF00917100087F10E125
:100B8000011320C001EA0093730004E8009374008D
:100B90000091740007FFFCCF00917100087F10E402
:100BA000011310C004E8009374000091740007FF63
:100BB000FCCF00917100087F18E5011303C000917C
:100BC0007300689414E9109374001F9108959001C4
:100BD0004155574143414C4C202020209201415522
:100BE0005741564152202020202094014055574122
:100BF00056414C2020202020950141554D494E530F
:100C00005441434B2020000000002F933F93EF936B
:100C1000FF939801E2E6FCE009E010E00E94F00496
:100C200089014BE2002332F4109500952FEF121B3F
:100C3000020B4DE22AD022E038E511961ED020E0CA
:100C40003CE311961AD020E03AE040E3129615D02A
:100C500020E031E0119611D0FF91EF913F912F915B
:100C600008952B30303A30302020580200003C00EC
:100C700000000A0000000100000040E34395131B40
:100C8000020BE0F74A95130F021F5C914C93451736
:100C900001F008958F939F93CF93DF938FB78F9336
:100CA00080919401D0919201C091930198819817FD
:100CB00059F090939401DEB7CDB78F819E81029752
:100CC00090939001809391018F918FBFDF91CF918D
:100CD0009F918F9108959F93CF93DF93D09192012D
:100CE000C0919301988190939401DF91CF919F914E
:100CF00008950F931F932F933F934F934FB7F894FB
:100D00000EB71DB720919601121720919501120779
:100D100020F400939501109396014FBF4F913F919E
:100D20002F911F910F9108951F932F9315E12DEF90
:100D30002A95F1F71A95D9F70A95C1F72F911F91C6
:100D40000895000000000000000000000000000006
:100D50000000000000000A95A1F708957FF8000048
:100D60000000000000000000000000003FF0000054
:100D700000000000BFF00000000000004000000084
:100D800000000000400800000000000040240000B7
:100D9000000000003FB99999999999993F847AE1A7
:100DA00047AE147B3FE00000000000003FD0000091
:100DB00000000000400921FB54442D183FF921FB9D
:100DC00054442D18BFF921FB54442D183FE921FB51
:100DD00054442D18401921FB54442D184012D97C3D
:100DE0007F3321D247E00000000000004066800011
:100DF0000000000040AADB7E58C4BD340895232DB6
:100E0000222929F12FEF37E02216330601F1200EB7
:100E1000311E11236AF022163306C8F0190144244A
:100E200055246624772488249924AA24BB24089571
:100E300033201AF061F4222051F433242224442474
:100E400055246624772488249924AA24BB24089551
:100E50000080C0E0F0F8FCFEEF93FF9313E00FEF8B
:100E6000201A310A332052F444202AF4E4E7FDE04A
:100E70000E9468146EC00E945D146BC03320E9F7B5
:100E8000022D0433D0F7045007701127E0E5FEE08F
:100E9000E00FF11F0490102C1094022D0C3220F062
:100EA0000B2D0025B02045C0043228F01A201B2845
:100EB000A020BB243EC00C3138F019201A281B2872
:100EC0009020AA24BB2435C0043148F018201928EA
:100ED0001A281B2880209924AA24BB242AC00C305D
:100EE00058F01720182819281A281B287020882441
:100EF0009924AA24BB241DC0043068F016201728AA
:100F0000182819281A281B28602077248824992457
:100F1000AA24BB240EC01520162817281828192823
:100F20001A281B2850206624772488249924AA2470
:100F3000BB2403E01FEF210E301E112051F044208E
:100F400042F40E941414ECE6FDE00E9468140E9432
:100F5000130BFF91EF9108950BE0201A04E0300A83
:100F6000C0F4339419F403EF201620F455246624BA
:100F7000689408955594679477942394DAF3442001
:100F800012F1772022F40894621C521C7AF06894C3
:100F90000895332021F4239404E0201680F04420A7
:100FA0002AF400E8502E6624E89408950FE7502EA6
:100FB0000FEF602EE8940895770C661C551C2A9458
:100FC000D9F74420F2F6609450940FEF601A500A5B
:100FD000772022F40894620852081AF7689408955A
:100FE0000BE1201A04E0300AF0F4339419F403EE14
:100FF000201630F4552466247724882468940895B4
:10100000559467947794879497942394CAF34420D3
:1010100052F1992032F40894821C721C621C521CFA
:101020008AF068940895332021F4239404E0201674
:10103000B0F044203AF400E8502E66247724882447
:10104000E89408950FE7502E0FEF602E702E802E3B
:10105000E8940895990C881C771C661C551C2A94EA
:10106000C9F74420B2F680947094609450940FEFC6
:10107000801A700A600A500A992032F40894820893
:10108000720862085208BAF668940895052C06287A
:1010900011F40C948E14442455203AF45094609426
:1010A0000FEF601A500A00E8402E77248824992414
:1010B000AA24BB240BE0202E04E0302E00E25016C0
:1010C00040F055946794779401E0200E00E0301EC4
:1010D000F5CF00E1501638F4660C551C01E0201ADB
:1010E00000E0300AF6CF0895052C062807280828C6
:1010F00011F40C948E14442455205AF450946094A6
:10110000709480940FEF801A700A600A500A00E809
:10111000402E9924AA24BB240BE1202E04E0302E7B
:1011200000E2501650F05594679477948794979402
:1011300001E0200E00E0301EF3CF00E1501648F42D
:10114000880C771C661C551C01E0201A00E0300A50
:10115000F4CF0895A7EAB1E00DE20D9301E30D93FA
:1011600000E20D93A7EAB1E0CF93DF93CDB7DEB7EE
:10117000C951D040F894CDBFDEBF78940000000084
:101180000D910032E9F3098B0B3219F00D3209F0A1
:101190001197BA8BAB8BECE6FDE00E946814AC2F84
:1011A000BD2FAF5FBF4F0E94A614E4E6FDE00E9492
:1011B0006814BA89AB890D91BA8BAB8B0C8B002369
:1011C00009F4B5C00E3219F10C3209F1053411F0F1
:1011D000053609F45BC0005340F40A3030F0E8945F
:1011E000E4E6FDE00E946814A2C00D8B0E94141476
:1011F000ECE8FDE00E9468140E94070C0E941414A1
:101200006D8855240E9446080E94150BD2CFAC2F42
:10121000BD2FA75FBF4F0E94A614BA89AB890D915D
:10122000BA8BAB8B0C8B002309F481C0053471F1B0
:10123000053661F1005340F40A3030F0E4E6FDE099
:101240000E946814E89473C00D8B0E941414AC2F94
:10125000BD2FAF5FBF4F0E9454140E941414E4E9E5
:10126000FDE00E9468140E94070CAC2FBD2FAF5FF9
:10127000BF4F0E94A6140E9414146D8855240E942A
:1012800046080E94070C0E94150BC7CF1127BA8988
:10129000AB890D910E8B0D3219F00B3209F01197BD
:1012A00011272227332764E00D910033E9F301C0B1
:1012B0000D91005380F00A3070F4422F532F220F0B
:1012C000331F220F331F240F351F220F331F200F10
:1012D000311F6A9569F701E02C32300728F0E4E607
:1012E000FDE00E94681423C03F8B288F0E890D32C9
:1012F00079F49F89888D0197D2F09F8B888F0E9407
:101300001414E4E9FDE00E9468140E94070CF1CF78
:101310009F89888D01975AF09F8B888F0E941414A3
:10132000ECE8FDE00E9468140E94070CF1CF0989E7
:101330000D3211F400E840266894C75EDF4FF89440
:10134000CDBFDEBF7894DF91CF9108953D95FD7FAD
:10135000E1796495CF93DF93CDB7DEB7CC51D04020
:10136000F894CDBFDEBF7894EF93FF93AC2FBD2FE1
:10137000AF5FBF4F0E94A61407E0301669F40FEF6D
:10138000201651F40EE40E94010301E40E940103BF
:101390000EE40E94010314C1332061F4222051F4B1
:1013A00000E30E9401030EE20E94010300E30E9499
:1013B000010306C100E247FC0DE20E940103442440
:1013C000AC2FBD2FA75FBF4F0E94A61400270A8F26
:1013D000AC2FBD2FA75FBF4F0E9454140E9414145E
:1013E000ECE8FDE00E9468140E94130B4420C2F058
:1013F000AC2FBD2FA75FBF4F0E9454140E9414143E
:10140000E4E9FDE00E9468140E94070CAC2FBD2F98
:10141000A75FBF4F0E94A6140A8D03950A8FD8CFED
:10142000AC2FBD2FA75FBF4F0E9454140E9414140D
:10143000ECE6FDE00E9468140E94130B4420C2F405
:10144000AC2FBD2FA75FBF4F0E9454140E941414ED
:10145000ECE8FDE00E9468140E94070CAC2FBD2F41
:10146000A75FBF4F0E94A6140A8D0A950A8FD8CF96
:10147000AC2FBD2FA75FBF4F0E9454140E941414BD
:10148000ECE4F3E10E9468140E94150BAC2FBD2F11
:10149000A75FBF4F0E94A6140E941414ECE8FDE061
:1014A0000E9468140E94130B4420BAF0AC2FBD2F89
:1014B000A75FBF4F0E9454140E941414E4E9FDE09A
:1014C0000E9468140E94070CAC2FBD2FA75FBF4F6E
:1014D0000E94A6140A8D03950A8FAC2FBD2FA75F1B
:1014E000BF4F0E9454140E942C07AC2FBD2FAE5E3C
:1014F000BF4F0E94A6140E94AC0700E3060D0E9495
:1015000001030EE20E9401030BE0098BAC2FBD2FFB
:10151000A75FBF4F0E9454140E941414AC2FBD2F1C
:10152000AE5EBF4F0E9454140E94130B0E9414140D
:10153000ECE8FDE00E9468140E94070CAC2FBD2F60
:10154000A75FBF4F0E94A6140E942C07AC2FBD2F8F
:10155000AE5EBF4F0E94A6140E94AC0700E3060DCA
:101560000E94010309890A95098B09F0CFCF05E68E
:101570000E9401030BE21A8D11231AF40DE211955A
:101580001A8F0E9401031A8D00E3143620F01456BE
:101590001A8F0395FACF0E9401031A8D00E31A30C7
:1015A00020F01A501A8F0395FACF0E9401031A8D6A
:1015B00000E3113018F011500395FBCF0E94010396
:1015C000AC2FBD2FAF5FBF4F0E945414FF91EF911E
:1015D000C45EDF4FF894CDBFDEBF7894DF91CF912A
:1015E0000895DF91CF910F911F910F900F900F9061
:1015F0000F900F900F900F900F900F900F901F93E0
:101600000F930895DF91CF910F911F914F903F90CD
:101610002F905F906F907F908F909F90AF90BF9032
:101620001F930F93089500E84026CF93DF93CDB723
:10163000DEB707E0301621F40FEF201609F4D1CF02
:10164000332019F4222009F4DDCF0E811F810023FD
:1016500021F4112311F40C94F10A073019F41F3FFF
:1016600009F4D0CF1219030918F50D804D82402CD2
:101670000E803E82302C0F802F82202C08845886CA
:10168000502C09846986602C0A847A86702C0B841D
:101690008B86802C0C849C86902C0D84AD86A02C8F
:1016A0000E84BE86B02C002410950095101D001DE0
:1016B0000023B9F61533A8F6210E301E002409C008
:1016C0000B2CBA2CA92C982C872C762C652C552405
:1016D00018501830A8F7112351F056946794779456
:1016E00087949794A794B79407941A95B1F700201C
:1016F0004AF400240894B01CA01C901C801C701C90
:10170000601C501C0D81042552F11E84B10C1D84F7
:10171000A11C1C84911C1B84811C1A84711C1984BB
:10172000611C1884511C55FE19C056946794779417
:1017300087949794A794B79401E0200E00E0301EA0
:101740000FEF17E02016310648F044241801502E00
:10175000602E702E802E902EA02EB02E42CF4D8067
:101760001E841B18B12C1D841A08A12C1C84190876
:10177000912C1B841808812C1A841708712C198449
:101780001608612C18841508512C88F4B094A09484
:10179000909480947094609450940027B01EA01E82
:1017A000901E801E701E601E501E00E8402606E03F
:1017B000552069F01AC00A95F9F0672C782C892C0D
:1017C0009A2CAB2CBB2418E0211A10E0310A6620B9
:1017D00091F30BC001E0201A00E0300ABB0CAA1CF8
:1017E000991C881C771C661C551C54FA9EF73320E4
:1017F0001AF061F4222051F4332422244424552485
:101800006624772488249924AA24BB24EACECF9383
:10181000DF93CDB7DEB707E0301621F40FEF2016C7
:1018200009F4DFCE332019F4222009F4DACE0E8138
:101830001F81002319F4112309F4E4CE073021F4A9
:101840001F3F11F40C94020BC52CD62CE72CF82C5E
:10185000292D3A2D4B2D01E010E0552466247724E4
:1018600088249924AA24BB24B3940E84049E0020C7
:101870000AF41394B12C0D84049EB00CA11C911E8B
:101880000E84039EB00CA11C911EBB2012F4A00E6E
:10189000911EBA2CA92C99240C84049EB00CA11C76
:1018A000911E0D84039EB00CA11C911E0E84029EFD
:1018B000B00CA11C911EBB2012F4A00E911EBA2CDC
:1018C000A92C99240B84049EB00CA11C911E0C849D
:1018D000039EB00CA11C911E0D84029EB00CA11C95
:1018E000911E0E840F9CB00CA11C911EBB2012F403
:1018F000A00E911EBA2CA92C99240A84049EB00C27
:10190000A11C911E0B84039EB00CA11C911E0C8483
:10191000029EB00CA11C911E0D840F9CB00CA11C4A
:10192000911E0E840E9CB00CA11C911EBB2012F4C3
:10193000A00E911EBA2CA92C99240984049EB00CE7
:10194000A11C911E0A84039EB00CA11C911E0B8445
:10195000029EB00CA11C911E0C840F9CB00CA11C0B
:10196000911E0D840E9CB00CA11C911E0E840D9C2A
:10197000B00CA11C911EBB2012F4A00E911EBA2C1B
:10198000A92C99240884049EB00CA11C911E0984E2
:10199000039EB00CA11C911E0A84029EB00CA11CD7
:1019A000911E0B840F9CB00CA11C911E0C840E9CEC
:1019B000B00CA11C911E0D840D9CB00CA11C911E9D
:1019C0000E840C9CB00CA11C911E0884039EA00CDC
:1019D000911C811E0984029EA00C911C811E0A8408
:1019E0000F9CA00C911C811E0B840E9CA00C911CC2
:1019F000811E0C840D9CA00C911C811E0D840C9CDE
:101A0000A00C911C811E0884029E900C811C711EEA
:101A100009840F9C900C811C711E0A840E9C900CF2
:101A2000811C711E0B840D9C900C811C711E0C84FA
:101A30000C9C900C811C711E08840F9C800C711CE6
:101A4000611E09840E9C800C711C611E0A840D9C11
:101A5000800C711C611E0B840C9C800C711C611E1F
:101A600008840E9C700C611C511E09840D9C700C26
:101A7000611C511E0A840C9C700C611C511E0027B5
:101A800008840D9C600C511C011F09840C9C600C87
:101A9000511C011F08840C9C500C011D0D8040241A
:101AA0000F80200C0E80301C1FEF211A13E0310A2A
:101AB000069557946794779487949794A794B794CE
:101AC000069557946794779487949794A794B794BE
:101AD00056946794779487949794A794B794569460
:101AE0006794779487949794A794B79455FE0BC006
:101AF00056946794779487949794A794B79401E049
:101B0000200E00E0301E0FEF17E02016310650F0D7
:101B100044241801502E602E702E802E902EA02E60
:101B2000B02E5FCD33201AF061F4222051F433241B
:101B30002224442455246624772488249924AA2422
:101B4000BB240C94F10ACF93DF93CDB7DEB707E047
:101B5000301621F40FEF201609F443CD332039F469
:101B6000222029F40FEF202E07E0302E3ACD0F81EE
:101B70001E81112319F4002309F444CD173019F400
:101B80000F3F09F43FCD0219130901501C4F1801F2
:101B90000D804024C884D984EA84FB842C853D854B
:101BA0004E8507E010E100244B193A092909F8088D
:101BB000E708D608C50810F0012A07C04B0D3A1DEA
:101BC000291DF81CE71CD61CC51C440F331F221FFF
:101BD000FF1CEE1CDD1CCC1C169531F70F92002467
:101BE00010E80A9509F74B153A052905F804E704AA
:101BF000D604C504BF90AF909F908F907F906F9058
:101C00005F9040F00894B01CA01C901C801C701CBD
:101C1000601C501C54FA56F0BB0CAA1C991C881C62
:101C2000771C661C551C08942008300803281AF0FD
:101C3000022809F0D6CC33242224442455246624D7
:101C4000772488249924AA24BB24CBCCCF93DF9378
:101C5000CDB7DEB7C550D040F894CDBFDEBF789485
:101C600009831A832B833C83B981AA8110960E9431
:101C700054140E941414BB81AC8110960E94541419
:101C80000E94070C0E941414B981AA8118960E9420
:101C900054140E941414BB81AC8118960E945414F1
:101CA0000E94070C0E94150B0E941414B981AA818E
:101CB00050960E9454140E941414BB81AC8150961B
:101CC0000E9454140E94070C0E94150BCB5FDF4F3B
:101CD000F894CDBFDEBF7894DF91CF910895CF9374
:101CE000DF93CDB7DEB7C750D040F894CDBFDEBF8D
:101CF000789409831A832B833C834D835E83B98157
:101D0000AA8118960E9454140E941414BB81AC81BD
:101D100050960E9454140E94070C0E941414B9811A
:101D2000AA8150960E9454140E941414BB81AC8165
:101D300018960E9454140E94070C0E94130BBD8138
:101D4000AE8110960E94A614B981AA8150960E9475
:101D500054140E941414BB81AC8110960E94541438
:101D60000E94070C0E941414B981AA8110960E9447
:101D700054140E941414BB81AC8150960E945414D8
:101D80000E94070C0E94130BBD81AE8118960E9421
:101D9000A614B981AA8110960E9454140E941414AA
:101DA000BB81AC8118960E9454140E94070C0E94BB
:101DB0001414B981AA8118960E9454140E94141414
:101DC000BB81AC8110960E9454140E94070C0E94A3
:101DD000130BBD81AE8150960E94A614C95FDF4FE0
:101DE000F894CDBFDEBF7894DF91CF910895CF9363
:101DF000DF93CDB7DEB7C550D040F894CDBFDEBF7E
:101E0000789409831A832B833C8398011FDF332046
:101E100021F4222011F4E89437C00E94C9140E94D2
:101E20001414ECE6FDE00E9468140E9432140E9433
:101E3000A30D0E9414140E9414140E941414B9815A
:101E4000AA8110960E9454140E94070CBB81AC8199
:101E500010960E94A614B981AA8118960E94541463
:101E60000E94070CBB81AC8118960E94A614B98110
:101E7000AA8150960E9454140E94070CBB81AC8129
:101E800050960E94A6146894CB5FDF4FF894CDBFA4
:101E9000DEBF7894DF91CF910895CF93DF93CDB7D4
:101EA000DEB7C550D040F894CDBFDEBF78942B8309
:101EB0003C8309831A83BB81AC8110960E94541421
:101EC0000E941414B981AA8110960E9454140E9491
:101ED000070C0E941414BB81AC8118960E94541404
:101EE0000E941414B981AA8158960E9454140E9429
:101EF000070C0E94150B0E941414BB81AC815096F4
:101F00000E9454140E941414B981AA81D0960E9490
:101F100054140E94070C0E94150BCB5FDF4FF894FE
:101F2000CDBFDEBF7894DF91CF910895CF93DF933B
:101F3000CDB7DEB7C052D040F894CDBFDEBF7894A5
:101F400009831A832B833C834D835E8300E10F83D7
:101F500009811A8144275F81150F041F2B813C8161
:101F60009CDFDE0118961F810027A10FB01F0E9481
:101F7000A6140F8108500F8358F7BD81AE81FE0172
:101F8000389608E101900D920A95E1F7C05EDF4FA7
:101F9000F894CDBFDEBF7894DF91CF910895CF93B1
:101FA000DF93CDB7DEB7C950D040F894CDBFDEBFC8
:101FB000789409831A832B833C834D835E8300E3EB
:101FC000088700E10F8309811A8144275F81150F7B
:101FD000041F2B813C8144275885350F241F5DDF6A
:101FE0000F811885100F0027BD81AE81A10FB01F92
:101FF0000E94A6140F8108500F8328F70885085106
:102000000887F8F6C75FDF4FF894CDBFDEBF78943E
:10201000DF91CF910895CF93DF93CDB7DEB7C6514F
:10202000D040F894CDBFDEBF7894B02FA12FB983F4
:10203000AA835896BB83AC835896BD83AE83B22FD8
:10204000A32FBF83A8875896B987AA875896BB87BE
:10205000AC87BB81AC8118960E9454140E94141462
:10206000BD81AE8150960E9454140E94070C0E94BC
:102070001414BB81AC8150960E9454140E94141415
:10208000BD81AE8118960E9454140E94070C0E94D4
:10209000130BBF81A88510960E94A6140E941414E9
:1020A000B981AA8110960E9454140E94070C0E94C4
:1020B0001414BB81AC8150960E9454140E941414D5
:1020C000BD81AE8110960E9454140E94070C0E949C
:1020D0001414BB81AC8110960E9454140E941414F5
:1020E000BD81AE8150960E9454140E94070C0E943C
:1020F000130BB985AA8510960E94A6140E94141489
:10210000B981AA8118960E9454140E94070C0E945B
:10211000150B0E941414BB81AC8110960E945414BC
:102120000E941414BD81AE8118960E9454140E941E
:10213000070C0E941414BB81AC8118960E945414A1
:102140000E941414BD81AE8110960E9454140E9406
:10215000070C0E94130BBB85AC8510960E94A61439
:102160000E941414B981AA8150960E9454140E94AE
:10217000070C0E94150BAC2FBD2FA35FBF4F0E9411
:10218000A614B981AA8150960E9454140E94141476
:10219000BD81AE8118960E9454140E94070C0E94C3
:1021A0001414B981AA8118960E9454140E94141420
:1021B000BD81AE8150960E9454140E94070C0E946B
:1021C000130BBF81A88518960E94A614B981AA8115
:1021D00010960E9454140E941414BD81AE81509632
:1021E0000E9454140E94070C0E941414B981AA8101
:1021F00050960E9454140E941414BD81AE81109612
:102200000E9454140E94070C0E94130BB985AA85E2
:1022100018960E94A614B981AA8118960E94541497
:102220000E941414BD81AE8110960E9454140E9425
:10223000070C0E941414B981AA8110960E945414AC
:102240000E941414BD81AE8118960E9454140E94FD
:10225000070C0E94130BBB85AC8518960E94A61430
:10226000B981AA8118960E9454140E941414BB814B
:10227000AC8150960E9454140E94070C0E941414C2
:10228000B981AA8150960E9454140E941414BB81F3
:10229000AC8118960E9454140E94070C0E94130BE4
:1022A000BF81A88550960E94A614B981AA81509634
:1022B0000E9454140E941414BB81AC8110960E9499
:1022C00054140E94070C0E941414B981AA8110961C
:1022D0000E9454140E941414BB81AC8150960E9439
:1022E00054140E94070C0E94130BB985AA855096BE
:1022F0000E94A614B981AA8110960E9454140E94CB
:102300001414BB81AC8118960E9454140E94070CCF
:102310000E941414B981AA8118960E9454140E9434
:102320001414BB81AC8110960E9454140E94070CB7
:102330000E94130BBB85AC8550960E94A61400E446
:102340000D8BBF81A88500271D89A10FB01F0E949A
:1023500054140E941414AC2FBD2FA35FBF4F0E94D2
:1023600054140E94A30DBF81A88500271D89A10FC9
:10237000B01F0E94A6140D8908500D8B10F7CA5E7D
:10238000DF4FF894CDBFDEBF7894DF91CF910895F1
:10239000CF93DF93CDB7DEB7C750D040F894CDBF11
:1023A000DEBF7894B02FA12FB983AA835896BB8340
:1023B000AC835896BD83AE830E9414140E94021809
:1023C000BB81AC8150960E94A61400E84026BD81D6
:1023D000AE8118960E94A6140E9423140E94B3177F
:1023E000BB81AC8118960E94A614BD81AE81509627
:1023F0000E94A614ECE6FDE00E946814B981AA814F
:1024000010960E94A614E4E6FDE00E946814B981CB
:10241000AA8118960E94A614B981AA8150960E949A
:10242000A614BB81AC8110960E94A614BD81AE811A
:1024300010960E94A614C95FDF4FF894CDBFDEBF8F
:102440007894DF91CF910895CF93DF93CDB7DEB726
:10245000C750D040F894CDBFDEBF7894B02FA12FE5
:10246000B983AA835896BB83AC835896BD83AE8349
:102470000E9414140E940218BD81AE8110960E9421
:10248000A61400E84026B981AA8150960E94A6149D
:102490000E9423140E94B317B981AA8110960E944A
:1024A000A614BD81AE8150960E94A614ECE6FDE014
:1024B0000E946814BB81AC8118960E94A614E4E6C1
:1024C000FDE00E946814B981AA8118960E94A614A2
:1024D000BB81AC8110960E94A614BB81AC81509642
:1024E0000E94A614BD81AE8118960E94A614C95FF1
:1024F000DF4FF894CDBFDEBF7894DF91CF91089580
:10250000CF93DF93CDB7DEB7C750D040F894CDBF9F
:10251000DEBF7894B02FA12FB983AA835896BB83CE
:10252000AC835896BD83AE830E9414140E94021897
:10253000B981AA8118960E94A61400E84026BB81A2
:10254000AC8110960E94A6140E9423140E94B31717
:10255000B981AA8110960E94A614BB81AC811896FD
:102560000E94A614ECE6FDE00E946814BD81AE81D5
:1025700050960E94A614E4E6FDE00E946814B9811A
:10258000AA8150960E94A614BB81AC8150960E94ED
:10259000A614BD81AE8110960E94A614BD81AE81A5
:1025A00018960E94A614C95FDF4FF894CDBFDEBF16
:1025B0007894DF91CF910895E894032C022819F0C4
:1025C00044200AF068940895E894032C022809F046
:1025D00047FA08956894032C022819F044200AF45D
:1025E000E89408956894032C0228D9F347FA0895D3
:1025F0006894032C022809F0E89408956894032C49
:102600000228D9F7E8940895CF93DF93CDB7DEB7CA
:10261000E8940D804014E9F50E800314D1F50F8085
:102620000214B9F5BF92AF929F928F927F926F92F0
:102630005F9200271FEF0E84B0180D84A0080A29AE
:102640001A210C849008092919210B848008082973
:1026500018210A84700807291721098460080629AF
:102660001621088450080529152130F0002351F463
:102670000B2D063038F405C01B3F20F01B2D1F3FEB
:1026800008F068945F906F907F908F909F90AF90CC
:10269000BF90DF91CF910895CF93DF93CDB7DEB791
:1026A00068940D80401438F129F5442092F10E8091
:1026B000031408F1F9F40F800214E8F0D9F4088447
:1026C0000514C8F0B9F409840614A8F099F40A8432
:1026D000071488F079F40B84081468F059F40C841A
:1026E000091448F039F40D840A1428F019F40E8402
:1026F0000B1408F0E894DF91CF910895CF93DF9306
:10270000CDB7DEB7E8940D80401438F129F54420A8
:1027100072F20E80031408F1F9F40F800214E8F04D
:10272000D9F408840514C8F0B9F409840614A8F093
:1027300099F40A84071488F079F40B84081468F07B
:1027400059F40C84091448F039F40D840A1428F063
:1027500019F40E840B1408F06894DF91CF9108955A
:10276000CF93DF93CDB7DEB7E8940D80401430F1FE
:1027700031F5442092F10E80031400F101F50F8031
:102780000214E0F0E1F408840514C0F0C1F40984F7
:102790000614A0F0A1F40A84071480F081F40B84DD
:1027A000081460F061F40C84091440F041F40D84C5
:1027B0000A1420F021F40E84B01408F06894DF911C
:1027C000CF910895CF93DF93CDB7DEB768940D8096
:1027D000401430F131F5442072F20E80031400F100
:1027E00001F50F800214E0F0E1F408840514C0F054
:1027F000C1F409840614A0F0A1F40A84071480F03F
:1028000081F40B84081460F061F40C84091440F026
:1028100041F40D840A1420F021F40E84B01400F069
:10282000E894DF91CF9108950F901F90BF92AF92DF
:102830009F928F927F926F925F922F923F924F92D0
:102840001F920F9208950F901F904F903F902F90DE
:102850005F906F907F908F909F90AF90BF901F92EE
:102860000F920895ADB7BEB713960C904D92402CC1
:102870000C903D92302C0C902D92202C0C905D925F
:10288000502C0C906D92602C0C907D92702C0C90C2
:102890008D92802C0C909D92902C0C90AD92A02C3F
:1028A0000C90BD92B02C08954D905D906D907D90F0
:1028B0008D909D90AD90BD9013C04424332422246C
:1028C00055246624772488249924AA24BB240895B7
:1028D000459055906590759085909590A590B59090
:1028E000042D0529D9F0042D0F770F3721F4052D7C
:1028F000007F003FF1F0342C00E84022232C22948A
:1029000000EF2022329407E03022052D02950F704F
:10291000202A0FE0502200E1502A08954424332455
:10292000222455246624772488249924AA24BB24AD
:102930000895442407E0302E0FEF202E55246624FE
:10294000772488249924AA24BB240895022D007F8B
:102950000295132D17701295012B04290D93022D4A
:102960000295007F152D1F70012B0D936D927D92A6
:102970008D929D92AD92BD9208953FF6A09E667F86
:102980003BCD3FDAB52AEF348E523FE2E29B8F2FE8
:10299000CF79CF93DF93CDB7DEB7C251D040F89453
:1029A000CDBFDEBF7894EF93FF9307E0301621F49C
:1029B0000FEF201609F412C0332011F4222071F019
:1029C00044206AF40FEF202E07E0302E44245524D3
:1029D0006624772488249924AA24BB2481C0AC2FA0
:1029E000BD2FAF5FBF4F0E94A61413E00EEF201A59
:1029F000310A398A2A8A0EEF202E03E0302E0E94F7
:102A00001414EAE8F9E20E9468140E94070C0E947C
:102A10001414E2E8F9E20E9468140E94150B198967
:102A20000A8915950795200E311E0A8900FB46F488
:102A30000E941414EAE7F9E20E9468140E94070C4D
:102A40000E9414140E941414AC2FBD2FAF5FBF4F0F
:102A50000E9454140E9432140E94A30D0E94150B70
:102A600001E0201A00E0300A0E9414140E9414149D
:102A7000AC2FBD2FAF5FBF4F0E9454140E94321481
:102A80000E94A30D0E94150B01E0201A00E0300AFD
:102A90000E9414140E941414AC2FBD2FAF5FBF4FBF
:102AA0000E9454140E9432140E94A30D0E94150B20
:102AB00001E0201A00E0300A0E9414140E9414144D
:102AC000AC2FBD2FAF5FBF4F0E9454140E94321431
:102AD0000E94A30D0E94150B01E0201A00E0300AAD
:102AE000FF91EF91CE5EDF4FF894CDBFDEBF7894BB
:102AF000DF91CF910895EF93FF93E8E0FBE20E940E
:102B0000D515FF91EF9108953C62F49B46814157A2
:102B10003CA6827863B97D973CE952C77030AD4AD4
:102B20003D2AE7F3E733B81F3D6AE7F3E733B81F01
:102B30003DA93974A8C07C9D3DE6124613A86D09D5
:102B40003E21EED8EFF8D8983E5AE64567F544E4C2
:102B50003E927E4FB7789F5C3EC71DE3A556C734B3
:102B60003EFA01A01A01A01A3F2A01A01A01A01AD8
:102B70003F56C16C16C16C173F8111111111111113
:102B80003FA55555555555553FC555555555555561
:102B90003FE00000000000003FF0000000000000E7
:102BA0003FF0000000000000FFFFCF93DF93CDB7A0
:102BB000DEB7C950D040F894CDBFDEBF7894AC2FBB
:102BC000BD2FAF5FBF4F0E94A6140E946814C89526
:102BD000039489F00E941414AC2FBD2FAF5FBF4F38
:102BE0000E9454140E94070C0E9414140E9468143E
:102BF0000E94150BECCFC75FDF4FF894CDBFDEBF4F
:102C00007894DF91CF910895BFEC007FA1F72594D0
:102C1000C03028545B6B807AC052C08C36880273F7
:102C2000C05EB8BF2D05BA25C0503669FD28EC8EB0
:102C3000FFFF3FF00000000000004038DBC45B14E1
:102C4000603C4064A0DD43B8FA25407B0E18D2E218
:102C5000BE3B407E563F13B049EA4068519EFBBDE3
:102C600062ECFFFF4003504F333F9DE63FE51EB847
:102C700051EB851FCF93DF93CDB7DEB7C352D04062
:102C8000F894CDBFDEBF7894EF93FF9307E0301642
:102C900021F40FEF201609F4B0C049A24424AC2F50
:102CA000BD2FAF5FBF4F0E94A6140E941414E4E62C
:102CB000FCE20E9468140E94E213DEF4ECEBFDE0FB
:102CC0000E946814AC2FBD2FA75FBF4F0E94A614AF
:102CD000E4E7FDE00E9468140E9432140E94A30DF4
:102CE000AC2FBD2FAF5FBF4F0E94A61401E00AA317
:102CF0003EC0ECE6FCE20E9468140E94B0136EF441
:102D00000E945D14AC2FBD2FA75FBF4F0E94A61479
:102D10000E94231400270AA32AC0ECECFDE00E94C5
:102D20006814AC2FBD2FA75FBF4F0E94A614ECE61E
:102D3000FDE00E9468140E94130B0E941414AC2F33
:102D4000BD2FAF5FBF4F0E9454140E941414ECE6D5
:102D5000FDE00E9468140E94150B0E94A30DAC2F89
:102D6000BD2FAF5FBF4F0E94A61402E00AA30E94CE
:102D700014140E94070CAC2FBD2FAF5EBF4F0E94F2
:102D8000A6140E941414E8E0FCE20E94D5150E94EB
:102D9000070C0E941414AC2FBD2FAF5EBF4F0E94D2
:102DA0005414E2E3FCE20E94D5150E94A30D0E9498
:102DB0001414AC2FBD2FAF5FBF4F0E9454140E945C
:102DC000070C0E941414AC2FBD2FAF5FBF4F0E94A1
:102DD00054140E94150BAC2FBD2FAF5EBF4F0E9445
:102DE000A6140E941414AC2FBD2FA75FBF4F0E94E2
:102DF00054140E94150B09A04024FF91EF91CD5D62
:102E0000DF4FF894CDBFDEBF7894DF91CF91089566
:102E1000CF93DF93CDB7DEB7C451D040F894CDBF88
:102E2000DEBF7894EF93FF9307E0301621F40FEFA5
:102E3000201609F47FC0AC2FBD2FAF5FBF4F0E949B
:102E4000A6144594498A3A8A2B8A498C3A8C2B8C51
:102E50005C8C6D8C7E8C8F8C98A0A9A0BAA007E0AA
:102E6000301621F40FEF201609F464C0AC2FBD2FEB
:102E7000A75FBF4F0E94A61409880428098A0B89FE
:102E80001A89422D532D401B510BB0F00CE310E07A
:102E90004017510788F044202AF4E4ECFDE00E943A
:102EA000681448C0222019F4332009F443C0ECEB25
:102EB000FDE00E9468143EC0332069F4222059F4DA
:102EC0000989007419F40E945D1434C0E4EBFDE03C
:102ED0000E9468142FC00E941414AC2FBD2FAF5F46
:102EE000BF4F0E9454140E94A30D0E943A160989F4
:102EF000003C71F00038A9F0003409F01BC00E94BA
:102F00001414E4EBFDE00E9468140E94150B12C03B
:102F10000E941414E4EBFDE00E9468140E94130B5D
:102F200009C00E941414E4EBFDE00E9468140E94A2
:102F3000150B00C0FF91EF91CC5EDF4FF894CDBF31
:102F4000DEBF7894DF91CF910F911F910F900F907A
:102F50000F900F900F900F900F900F900F900F9079
:102F60001F930F9308950E941414EF93FF93ECEBBB
:102F7000FDE00E946814FF91EF910E94150B42C082
:102F80003DE5D8FD1FD19CCDBE5AE5E5A9291F5DC1
:102F90003EC71DE3567D48A1BF2A01A019BFDF032C
:102FA0003F8111111110F7D0BFC5555555555548E2
:102FB000FFFFBDA8FA49A0861A9B3E21EE9D7B4EDD
:102FC0003F05BE927E4F7EAC4BC63EFA01A019C8AB
:102FD00044F5BF56C16C16C14F913FA55555555587
:102FE000554BFFFF3FE921FB400000003E64442DAC
:102FF000000000003CE8469898CC517041CDCD656A
:1030000000000000CF93DF93CDB7DEB7CB52D040A6
:10301000F894CDBFDEBF7894EF93FF9349A6442484
:103020000E941414ECEFFFE20E9468140E947E13C9
:103030000E9423141EF40E945D1405C1AC2FBD2F05
:10304000AF5FBF4F0E94A6140E941414ECECFDE089
:103050000E9468140E94A30D0E942C07AC2FBD2F64
:10306000A75FBF4F0E94A614332011F42220B1F0B5
:1030700004E0201A0027300A0E942C0704E0200EEA
:103080000027301E0E941414AC2FBD2FA75FBF4F26
:103090000E9454140E94130B00E84026AC2FBD2F51
:1030A000AF5EBF4F0E94A61403E0201A55942394EC
:1030B000E9F75AA601E05022B9F00AA503950AA73C
:1030C000AC2FBD2FA75FBF4F0E9454140E94141451
:1030D000ECE6FDE00E9468140E94150BAC2FBD2F9A
:1030E000A75FBF4F0E94A6140AA50770043020F006
:1030F000045019A5105819A70AA7AC2FBD2FA75F18
:10310000BF4F0E9454140E941414E4EEFFE20E9488
:1031100068140E94070C00E840260E941414AC2F8B
:10312000BD2FAF5FBF4F0E9454140E94150B0E9429
:103130001414AC2FBD2FA75FBF4F0E9454140E94E0
:103140001414ECEEFFE20E9468140E94070C0E9427
:10315000130B0E941414AC2FBD2FA75FBF4F0E940A
:1031600054140E941414E4EFFFE20E9468140E94B9
:10317000070C0E94130BAC2FBD2FAF5EBF4F0E94F8
:10318000A6140E9414140E94070CAC2FBD2FA75E3A
:10319000BF4F0E94A6140AA5013011F0023079F544
:1031A000E2EBFFE20E94D5150E941414AC2FBD2F54
:1031B000A75EBF4F0E9454140E9414140E94070C73
:1031C0000E94070C0E941414ECE6FDE00E946814B3
:1031D0000E941414AC2FBD2FA75EBF4F0E94541441
:1031E00001E0201A00E0300A0E94130B0E94150B28
:1031F000AC2FBD2FA75FBF4F0E94A61422C0E0E8EE
:10320000FFE20E94D5150E941414AC2FBD2FA75EBB
:10321000BF4F0E9454140E94070C0E941414AC2F3C
:10322000BD2FAF5EBF4F0E9454140E94070C0E9436
:103230001414AC2FBD2FAF5EBF4F0E9454140E94D8
:10324000150B09A5400EFF91EF91C55DDF4FF89476
:10325000CDBFDEBF7894DF91CF91089509D26FD2B0
:10326000A5D2E7D2CCD324D35ED383D312D42BD42C
:103270000895811915464E4F5020202020202020EF
:1032800088191541444420202020202020209F1907
:10329000155355422020202020202020B619154DFE
:1032A000554C2020202020202020CD19154449569F
:1032B0002020202020202020E419154154414E32A6
:1032C000202020202020FB191553494E20202020AB
:1032D000202020200C1A15434F532020202020208E
:1032E00020201D1A154154414E202020202020204E
:1032F0002E1A155351525420202020202020000047
:103300000000CED026F4AFE2B2E00C943441089530
:10331000B6D0A6F4AFE2B2E00E9454140E94141496
:10332000A7E3B2E00E9454140E94150BAFE3B2E091
:103330000E94A614AFE3B2E00C94344108959FD0EC
:10334000A6F4AFE2B2E00E9454140E941414A7E362
:10335000B2E00E9454140E94130BAFE3B2E00E944B
:10336000A614AFE3B2E00C943441089588D0A6F4DB
:10337000AFE2B2E00E9454140E941414A7E3B2E03A
:103380000E9454140E94070CAFE3B2E00E94A614FE
:10339000AFE3B2E00C943441089571D0A6F4AFE2EB
:1033A000B2E00E9454140E941414A7E3B2E00E94F9
:1033B00054140E94A30DAFE3B2E00E94A614AFE341
:1033C000B2E00C94344108955AD0A6F4AFE2B2E0D2
:1033D0000E9454140E941414A7E3B2E00E945414F3
:1033E0000E940817AFE3B2E00E94A614AFE3B2E078
:1033F0000C943441089554D076F4AFE2B2E00E94C8
:1034000054140E940218AFE3B2E00E94A614AFE386
:10341000B2E00C943441089543D076F4AFE2B2E0C8
:103420000E9454140E94B317AFE3B2E00E94A614A6
:10343000AFE3B2E00C943441089532D076F4AFE2B9
:10344000B2E00E9454140E943A16AFE3B2E00E9428
:10345000A614AFE3B2E00C943441089521D076F481
:10346000AFE2B2E00E9454140E94C914AFE3B2E08C
:103470000E94A614AFE3B2E00C9434410895E8949E
:103480000E949C4266F4AFE2B2E00E94A6140E9441
:103490009C422EF4A7E3B2E00E94A614689408951B
:1034A000E8940E949C423EF4AFE2B2E0AFE2B2E0A8
:1034B0000E94A6146894089540283EF9DB22D0E5C6
:1034C000C0283EF9DB22D0E500000000000000002B
:1034D00040283EF9DB22D0E540147DF3B645A1CB70
:1034E00040313EF9DB22D0E540283EF9DB22D0E531
:1034F000C0147DF3B645A1CB401BFFFFFFFFFFFFCC
:1035000040147DF3B645A1CBC0283EF9DB22D0E5BF
:10351000C01BFFFFFFFFFFFFC0147DF3B645A1CB2B
:1035200040283EF9DB22D0E5401BFFFFFFFFFFFFF5
:10353000C01154FDF3B645A2C019BB645A1CAC08B7
:10354000C025883126E978D5C0147DF3B645A1CBD6
:1035500040283EF9DB22D0E5401BFFFFFFFFFFFFC5
:10356000FFFFE8EBF4E3C8950FEF001649F00E9467
:1035700068140E94AA09B2E0A7E40E94B408F3CF3D
:103580000895AF93BF93B0916702A09168020D9325
:10359000B0936702A0936802BF91AF9108950F9313
:1035A0001F93AF93BF93A7E4B2E0B0936702A093D9
:1035B000680200E210E21D930A95E9F7BF91AF910E
:1035C0001F910F91089540283EF9DB22D0E5C028D5
:1035D0003EF9DB22D0E5000000000000000040289A
:1035E0003EF9DB22D0E540147DF3B645A1CB403156
:1035F0003EF9DB22D0E540283EF9DB22D0E5C014BD
:103600007DF3B645A1CB401BFFFFFFFFFFFF40143A
:103610007DF3B645A1CBC0283EF9DB22D0E5C01B27
:10362000FFFFFFFFFFFFC0147DF3B645A1CB40288D
:103630003EF9DB22D0E5401BFFFFFFFFFFFFC0117B
:1036400054FDF3B645A2C019BB645A1CAC08C02592
:10365000883126E978D5C0147DF3B645A1CB402842
:103660003EF9DB22D0E5401BFFFFFFFFFFFFFFFF1E
:10367000E6ECF5E3C8950FEF0016B9F00E94681468
:103680000E9414140E9468140E94150B0E941414C6
:103690000E9468140E9404130E9423145EF3AFE991
:1036A000B1E00E94A6140E94FE06089540283EF94B
:1036B000DB22D0E540283EF9DB22D0E50000000007
:1036C0000000000040313EF9DB22D0E540283EF901
:1036D000DB22D0E540147DF3B645A1CA401C0000B2
:1036E0000000000040283EF9DB22D0E5C0147DF345
:1036F000B645A1CAC01C00000000000040147DF3C4
:10370000B645A1CBC0283EF9DB22D0E6401BFFFF27
:10371000FFFFFFFFC0147DF3B645A1CB40283EF963
:10372000DB22D0E6C025883126E978D5C01154FDCA
:10373000F3B645A2C019BB645A1CAC08FFFFECEA03
:10374000F6E3C8950FEF0016B9F00E9468140E94C6
:1037500014140E9468140E94130B0E9414140E94F7
:1037600068140E9404130E9423145EF3AFE9B1E0D1
:103770000E94A6140E94FE0608953FF3C083126EB5
:10378000978D3FFBEDFA43FE5C9240013D52DC45D4
:10379000E694C0283EF9DB22D0E5C0147DF3B6459F
:1037A000A1CB404F0D95A294141EFFFFEAE7F7E36B
:1037B000C8950FEF0016B9F00E9468140E94141407
:1037C0000E9468140E94070C0E9414140E9468143E
:1037D0000E9404130E9423145EF3AFE9B1E00E943B
:1037E000A6140E94FE0608953FF0000100000000AC
:1037F0003FF00000000000003FF00001000000006A
:10380000404F0D95A294141E3FF0000000000000F0
:10381000404F0D95A294141E404F0D95A294141F75
:10382000C0283EF9DB22D0E5C0147DF3B645A1CB1C
:10383000FFFFE8EEF7E3C8950FEF0016B9F00E941E
:1038400068140E9414140E9468140E94A30D0E9420
:1038500014140E9468140E9404130E9423145EF33F
:10386000AFE9B1E00E94A6140E94FE0608953FD081
:103870000000000000003FE0000000000000000029
:103880000000000000000000000000000000C01464
:103890007DF3B645A1CB7FF0000000000000405E44
:1038A000E00000000000402639E2653E421BFFFFB9
:1038B000EEE6F8E3C8950FEF001699F00E94681441
:1038C0000E94C9140E9414140E9468140E940413D8
:1038D0000E9423147EF3AFE9B1E00E94A6140E9477
:1038E000FE06089540040000000000003FF30B6D49
:1038F000796A4DA83FF00000000000003FE921FB7D
:1039000054442D183FE00000000000003FDDAC678C
:103910000561BB4FBFE0000000000000BFDDAC67E9
:103920000561BB4FFFFFE4EEF8E3C895039499F0FF
:103930000E9468140E943A160E9414140E9468148F
:103940000E9404130E94231486F3AFE9B1E00E94A1
:10395000A6140E94FE060895400400000000000026
:103960003FF00000000000003FF30B6D796A4DA8A6
:10397000FFFFE8E5F9E3C8950394B9F00E946814E5
:103980000E9414140E9468140E9408170E941414C4
:103990000E9468140E9404130E94231466F3AFE986
:1039A000B1E00E94A6140E94FE0608954012000095
:1039B0000000000040100000000000003FE1999965
:1039C0009999999A0000000000000000C0120000C0
:1039D00000000000C014000000000000C012000041
:1039E00000000000C014000000000000BFE1999931
:1039F0009999999ABFF0000000000000FFFFECEADF
:103A0000F9E3C895039499F00E9468140E942C076A
:103A10000E9414140E9468140E9404130E9423142C
:103A200086F3AFE9B1E00E94A6140E94FE06089555
:103A3000408F4000000000003FEA75CC150A206B63
:103A4000C0280000000000003FE12B9AF7D765A5D1
:103A50003FE00000000000003FDEAEE8744B05F0E0
:103A60003FF00000000000003FEAED548F090CEE2B
:103A700040000000000000003FED18F6EAD1B44617
:103A800040080000000000003FC210386DB6D55B52
:103A9000FFFFE0E3FAE3C895039499F00E946814ED
:103AA0000E9402180E9414140E9468140E940413B9
:103AB0000E94231486F3AFE9B1E00E94A6140E948D
:103AC000FE060895FFFFE4ECFAE3C895039499F02D
:103AD0000E9468140E94B3170E9414140E94681474
:103AE0000E9404130E94231486F3AFE9B1E00E9400
:103AF000A6140E94FE060895B91E1441504F53317A
:103B00002020202020204E1F1441504F53322020CF
:103B100020202020E31F1441504F53332020202029
:103B2000202078201441504F532020202020202096
:103B30003421154143414C43202020202020E526FC
:103B40001541414E412020202020202051022041BB
:103B50004541525241592020202047044041454FC1
:103B600050454E20202020205004404145434F55D1
:103B70004E54455220204804434145525253554D1E
:103B800020202020560842434C4F434B2020202029
:103B900020205A0840434C4F434B5354455020205B
:103BA0006B02414152454354494E543120206D022D
:103BB00041414445434C494E543120206F0243411A
:103BC00052454354524144312020770243414445F9
:103BD000434C5241443120207F02424154494D45DB
:103BE00031202020202083024241415A5354455025
:103BF0005331202087024241414C54535445505385
:103C000031208B024341415A52414431202020202F
:103C100093024341414C5452414431202020FB0245
:103C20004041464C41475331202020209B024141D6
:103C300052454354494E543220209D02414144454F
:103C4000434C494E543220209F0243415245435435
:103C5000524144322020A70243414445434C524143
:103C600044322020AF02424154494D4532202020A9
:103C70002020B3024241415A535445505332202030
:103C8000B7024241414C5453544550533220BB0279
:103C90004341415A5241443220202020C302434133
:103CA000414C5452414432202020FC024041464CB9
:103CB0004147533220202020690240415345415260
:103CC00043485A3320206A024041535A33455252E6
:103CD0004E4F2020FF0243414D4E54564543312064
:103CE0002020170343414D4E545645433220202097
:103CF0002F0343414D4E5456454333202020470364
:103D00004341534B59564543312020205F034341E3
:103D1000534B595645433220202077034341534BA0
:103D200059564543332020201F0443414D494E5AE4
:103D3000332020202020270443414D41585A33206E
:103D4000202020202F0443414D494E534550202030
:103D50002020370443414D41585345502020202016
:103D60003F04434154525545534550202020000004
:103D7000000001E60E9401030AE70E9401030DE32F
:103D80000E94010300E30E94010308E70E9401036F
:103D9000009183020E944C42009184020E944C4296
:103DA000009185020E944C42009186020E944C4282
:103DB00000E20E94010301E60E9401030CE60E945A
:103DC000010304E70E9401030DE30E94010300E3E5
:103DD0000E94010308E70E940103009187020E94EC
:103DE0004C42009188020E944C42009189020E943C
:103DF0004C4200918A020E944C4200E20E94010360
:103E000004E70E9401030DE30E94010300E30E9406
:103E1000010308E70E94010300917F020E944C42C7
:103E2000009180020E944C42009181020E944C420B
:103E3000009182020E944C4200E20E94010302E7CC
:103E40000E9401030DE30E94010300E30E940103AD
:103E500008E70E94010300916B020E944C4200910E
:103E60006C020E944C4200E20E94010304E60E94A0
:103E700001030DE30E94010300E30E94010308E730
:103E80000E94010300916D020E944C4200916E025B
:103E90000E944C420DE00E940103089501E60E9439
:103EA00001030AE70E9401030DE30E94010300E3FE
:103EB0000E94010308E70E9401030091B3020E94DF
:103EC0004C420091B4020E944C420091B5020E9403
:103ED0004C420091B6020E944C4200E20E94010353
:103EE00001E60E9401030CE60E94010304E70E9420
:103EF00001030DE30E94010300E30E94010308E7B0
:103F00000E9401030091B7020E944C420091B80246
:103F10000E944C420091B9020E944C420091BA02A8
:103F20000E944C4200E20E94010304E70E94010348
:103F30000DE30E94010300E30E94010308E70E94D1
:103F400001030091AF020E944C420091B0020E9416
:103F50004C420091B1020E944C420091B2020E9478
:103F60004C4200E20E94010302E70E9401030DE3BC
:103F70000E94010300E30E94010308E70E9401037D
:103F800000919B020E944C4200919C020E944C4274
:103F900000E20E94010304E60E9401030DE30E9477
:103FA000010300E30E94010308E70E94010300915E
:103FB0009D020E944C4200919E020E944C420DE0E4
:103FC0000E940103089501E60E9401030AE70E948E
:103FD00001030DE30E94010300E30E94010308E7CF
:103FE0000E9401030091E3020E944C420091E4020E
:103FF0000E944C420091E5020E944C420091E60270
:104000000E944C4200E20E94010301E60E9401036B
:104010000CE60E94010304E70E9401030DE30E94E5
:10402000010300E30E94010308E70E9401030091DD
:10403000E7020E944C420091E8020E944C4200912B
:10404000E9020E944C420091EA020E944C4200E2C6
:104050000E94010304E70E9401030DE30E94010393
:1040600000E30E94010308E70E9401030091DF02C0
:104070000E944C420091E0020E944C420091E102F9
:104080000E944C420091E2020E944C4200E20E94D7
:10409000010302E70E9401030DE30E94010300E314
:1040A0000E94010308E70E9401030091CB020E94D5
:1040B0004C420091CC020E944C4200E20E9401035B
:1040C00004E60E9401030DE30E94010300E30E9445
:1040D000010308E70E9401030091CD020E944C42B7
:1040E0000091CE020E944C420DE00E94010308950F
:1040F0000E949C422EF5F8948092B3069092B406EA
:10410000A092B506B092B60678940E949C42C6F47E
:10411000F8948092EA069092EB06A092EC06B09298
:10412000ED0678940E949C425EF4F89480925608C2
:1041300090925708A0925808B092590878946894C1
:104140000895E4E6FDE00E946814A2E5B5E00E944F
:10415000A614AAE6B5E00E94A614A2E7B5E00E9464
:10416000A61400E010E9ABE6B2E00D931A95E9F76A
:1041700000E00093FB020093FC020093FD0200E0CC
:104180000093FE0200E000935004089500E010E068
:1041900029EF3DEA00938302109384022093850265
:1041A000309386020FEF1FEF2CEF3DE7009387025D
:1041B000109388022093890230938A0200E010E075
:1041C00024E030E000937F0210938002209381026C
:1041D000309382020AE11FEA00936B0210936C0293
:1041E0000DE717E800936D0210936E0200E01DE4E6
:1041F0002EEB37E70093B3021093B4022093B5027D
:104200003093B6020FEF19EE2BEC33E90093B702AF
:104210001093B8022093B9023093BA0200E010E084
:104220002DE530E00093AF021093B0022093B1026D
:104230003093B2020AE610EF00939B0210939C02A7
:1042400000E114ED00939D0210939E0201E00093A3
:10425000FB020093FC0208953F196B0F1FBF73848C
:104260003F096B0F1FBF73840091FB02013091F572
:104270005524662470906B0280906C020E94740832
:104280000E941414E8E5F2E40E9468140E94070CEE
:10429000AFE6B2E00E94A61450906D0260906E02EC
:1042A0000E9446080E941414E0E6F2E40E9468149A
:1042B0000E94070CA7E7B2E00E94A61402E01FE6E6
:1042C00023E037E40E94B02402E00093FB020027C1
:1042D0000093FE020091FC02013009F036C0552423
:1042E000662470909B0280909C020E9474080E9439
:1042F0001414E8E5F2E40E9468140E94070CAFE988
:10430000B2E00E94A61450909D0260909E020E940E
:1043100046080E941414E0E6F2E40E9468140E9429
:10432000070CA7EAB2E00E94A61402E01FE923E00E
:104330003FE50E94B02403E017E40E94952502E0C7
:104340000093FC0200270093FE020091FB02023062
:1043500021F40091FC02023009F008950091FE0260
:104360000023D9F700916902002311F0C8D0C6F0EC
:1043700002E013E822E03BE80E94282502E013E86F
:1043800022E03FEF0E94D92E02E013EB22E03BEB4C
:104390000E94282502E013EB23E037E10E94D92E8A
:1043A00002E01FEF0E94952502E01FEF23E037E1B6
:1043B0000E94260E0E94141403E017E423E03FE558
:1043C0000E94260E0E94130B02E01FEF22E03FEF37
:1043D0000E94260E03E017E123E037E10E94260E3B
:1043E00003E01FE223E03FE20E94260E02E01FEFFF
:1043F00023E03FE20E94260E03E017E123E03FE2C4
:104400000E94260E03E017E423E037E40E94260E04
:1044100003E01FE523E03FE50E94260E03E017E7D7
:1044200023E037E70E94260E03E017E423E037E796
:104430000E94260E03E01FE523E037E70E94260EC8
:1044400002E01FEF21E03FEC0E940B1002E01FEFA3
:1044500021E03FEC43E05FE80E94CF0F03E017E468
:1044600021E03FEC43E05FE80E94CF0F03E01FE84C
:1044700023E037ED0E940B1003E01FE823E037ED47
:1044800041E05FEC0E94CF0F03E01FE822E03FEF26
:1044900041E05FEC0E94960F03E01FE823E037E164
:1044A00041E057EE0E94960F03E01FE823E03FE251
:1044B00041E05FEF0E94960F03E017ED23E037E441
:1044C00041E05FEC0E94960F03E017ED23E03FE52B
:1044D00041E057EE0E94960F03E017ED23E037E727
:1044E00041E05FEF0E94960F01E00093FE0200E0C2
:1044F0000093C80408953FEF838B8C811C17CF93E2
:10450000DF93CDB7DEB7CA53D040F894CDBFDEBF3E
:10451000789400E000936A02A2E5B5E00E9454148A
:10452000AC2FBD2FAF5FBF4F0E94A614E4E6FDE0A5
:104530000E946814A2E5B5E00E94A61402E013E808
:1045400022E03BE80E94282502E013E822E03FEF4A
:104550000E94D92E02E013EB22E03BEB0E942825BB
:1045600002E013EB23E037E10E94D92EE4E6FDE000
:104570000E946814AFE0B3E00E94A614A7E2B3E083
:104580000E94A61402E01FEF98010E94F70E7EF031
:1045900001E000936A02AC2FBD2FAF5FBF4F0E94B6
:1045A0005414A2E5B5E00E94A614E894ADC103E05E
:1045B00017E198010E94F70E7EF002E000936A0274
:1045C000AC2FBD2FAF5FBF4F0E945414A2E5B5E0E2
:1045D0000E94A614E89498C102E01FEF23E037E19F
:1045E0000E94260E0E941414E6EFF4E40E94681460
:1045F0000E94130B4420DAF003E000936A02EEE11C
:10460000F6E40E94C547AC2FBD2FAF5FBF4F0E949D
:104610005414A2E5B5E00E94A614E89475C1457251
:10462000726F72203033417A20536570202003E08E
:1046300017E423E03FE50E94260EAC2FBD2FA75FB5
:10464000BF4F0E94A614AFE3B4E00E94A614442416
:104650000E941414E6EFF4E40E9468140E94130B05
:104660004420DAF004E000936A02EAE8F6E40E94EB
:10467000C547AC2FBD2FAF5FBF4F0E945414A2E5BA
:10468000B5E00E94A614E8943FC14572726F722093
:1046900030345472756520536570A3E9B2E00E940E
:1046A00054140E941414A3ECB2E00E9454140E940B
:1046B000130B44206AF1ECEBFDE00E9468140E94A9
:1046C0001414A3E9B2E00E9454140E94130BAC2FFF
:1046D000BD2FAF5EBF4F0E94A614A7E2B4E00E94B8
:1046E000A614E4E6FDE00E9468140E941414A3ECF2
:1046F000B2E00E9454140E94130BAC2FBD2FA75E92
:10470000BF4F0E94A614AFE1B4E00E94A6142CC0D3
:10471000ECEBFDE00E9468140E941414A3ECB2E0DC
:104720000E9454140E94130BAC2FBD2FAF5EBF4FDD
:104730000E94A614A7E2B4E00E94A614E4E6FDE0FD
:104740000E9468140E941414A3E9B2E00E94541459
:104750000E94130BAC2FBD2FA75EBF4F0E94A61463
:10476000AFE1B4E00E94A614AC2FBD2FA75EBF4FEF
:104770000E945414A2E5B5E00E94A614CED0AFE288
:10478000B4E00E94A6140E941414AC2FBD2FA75FA2
:10479000BF4F0E9454140E94130BAC2FBD2FA75D76
:1047A000BF4F0E94A614AC2FBD2FAF5EBF4F0E941B
:1047B0005414A2E5B5E00E94A614AFD0A7E3B4E07C
:1047C0000E94A6140E941414AC2FBD2FA75FBF4FE8
:1047D0000E9454140E94130BAC2FBD2FAF5DBF4F2E
:1047E0000E94A6144F92AC2FBD2FA75DBF4F0E9411
:1047F00054140F9104250023EAF005E000936A02A7
:10480000AC2FBD2FAF5FBF4F0E945414A2E5B5E09F
:104810000E94A614E0E2F8E40E94C547E89474C040
:104820004572726F722030353F3F3F3F3F3F3F3F01
:104830000CE009AFAC2FBD2FA75EBF4F0E945414F0
:104840000E941414AC2FBD2FAF5EBF4F0E945414B2
:104850000E94150B01E0201A00E0300AA2E5B5E045
:104860000E94A6145AD00E941414AC2FBD2FA75F2B
:10487000BF4F0E9454140E94130BAC2FBD2FAF5C8E
:10488000BF4F0E94A6144F92AC2FBD2FA75DBF4F04
:104890000E9454140F9104250023BAF0A2E5B5E05C
:1048A0000E945414AC2FBD2FA75EBF4F0E94A614C8
:1048B000AC2FBD2FAF5CBF4F0E945414AC2FBD2F47
:1048C000A75DBF4F0E94A61416C0A2E5B5E00E94E6
:1048D0005414AC2FBD2FAF5EBF4F0E94A614AC2F57
:1048E000BD2FAF5CBF4F0E945414AC2FBD2FAF5DE6
:1048F000BF4F0E94A61409AD0A9509AF09F09ACFDF
:1049000003E600936A026894C65CDF4FF894CDBF5B
:10491000DEBF7894DF91CF91089502E013E822E0A2
:104920003BE80E94282502E013E822E03FEF0E94C6
:10493000D92E02E013EB22E03BEB0E94282502E097
:1049400013EB23E037E10E94D92E02E01FEF23E0B2
:1049500037E10E94260E08953EA31DA7F687272C57
:10496000CF93DF93CDB7DEB7C551D040F894CDBF1C
:10497000DEBF789409831A832B833C83B981AA8193
:1049800018960E9454140E94B317AC2FBD2FAB5F32
:10499000BF4F0E94A614B981AA8150965D906D9078
:1049A0007D908D900E9474080E941414E8E5F9E44B
:1049B0000E9468140E94070C00E840260E9414140C
:1049C000B981AA810E9454140E94150BAC2FBD2FEF
:1049D000A35FBF4F0E94A6140E94B3170E94141435
:1049E000AC2FBD2FAB5FBF4F0E9454140E94070C29
:1049F000BB81AC810E94A614AC2FBD2FA35FBF4F1B
:104A00000E9454140E9402180E941414AC2FBD2F4F
:104A1000AB5FBF4F0E9454140E94070CBB81AC8156
:104A200018960E94A614B981AA8118960E9454145F
:104A30000E940218BB81AC8150960E94A614CB5EE6
:104A4000DF4FF894CDBFDEBF7894DF91CF9108950A
:104A5000CF93DF93CDB7DEB7C550D040F894CDBF2C
:104A6000DEBF789409831A832B833C83B981AA81A2
:104A70005D906D907D908D900E9474080E9414143A
:104A8000AAE2B5E00E9454140E94070C44204AF4A4
:104A90000E941414E4EDFDE00E9468140E94150BBE
:104AA000F5CFBB81AC8110960E94A6140E9414140D
:104AB000E4EDFDE00E9468140E94130B442032F0E4
:104AC000BB81AC8110960E94A614F0CFB981AA8157
:104AD00014965D906D907D908D900E9474080E9458
:104AE0001414A2E3B5E00E9454140E94070C0E9423
:104AF0001414AAE3B5E00E9454140E94150B0E94FE
:104B00001414A2E5B5E00E9454140E94150BBB8159
:104B1000AC8118960E94A614CB5FDF4FF894CDBFEE
:104B2000DEBF7894DF91CF910895CF93DF93CDB717
:104B3000DEB7CF50D040F894CDBFDEBF7894098364
:104B40001A83B02FA12F5896BB83AC835896BD8390
:104B5000AE83B981AA8118960E9454140E9414143D
:104B6000BB81AC8150960E9454140E94070C0E9495
:104B70001414B981AA8150960E9454140E941414EE
:104B8000BB81AC8118960E9454140E94070C0E94AD
:104B9000130BBD81AE8110960E94A614B981AA8123
:104BA00050960E9454140E941414BB81AC8110963C
:104BB0000E9454140E94070C0E941414B981AA8107
:104BC00010960E9454140E941414BB81AC8150961C
:104BD0000E9454140E94070C0E94130BBD81AE81E9
:104BE00018960E94A614B981AA8110960E945414A6
:104BF0000E941414BB81AC8118960E9454140E9428
:104C0000070C0E941414B981AA8118960E945414AA
:104C10000E941414BB81AC8110960E9454140E940F
:104C2000070C0E94130BBD81AE8150960E94A61402
:104C30000D811E81202F312F0E94260E0E94C91443
:104C4000AC2FBD2FA95FBF4F0E94A614BD81AE81BE
:104C500010960E9454140E941414AC2FBD2FA95F0B
:104C6000BF4F0E9454140E94A30DBD81AE811096C7
:104C70000E94A614BD81AE8118960E9454140E9411
:104C80001414AC2FBD2FA95FBF4F0E9454140E9473
:104C9000A30DBD81AE8118960E94A614BD81AE8180
:104CA00050960E9454140E941414AC2FBD2FA95F7B
:104CB000BF4F0E9454140E94A30DBD81AE81509637
:104CC0000E94A614C15FDF4FF894CDBFDEBF789479
:104CD000DF91CF91089500904704002009F40895D2
:104CE0000A951AF4009150040E5FE1E5F2E018E134
:104CF000019FE00DF11D11E00030D9F4B2E0A3E80E
:104D000004E00E94CE04B2E0A7E804E00E94CE04D2
:104D1000B2E0AFE704E00E94CE04B2E0ABE602E00E
:104D20000E94CE04B2E0ADE602E00E94CE0447D07D
:104D300045C00130D9F4B2E0A3EB04E00E94CE04F8
:104D4000B2E0A7EB04E00E94CE04B2E0AFEA04E0D8
:104D50000E94CE04B2E0ABE902E00E94CE04B2E0D1
:104D6000ADE902E00E94CE042AD028C0063634F510
:104D7000B2E0A3EE04E00E94CE04B2E0A7EE04E0AD
:104D80000E94CE04B2E0AFED04E00E94CE04B2E097
:104D9000ABEC02E00E94CE04B2E0ADEC02E00E9477
:104DA000CE040DD03C960FEF0E94BD0431960E94B8
:104DB000BD04009150040395009350040895AEE99A
:104DC000B8E011E008E00C94CE04CF93DF93CDB7A8
:104DD000DEB7C859D040F894CDBFDEBF7894E4E682
:104DE000FDE00E946814A8E4B4E00E94A614F2E07A
:104DF000E1E8FA83EB83FA81EB813C960E94C704D9
:104E00000F3F31F431960E94C7040F3F09F4D1C01F
:104E1000FA81EB81DE01589610E004E00E94CE0496
:104E2000DE015C9610E004E00E94CE04DE015496A0
:104E300010E004E00E94CE04552466240E94C704BA
:104E4000702E31960E94C704802E3196FA83EB8330
:104E50000E9474080E941414E8E5F2E40E946814A9
:104E60000E94070CAC2FBD2FAC5FBF4F0E94A61451
:104E7000FA81EB810E94C704502E31960E94C7042C
:104E8000602E3196DE01D09610E008E00E94CE043C
:104E9000FA83EB830E9446080E941414E0E6F2E4D1
:104EA0000E9468140E94070CAC2FBD2FA45FBF4F57
:104EB0000E94A61400E018E11C0F0D1F20E030E254
:104EC0003C0F2D1F0E942825AC2FBD2FA05EBF4F89
:104ED0000E945414AC2FBD2FA85DBF4F0E945414E4
:104EE00000E018E11C0F0D1F20E038E33C0F2D1FE0
:104EF0000E94D92E03E01FE820E038E33C0F2D1F6D
:104F000040E050E55C0F4D1F0E94960F00E014E05A
:104F10001C0F0D1F20E038E63C0F2D1F0E94B0240F
:104F200000E010E51C0F0D1F20E038E63C0F2D1FA0
:104F300040E050E85C0F4D1F0E946F0E00E010E84B
:104F40001C0F0D1F20E030E83C0F2D1F0E94260E85
:104F50000E94C9140E941414E4EFFDE00E9468143A
:104F60000E94070C18E0DE01D0960D910E9401030B
:104F70001A95D9F700E20E9401030AE30E94010397
:104F800000E20E9401030E94AA090DE00E940103B1
:104F90000E9414140E94070C0E941414A8E4B4E0A8
:104FA0000E9454140E94150BA8E4B4E00E94A614B9
:104FB00022CF5524609050046620F1F00E944608EC
:104FC0000E941414A8E4B4E00E9454140E94321405
:104FD0000E94A30D0E94C914A8E4B4E00E94A61484
:104FE0000DE00E940103EEE3F1E00E94F5020E9451
:104FF000AA090DE00E940103C856DF4FF894CDBF07
:10500000DEBF7894DF91CF91689408958B28154383
:1050100043414C4320202020202051044243415A48
:10502000535445505320202055044243414C54537F
:1050300054455053202059044343415A524144207F
:105040002020202061044343414C545241442020FD
:105050002020690443434D4E5456454320202020D0
:1050600081044343534B5956454320202020990443
:10507000434352454354202020202020A104434391
:105080004445434C202020202020A9044243544979
:105090004D4520202020202000000000E4E6FDE017
:1050A0000E946814A9E9B4E00E94A614A1EAB4E041
:1050B0000E94A61401E00093C304089500E015E2E5
:1050C0002BEF3FEA009351041093520420935304B2
:1050D0003093540400E018E027E13DE100935504CB
:1050E00010935604209357043093580400E011E0C5
:1050F00021E830E00093A9041093AA042093AB04A4
:105100003093AC04089540A1E7A9907E593B40AA92
:10511000DB7E58BD85D80FB7F8940090B306109089
:10512000B4062090B5063090B6064090EA0650903E
:10513000EB066090EC067090ED068090560890901B
:105140005708A0905808B09059080FBF009251041A
:105150001092520420925304309254044092550409
:105160005092560460925704709258048092A90499
:105170009092AA04A092AB04B092AC0404E011E5B2
:1051800024E039E50E94282504E011E524E039E611
:105190000E94D92E0091FE02002371F400271127EE
:1051A000B4E0A1EB64D000271127B4E0AAEB90D0C3
:1051B00000E00093C80408950091FE020E94123797
:1051C00003E01FE824E039E644E051E80E94960F2E
:1051D00004E011E824E039E9BCD0A9E9B4E00E9478
:1051E00054140E941414E6E0F1E50E9468140E9431
:1051F000070C0E94AC075092AD046092AE04A1EA85
:10520000B4E00E9454140E941414EEE0F1E50E94F0
:1052100068140E94070C0E94AC075092AF04609281
:10522000B0040091C804003099F4A9E9B4E00E94E8
:105230005414A5EDB4E00E94A614A1EAB4E00E94C3
:105240005414ADEDB4E00E94A61402E00093C8042B
:105250000091AD041091AE04B4E0A1EB08D0009130
:10526000AF041091B004B4E0AAEB32D008952F93AC
:105270003F93EF93FF939801E6ECF2E509E010E02D
:105280000E94F0048901103428E3020710F0105442
:105290000843119627E130E74CD0119622E038E51B
:1052A00048D0129620E034E644D0119620E03AE04F
:1052B00040D0129620E031E040E33BD0FF91EF91E7
:1052C0003F912F9108952030303A30302E30000039
:1052D0002F933F93EF93FF939801E8E2F3E509E002
:1052E00010E00E94F00489014BE2002332F4109593
:1052F00000952FEF121B020B4DE223D022E038E580
:10530000119617D020E03CE3119613D020E03AE04C
:1053100040E312960ED020E031E011960AD0FF91C2
:10532000EF913F912F9108952B30303A303020206B
:10533000000040E34395131B020BE0F74A95130F5F
:10534000021F5C914C93451719F041E04093C30450
:105350000895CF93DF93CDB7DEB7C650D040F89411
:10536000CDBFDEBF789409831A832B833C83B98138
:10537000AA8118960E9454140E941414B981AA811B
:1053800010960E9454144D820E94A30D0E943A165A
:105390000D80002042F40E941414E4EBFDE00E9412
:1053A00068140E94130B0E941414BB81AC815096A8
:1053B0005D906D907D908D900E9474080E941414F1
:1053C000E8E5F9E40E9468140E94070C0E94150B9E
:1053D0000E941414E4EDFDE00E9468140E947E1304
:1053E00076F00E9423140E94E4125EF40E941414CA
:1053F000E4EDFDE00E9468140E94150B02C00E94BB
:10540000130BBB81AC8110960E94A614B981AA81AE
:1054100010960E9454140E9414140E94070C0E94BB
:105420001414B981AA8118960E9454140E9414146D
:105430000E94070C0E94150B0E94C9140E941414AC
:10544000B981AA8150960E9454140E9432140E947D
:10545000A30D0E943A16BB81AC8118960E94A61437
:10546000CA5FDF4FF894CDBFDEBF7894DF91CF9154
:105470000895A22A155443414C4320202020202087
:10548000C4044254434F554E544552202020C80472
:10549000405453544154555320202020190543545F
:1054A000415A202020202020202021054354414C17
:1054B0005420202020202020C9044254415A535413
:1054C000455053202020CD044254414C5453544560
:1054D00050532020010543544D4E5456454320203F
:1054E0002020E9044354534B5956454320202020A3
:1054F000D104415452454354494E54202020D304F2
:1055000041544445434C494E54202020D504435433
:1055100052454354202020202020DD04435444459C
:10552000434C202020202020E504425454494D457E
:105530002020202020200000000000E00093C8046C
:1055400001C00895CF93DF93CDB7DEB7C952D040E5
:10555000F894CDBFDEBF78940091C804003091F478
:1055600000E00093A3060093A4060093A506009311
:10557000A6060093DA060093DB060093DC06009390
:10558000DD062BC20091C804013049F5552466247C
:105590007090D1048090D2040E9474080E94141468
:1055A000E8E5F2E40E9468140E94070CA5EDB4E05F
:1055B0000E94A6145090D3046090D4040E94460820
:1055C0000E941414E0E6F2E40E9468140E94070CA2
:1055D000ADEDB4E00E94A61402E00093C80400916F
:1055E000C804023009F0F9C10091FD02002309F45A
:1055F00049C0E4E6FDE00E946814AAE6B5E00E9416
:10560000A614A2E7B5E00E94A6142090DF02309015
:10561000E0024090E1025090E2022092E5043092D4
:10562000E6044092E7045092E80455246624709002
:10563000CB028090CC020E9474080E941414E8E50A
:10564000F2E40E9468140E94070CA5EDB4E00E94E9
:10565000A6145090CD026090CE020E9446080E948F
:105660001414E0E6F2E40E9468140E94070CADED09
:10567000B4E00E94A61402E013EE22E03BEE0E948A
:10568000282519C0F8942090A9043090AA044090CD
:10569000AB045090AC04789400E010E80024510E64
:1056A000401E301C201C2092E5043092E6044092FB
:1056B000E7045092E80404E015ED24E039EE0E947E
:1056C000B02403E017ED24E039EE45E051E00E94FC
:1056D000960F05E011E025E039E10E94D22F0091FC
:1056E000FD02002321F1ABEEB2E00E9454140E94AF
:1056F0001414A9E1B5E00E9454140E94130BAAE609
:10570000B5E00E94A614A3EFB2E00E9454140E94D8
:105710001414A1E2B5E00E9454140E94130BA2E7F6
:10572000B5E00E94A61400270093FD0256C1A9E12E
:10573000B5E00E9454140E941414A9E5B4E00E943C
:1057400054140E94130BAC2FBD2FAF5DBF4F0E94AE
:10575000A6140E941414E4EBFDE00E9468140E9459
:10576000130B4420AAF0AC2FBD2FAF5DBF4F0E949A
:1057700054140E941414E4EDFDE00E9468140E9489
:10578000130BAC2FBD2FAF5DBF4F0E94A6141EC0E0
:105790000E941414E4EDFDE00E9468140E94150BB1
:1057A0004420A2F4AC2FBD2FAF5DBF4F0E94541414
:1057B0000E941414E4EDFDE00E9468140E94150B91
:1057C000AC2FBD2FAF5DBF4F0E94A614AC2FBD2FD5
:1057D000AF5DBF4F0E9454140E941414AAE2B5E0BA
:1057E0000E9454140E94A30D00E1200E0027301ED9
:1057F0000E941414E8E9F2E70E9468140E94A30DC5
:10580000AC2FBD2FAF5EBF4F0E94A614A1E2B5E042
:105810000E9454140E941414AAE3B5E00E94541488
:105820000E94130B0E941414A2E5B5E00E945414C8
:105830000E94130B0E941414A2E3B5E00E945414BA
:105840000E94A30D0E9414145090550460905604B9
:1058500070905704809058040E9474080E94130BA3
:1058600000E1200E0027301E0E941414E8E9F2E740
:105870000E9468140E94A30DAC2FBD2FA75EBF4FDE
:105880000E94A6145090930660909406709095061E
:10589000809096060E9474080E941414AC2FBD2FAD
:1058A000AF5EBF4F0E94541444240E94A30D0E9477
:1058B0001414ECE6FDE00E9468140E94E21316F056
:1058C0000E943214AC2FBD2FAF5FBF4F0E94A614B1
:1058D0000E9423145090CA066090CB067090CC06AC
:1058E0008090CD060E9474080E941414AC2FBD2F26
:1058F000A75EBF4F0E94541444240E94A30D0E942F
:105900001414ECE6FDE00E9468140E94E21316F005
:105910000E943214AC2FBD2FA75FBF4F0E94A61468
:105920000E942314AC2FBD2FAF5EBF4F0E945414B2
:105930000E941414AC2FBD2FAF5FBF4F0E945414B0
:105940000E94070C0E94F007F8945092A306609200
:10595000A4067092A5068092A6067894AC2FBD2F5F
:10596000A75EBF4F0E9454140E941414AC2FBD2F89
:10597000A75FBF4F0E9454140E94070C0E94F007BB
:10598000F8945092DA066092DB067092DC06809200
:10599000DD067894F894089411270091C704011F3C
:1059A0000093C7040091C604011F0093C604009130
:1059B000C504011F0093C5040091C404011F009396
:1059C000C4047894F8940091F1060A952AF00093A3
:1059D000F10600E00093C8047894C75DDF4FF894A7
:1059E000CDBFDEBF7894DF91CF910895EEE2FAE566
:1059F0000E946814AAE7B5E00E94A614E6E3FAE55F
:105A00000E946814A2E8B5E00E94A614EEE3FAE54D
:105A10000E946814A2E4B5E00E94A614E6E4FAE548
:105A20000E946814AAE4B5E00E94A61408953FE21B
:105A3000FD3B29A1B9FA3FF2B5BE5D9E40C800000A
:105A4000000000000000000000000000000005E071
:105A500012E725E03AE80C94DE2E05E012E725E097
:105A60003AE80C94542F05E01AE825E032EA0C9449
:105A7000D72F05E01AE825E032EA0C945330592E6E
:105A8000154E45575A31322020202020BA2E155A63
:105A900031202020202020202020BF2E155A322007
:105AA0002020202020202020F62C154D494E49543E
:105AB000202020202020272D154D52325620202036
:105AC00020202020332D154D56325220202020201A
:105AD00020202D2D154D5232564E202020202020E2
:105AE000392D154D5632524E2020202020202905D8
:105AF000404D5A315A324143542020202A05434D0B
:105B0000415A50535445502020203205434D414CBA
:105B100054505354455020203A05434D414C545362
:105B20005441525420204205434D5A312020202018
:105B3000202020204A05434D5A32202020202020BA
:105B400020205205434D5A332020202020202020A1
:105B50006A05434D415A4F4646534554202072052D
:105B6000434D414C544F4646534554207A05434DCE
:105B700054455354415A202020208205434D54451A
:105B80005354414C542020208A05434D54455354CE
:105B90005820202020209205434D5445535459202D
:105BA000202020209A05434D544553545A2020204C
:105BB0002020A205434D54455354415A52202020E1
:105BC000AA05434D54455354414C54522020B2052C
:105BD000434D54455354502020202020BA05434DB6
:105BE00054455354512020202020C205434D544594
:105BF0005354442020202020CA05434D544553547B
:105C0000413120202020D205434D54455354413288
:105C100020202020DA05434D5445535441332020A1
:105C20002020E205434D54455354415A582020202A
:105C3000EA05434D54455354415A59202020F2055A
:105C4000434D54455354434F53502020FA05434D80
:105C5000544553545058202020200206434D5445AB
:105C600053545059202020200A06434D5445535484
:105C7000505A202020201206434D54455354434F80
:105C8000534120202206434D54455354505832204E
:105C900020202A06434D5445535450593220202089
:105CA0003206434D54455354505A322020200000B0
:105CB00000000091FE02002329F4EAE9F5E00E94C9
:105CC000F5022FC00E949C4266F50E941414E4EB7A
:105CD000FDE00E9468140E94070C0E941414ECEE70
:105CE000FDE00E9468140E94A30DA2E4B5E00E94AA
:105CF000A6140E949C42AEF40E941414E4EBFDE052
:105D00000E9468140E94070C0E941414ECEEFDE03F
:105D10000E9468140E94A30DAAE4B5E00E94A61494
:105D200002C0E89408950091FB02003019F001E0F0
:105D30000093FB020091FC02003019F001E0009397
:105D4000FC0200270093FE0200E00093C8040E94BA
:105D500034210E948B280E94A22A0E94E526A8E4F2
:105D6000B4E00E9454140E94AA090DE00E940103AD
:105D700068940895A2E4B5E00E94541404C0AAE413
:105D8000B5E00E9454140E941414ECEEFDE00E9451
:105D900068140E94070C0E941414E4EBFDE00E94BA
:105DA00068140E94A30D0E94AA090DE00E9401033D
:105DB000089500902905002009F076C0CF93DF9365
:105DC000CDB7DEB7CD51D040F894CDBFDEBF7894CB
:105DD00009831A832B833C83B981AA8150960E9440
:105DE00054140E941414A2E7B5E00E9454140E94B7
:105DF000130B0E94B317AC2FBD2FAB5FBF4F0E9498
:105E0000A6140E941414B981AA8118960E945414F1
:105E10000E941414AAE6B5E00E9454140E94130BC9
:105E20000E94B3170E94070CBB81AC8110960E94A0
:105E3000A614AC2FBD2FAB5FBF4F0E9454140E941D
:105E40001414B981AA8118960E9454140E94141443
:105E5000AAE6B5E00E9454140E94130B0E94021897
:105E60000E94070CBB81AC8118960E94A614B981D0
:105E7000AA8150960E9454140E941414A2E7B5E01F
:105E80000E9454140E94130B0E940218BB81AC8123
:105E900050960E94A614C35EDF4FF894CDBFDEBFBC
:105EA0007894DF91CF910895CF93DF93CDB7DEB78C
:105EB000CD51D040F894CDBFDEBF789409831A83CA
:105EC0002B833C83ECE6FDE00E946814BB81AC812F
:105ED00010960E94A614E4E6FDE00E946814BB81BF
:105EE000AC8118960E94A614BB81AC8150960E948A
:105EF000A614AAE4B5E00E94541401E01FEC0E942D
:105F0000801201E01FEC2B813C81A9010E94960FB9
:105F1000B981AA8150960E9454140E941414A2E7D9
:105F2000B5E00E9454140E94130B00E8402601E0E3
:105F30001FEC0E94241201E01FEC2B813C81A9017F
:105F40000E94960FA2E4B5E00E94541401E01FECF9
:105F50000E94C81101E01FEC2B813C81A9010E9425
:105F6000960FB981AA8118960E9454140E941414A5
:105F7000AAE6B5E00E9454140E94130B01E01FEC46
:105F80000E94801201E01FEC2B813C81A9010E943C
:105F9000960FC35EDF4FF894CDBFDEBF7894DF91DC
:105FA000CF91089500902905002009F07CC0CF937F
:105FB000DF93CDB7DEB7C650D040F894CDBFDEBF7B
:105FC000789409831A832B833C83B981AA8118961C
:105FD0000E9454140E941414B981AA8110960E9440
:105FE00054144D820E94A30D0E943A160E9414146C
:105FF000AAE6B5E00E9454140E94150B0D80002003
:1060000042F40E941414E4EBFDE00E9468140E9424
:10601000130B442042F40E941414E4EDFDE00E94AE
:1060200068140E94150BBB81AC8110960E94A614C7
:10603000B981AA8110960E9454140E9414140E94DF
:10604000070C0E941414B981AA8118960E94541456
:106050000E9414140E94070C0E94150B0E94C91480
:106060000E941414B981AA8150960E9454140E946F
:1060700032140E94A30D0E943A160E941414A2E743
:10608000B5E00E9454140E94150BBB81AC81189698
:106090000E94A614CA5FDF4FF894CDBFDEBF78948C
:1060A000DF91CF910895CF93DF93CDB7DEB7C0587E
:1060B000D040F894CDBFDEBF789409831A832B8338
:1060C0003C83A2E4B5E00E9454140E940218AAE5A1
:1060D000B5E00E94A614AAE4B5E00E9454140E9400
:1060E0000218A2E6B5E00E94A614B981AA81109612
:1060F0000E9454140E941414A2E6B5E00E945414A5
:106100000E94070C0E941414B981AA8110960E9463
:1061100054140E941414AAE5B5E00E9454140E947D
:10612000070C0E941414B981AA8150960E9454143D
:106130000E94070C0E94130B0E941414ECE7FDE070
:106140000E9468140E94070C0E941414B981AA814D
:1061500010960E9454140E9414140E94070C0E946E
:106160001414B981AA8118960E9454140E94141420
:106170000E94070C0E94150BAC2FBD2FA85EBF4FCD
:106180000E94A6140E94A30DAC2FBD2FA85FBF4F85
:106190000E94A614A2EBB5E00E94A614B981AA81C0
:1061A00018960E9454140E9414140E94070C0E9416
:1061B0001414AAE5B5E00E9454140E9414140E941D
:1061C000070C0E941414ECE6FDE00E9468140E9483
:1061D000130B0E94070C0E941414B981AA815096D7
:1061E0000E9454140E9414140E94070C0E9414145C
:1061F000AAE5B5E00E9454140E9414140E94070CF2
:106200000E94070C0E94150B0E941414B981AA81E8
:1062100050960E9454140E941414AAE5B5E00E94FE
:1062200054140E94070C0E941414A2E6B5E00E94C8
:1062300054140E94070C0E941414ECE7FDE00E9425
:1062400068140E94070C0E94130B0E941414A2E60B
:10625000B5E00E9454140E9414140E94070C0E947E
:10626000150B0E941414AC2FBD2FA85EBF4F0E94C7
:1062700054140E94A30DAC2FBD2FA05FBF4F0E94EE
:10628000A614AAEBB5E00E94A614AC2FBD2FA85F00
:10629000BF4F0E9454140E9414140E94070C0E94C5
:1062A0001414ECEAFDE00E9468140E94070C0E949E
:1062B0001414AC2FBD2FA05FBF4F0E9454140E9436
:1062C000130BA2ECB5E00E94A614442012F4E8944B
:1062D00042C20E94C914AC2FBD2FA05EBF4F0E94C6
:1062E000A61402E00D83AC2FBD2FA85FBF4F0E9404
:1062F000541400E840260E941414E4EAFDE00E94D1
:1063000068140E94070C0E941414AC2FBD2FA05ECD
:10631000BF4F0E9454140E94150BAC2FBD2FA85DD7
:10632000BF4F0E94A614AAECB5E00E94A614AC2FA1
:10633000BD2FA85BBF4F0E94A614AAEEB5E00E9435
:10634000A614B981AA8150960E9454140E94141474
:10635000AAE5B5E00E9454140E94070C0E94141490
:10636000B981AA8110960E9454140E941414AC2F73
:10637000BD2FA85DBF4F0E9454140E94070C0E94BD
:10638000130B0E941414A2E6B5E00E9454140E945C
:10639000130B0E941414B981AA8118960E945414F8
:1063A0000E94A30DAC2FBD2FA05DBF4F0E94A6146D
:1063B000A2EDB5E00E94A61400E84026AC2FBD2F48
:1063C000A05CBF4F0E94A614A2EEB5E00E94A614E6
:1063D000AAE5B5E00E94541400E84026AC2FBD2F7A
:1063E000A85CBF4F0E94A614AAEDB5E00E94A614B7
:1063F000B981AA8110960E9454140E941414AC2FE3
:10640000BD2FA85DBF4F0E9454140E94070C0E942C
:106410001414B981AA8118960E9454140E9414146D
:10642000AC2FBD2FA05DBF4F0E9454140E94070CDB
:106430000E94150B0E941414B981AA8150960E94E3
:1064400054140E941414AC2FBD2FA85CBF4F0E949F
:1064500054140E94070C0E94150BAC2FBD2FA05B9B
:10646000BF4F0E94A614A2EFB5E00E94A614B98106
:10647000AA8110960E9454140E941414AC2FBD2FB0
:10648000A05BBF4F0E9454140E941414AC2FBD2F68
:10649000A85DBF4F0E9454140E94070C0E94130B6A
:1064A000AC2FBD2FA85ABF4F0E94A614AAEFB5E08B
:1064B0000E94A614B981AA8118960E9454140E94C1
:1064C0001414AC2FBD2FA05BBF4F0E9454140E9428
:1064D0001414AC2FBD2FA05DBF4F0E9454140E9416
:1064E000070C0E94130BAC2FBD2FA05ABF4F0E9468
:1064F000A614A2E0B6E00E94A614AC2FBD2FA05CAB
:10650000BF4F0E9454140E941414AC2FBD2FA85AE0
:10651000BF4F0E9454140E94070C0E941414AC2F09
:10652000BD2FA85BBF4F0E9454140E941414AC2FBF
:10653000BD2FA05ABF4F0E9454140E94070C0E9406
:10654000150BAC2FBD2FA059BF4F0E94A614A2E17E
:10655000B6E00E94A6144420AAF40D810A950D838A
:1065600011F4E894F8C0AC2FBD2FA05EBF4F0E947D
:10657000541400E84026AC2FBD2FA05EBF4F0E94F0
:10658000A614B1CEB981AA8150960E9454140E94DB
:106590001414AC2FBD2FA05BBF4F0E9454140E9457
:1065A0001414AC2FBD2FA85CBF4F0E9454140E943E
:1065B000070C0E94130BAC2FBD2FA859BF4F0E9490
:1065C000A614AAE0B6E00E94A614AC2FBD2FA05CD2
:1065D000BF4F0E9454140E9414140E94070C0E9482
:1065E0001414AC2FBD2FA85BBF4F0E9454140E94FF
:1065F00014140E94070C0E94150B0E94C914AC2FA2
:10660000BD2FA858BF4F0E94A614AAE1B6E00E9471
:10661000A614AC2FBD2FA85BBF4F0E9454140E943C
:106620001414AC2FBD2FA05CBF4F0E9454144E8297
:106630000E94A30D0E943A160E80002042F40E9490
:106640001414E4EBFDE00E9468140E94130B442034
:1066500042F40E941414E4EDFDE00E9468140E94CC
:10666000150B0E941414AAE6B5E00E9454140E946F
:10667000150BBB81AC8110960E94A614A2EAB5E06E
:106680000E94A614BB81AC8110960E94541400E8AD
:10669000402601E01FEC0E94801201E01FEC2D2F2C
:1066A0003C2F385A2F4FA9010E94960FA2E4B5E063
:1066B0000E94541400E8402601E01FEC0E94C8111B
:1066C00001E01FEC2D2F3C2F385A2F4FA9010E94BB
:1066D000960FAC2FBD2FA85ABF4F0E945414A2E2B0
:1066E000B6E00E94A614AC2FBD2FA05ABF4F0E9447
:1066F0005414AAE2B6E00E94A614AC2FBD2FA859EC
:10670000BF4F0E945414A2E3B6E00E94A614AC2F1F
:10671000BD2FA859BF4F0E9454140E941414AC2FCF
:10672000BD2FA85ABF4F0E9454140E94A30D0E946F
:106730003A160E941414A2E7B5E00E9454140E9475
:10674000150BBB81AC8118960E94A614AAEAB5E08D
:106750000E94A6146894C058DF4FF894CDBFDEBFE6
:106760007894DF91CF910895B3341558474F544F23
:10677000202020202020C3341559474F544F20207B
:1067800020202020D334155859474F544F20202023
:1067900020206D34155852454620202020202020EE
:1067A00090341559524546202020202020202F3497
:1067B0001558595245462020202020203A0640589E
:1067C00059535441545553202020530643584D4D9E
:1067D00020202020202020205B0643594D4D2020E2
:1067E0002020202020203B0642583053544550534F
:1067F000202020203F06425930535445505320203A
:10680000202043064358304D4D20202020202020BA
:106810004B064359304D4D20202020202020630678
:1068200043585441524745544D4D20206B0643591F
:106830005441524745544D4D20200000000000E0D7
:1068400000933A06E4E6FDE00E946814A3E4B6E093
:106850000E94A614ABE4B6E00E94A61416C00E94E3
:106860009C42D6F5A3E4B6E00E94A614A3E5B6E0E8
:106870000E94A6140E949C427EF5ABE4B6E00E9402
:10688000A614ABE5B6E00E94A6140FB7F8940090EA
:10689000B3061090B4062090B5063090B60640902E
:1068A000EA065090EB066090EC067090ED060FBF84
:1068B00000923B0610923C0620923D0630923E0626
:1068C00040923F0650924006609241067092420606
:1068D00000E000933A06689408950E949C42FEF4FA
:1068E000A3E4B6E00E94A614A3E5B6E00E94A614B5
:1068F0000FB7F8940090B3061090B4062090B50638
:106900003090B6060FBF00923B0610923C062092D4
:106910003D0630923E0600E000933A0668940895E2
:106920000E949C42FEF4ABE4B6E00E94A614ABE5E4
:10693000B6E00E94A6140FB7F8944090EA06509073
:10694000EB066090EC067090ED060FBF40923F069C
:1069500050924006609241067092420600E0009319
:106960003A06689408950E949C4286F5A3E6B6E034
:106970000E94A614ABE5B6E00E945414ABE6B6E064
:106980000E94A6141EC00E949C4206F5ABE6B6E02B
:106990000E94A614A3E5B6E00E945414A3E6B6E054
:1069A0000E94A6140EC00E949C4286F4A3E6B6E0A4
:1069B0000E94A6140E949C424EF4ABE6B6E00E94F0
:1069C000A61401E000933A066894089500E000934D
:1069D0003A060895CF93DF93CDB7DEB7C952D040C2
:1069E000F894CDBFDEBF78940091F106002321F426
:1069F00000913A060030A9F400E00093A30600934A
:106A0000A4060093A5060093A6060093DA06009359
:106A1000DB060093DC060093DD0600E000933A06F7
:106A20002BC100913A06013009F026C10FB7F89446
:106A30005090B3066090B4067090B5068090B6068C
:106A40000FBF00903B0610903C0620903D06309012
:106A50003E0683187208610850080E9474080E945C
:106A60001414AAE2B5E00E9454140E94070C0E947C
:106A70001414A3E4B6E00E9454140E94150BA3E57D
:106A8000B6E00E94A6140FB7F8945090EA06609002
:106A9000EB067090EC068090ED060FBF00903F066D
:106AA00010904006209041063090420683187208EC
:106AB000610850080E9474080E941414A2E3B5E013
:106AC0000E9454140E94070C0E941414ABE4B6E018
:106AD0000E9454140E94150BABE5B6E00E94A61468
:106AE000A3E6B6E00E9454140E941414A3E5B6E095
:106AF0000E9454140E94130B0E941414AAE2B5E0E1
:106B00000E9454140E94A30D00E1200E0027301EA5
:106B10000E941414E8E9F2E70E9468140E94A30D91
:106B2000AC2FBD2FAF5EBF4F0E94A614ABE6B6E000
:106B30000E9454140E941414ABE5B6E00E94541451
:106B40000E94130B0E941414A2E3B5E00E94541497
:106B50000E94A30D00E1200E0027301E0E94141495
:106B6000E8E9F2E70E9468140E94A30DAC2FBD2F44
:106B7000A75EBF4F0E94A6145090930660909406A3
:106B800070909506809096060E9474080E941414D6
:106B9000AC2FBD2FAF5EBF4F0E94541444240E94FF
:106BA000A30D0E9414145090CA066090CB067090FA
:106BB000CC068090CD060E9474080E941414AC2F5D
:106BC000BD2FA75EBF4F0E94541444240E94A30D02
:106BD0000E94B01316F00E943214ECE6FDE00E9411
:106BE00068140E947E1316F00E943214AC2FBD2F41
:106BF000AF5FBF4F0E94A614AC2FBD2FA75FBF4F42
:106C00000E94A6140E942314AC2FBD2FAF5EBF4F6D
:106C10000E9454140E941414AC2FBD2FAF5FBF4FBD
:106C20000E9454140E94070C0E94F007F89450929E
:106C3000A3066092A4067092A5068092A606789498
:106C4000AC2FBD2FA75EBF4F0E9454140E94141496
:106C5000AC2FBD2FA75FBF4F0E9454140E94070C9A
:106C60000E94F007F8945092DA066092DB06709268
:106C7000DC068092DD067894C75DDF4FF894CDBFC7
:106C8000DEBF7894DF91CF910895F106404D4F54C7
:106C90004E4F545A45524F20B306424D4F54415027
:106CA0004F5320202020AF06424D4F5441535020D7
:106CB000202020209706424D4F54414853535020E6
:106CC00020209B06424D4F54414853502020202005
:106CD0009F06424D4F544148414343202020A30684
:106CE000424D4F544147535350202020A706424D58
:106CF0004F544147535020202020AB06424D4F5463
:106D000041474143432020207306424D4F54415395
:106D10005350312020207706424D4F544153535059
:106D2000322020207B06424D4F5441535350332094
:106D300020207F06424D4F54415353503420202091
:106D40009306424D4F544153535035202020B906ED
:106D5000404D4F5441494E5645525420EA06424D4B
:106D60004F5442504F5320202020E606424D4F54AE
:106D70004253502020202020CE06424D4F544248FE
:106D8000535350202020D206424D4F544248535076
:106D900020202020D606424D4F54424841434320F4
:106DA0002020DA06424D4F544247535350202020B2
:106DB000DE06424D4F544247535020202020E20629
:106DC000424D4F544247414343202020BA06424D92
:106DD0004F544253535031202020BE06424D4F5451
:106DE0004253535032202020C206424D4F5442534A
:106DF000535033202020C606424D4F544253535027
:106E000034202020CA06424D4F544253535035205F
:106E10002020F006404D4F5442494E5645525420D2
:106E200000000000CF93DF93CDB7DEB7C151D04053
:106E3000F894CDBFDEBF7894FF24001241C00090CB
:106E400073060092830600907406009284060090F8
:106E500075060092850600907606009286060090E0
:106E600077060092870600907806009288060090C8
:106E700079060092890600907A0600928A060090B0
:106E80007B0600928B0600907C0600928C06009098
:106E90007D0600928D0600907E0600928E06009080
:106EA0007F0600928F060090800600929006009068
:106EB0008106009291060090820600929206E7C039
:106EC000A1E6B4E00E9454140E941414E0EAF0E732
:106ED0000E9468140E944C1316F00E9432140E9403
:106EE00023140E94B3170E941414ECE6FDE00E94E4
:106EF00068140E9432140E94A30DAC2FBD2FAF5F07
:106F0000BF4F0E94A6145090930660909406709014
:106F10009506809096060E947408AC2FBD2FA75F3F
:106F2000BF4F0E94A6145090730660907406709034
:106F30007506809076060E9474080E941414AC2F87
:106F4000BD2FAF5FBF4F0E9454140E94070C0E94D8
:106F50001414AC2FBD2FA75FBF4F0E9454140E9482
:106F6000B01316F00E9432140E9423140E94F007FE
:106F700050928306609284067092850680928606FF
:106F800050907706609078067090790680907A0627
:106F90000E9474080E941414AC2FBD2FAF5FBF4F26
:106FA0000E9454140E94070C0E941414AC2FBD2F91
:106FB000A75FBF4F0E9454140E94B01316F00E94A6
:106FC00032140E9423140E94F007509287066092A8
:106FD00088067092890680928A0650907B0660909F
:106FE0007C0670907D0680907E060E9474080E9448
:106FF0001414AC2FBD2FAF5FBF4F0E9454140E94DA
:10700000070C0E941414AC2FBD2FA75FBF4F0E9426
:1070100054140E94B01316F00E9432140E942314DC
:107020000E94F00750928B0660928C0670928D063B
:1070300080928E0650907F06609080067090810648
:10704000809082060E9474080E941414AC2FBD2FF9
:10705000AF5FBF4F0E9454140E94070C0E9414148B
:10706000AC2FBD2FA75FBF4F0E9454140E94B013D6
:1070700016F00E9432140E9423140E94F0075092CE
:107080008F06609290067092910680929206CF5E73
:10709000DF4FF894CDBFDEBF7894DF91CF91089594
:1070A0003FF893011F426E1700271127222733272D
:1070B0005AC0088919892A893B8955C00027112798
:1070C000222733274B89341B4A89240B4989140B07
:1070D0004889040B48C00C851D852E853F8543C01B
:1070E00000271127222733274F85341B4E85240B79
:1070F0004D85140B4C85040B36C0088519852A85EF
:107100003B8531C000271127222733274B85341BAD
:107110004A85240B4985140B4885040B24C00C8137
:107120001D812E813F811FC0002711272227332771
:107130004F81341B4E81240B4D81140B4C81040B69
:1071400012C0088119812A813B810DC000271127B7
:10715000222733274B81341B4A81240B4981140B8E
:107160004881040B00C0F8940C8B1D8B2E8B3F8B39
:107170007894089508950895288C398C4A8C5B8CF6
:107180006CA07DA08EA09FA0590C481C371C261C0B
:10719000F8942CA63DA64EA65FA678940895F89480
:1071A000688079808A809B807894F8942C803D80D8
:1071B0004E805F807894F894A884B984CA84DB8474
:1071C0007894022D0058162D10585914480437048D
:1071D0000107E9F060F45D0C4C1C3B1C2A1C022DDD
:1071E0000058951484047304100768F010C05D18EB
:1071F0004C083B082A08022D00585914480437044B
:10720000010708F004C0262C372C482C592CF89480
:107210002C823D824E825F827894022D03290429BC
:10722000052908950024C3E8D6E008AA09AA0AAAF5
:107230000BAA0CAA0DAA0CA60DA60EA60FA608A2B4
:1072400009A20AA20BA20CA20DA20EA20FA20C8AE6
:107250000D8A0E8A0F8A088E098E0A8E0B8ECAEB53
:10726000D6E008AA09AA0AAA0BAA0CAA0DAA0CA67B
:107270000DA60EA60FA608A209A20AA20BA20CA296
:107280000DA20EA20FA20C8A0D8A0E8A0F8A088EFA
:10729000098E0A8E0B8E089540BE84800000000087
:1072A000E739154D4F5453494E2020202020010727
:1072B000414D4F5453494E33202020200307414D68
:1072C0004F5453494E35202020200507414D4F543F
:1072D00053494E3720202020F206404D4F544E4552
:1072E000575041524D20F506404D4F5441414354B3
:1072F00049564520F606404D4F54424143544956A5
:107300004520F706404D4F544153594E52454320B6
:10731000F806404D4F544253594E52454320F30610
:10732000404D4F54414F464654494D20F406404D80
:107330004F54424F464654494D20F906404D4F5454
:107340004144454354494D20FA06404D4F54424470
:10735000454354494D20FB06404D4F5441424C415A
:1073600054494D20FC06404D4F5442424C41544933
:107370004D20FD06404D4F54414445434D4F442060
:10738000FE06404D4F54424445434D4F4420FF06B6
:10739000404D4F544152414E474520200007404D3B
:1073A0004F544252414E47452020000000000CEF50
:1073B00007BB04EC08BB00E00093FD060093FE064B
:1073C00001E00093F5060093F606CBD20895A1E004
:1073D000B7E00D900F920D900F920D900F920D90BF
:1073E0000F920D900F920D900F920E949942DEF431
:1073F000A0920107B09202070E949942A6F4A092BF
:107400000307B09204070E9499426EF4A092050708
:10741000B09206070F900F900F900F900F900F9063
:1074200012D068940895A7E0B7E00F900E920F90E5
:107430000E920F900E920F900E920F900E920F9050
:107440000E92E8940895CF93DF93CDB7DEB7C25183
:10745000D040F894CDBFDEBF7894EAE4F1E00E941A
:10746000F502E4E6FDE00E946814AC2FBD2FA65F94
:10747000BF4F0E94A61400E00983698055240E9432
:1074800046080E941414EAE6F5E70E9468140E9478
:10749000070C0E941414E4EDFDE00E9468140E94A1
:1074A000070C6BD04424AC2FBD2FAE5FBF4F0E94A2
:1074B000A6140E9414140E941414AC2FBD2FA65FB2
:1074C000BF4F0E9454140E94130B44204AF00E94A4
:1074D0002314AC2FBD2FA65FBF4F0E94A61402C07D
:1074E0000E94231409810395098309F0C6CF00E0A7
:1074F0000983698055240E9446080E941414EAE614
:10750000F5E70E9468140E94070C0E941414E4ED31
:10751000FDE00E9468140E94070C2FD00E941414F2
:10752000E2E7F5E70E9468140E94070C0E94141419
:10753000AC2FBD2FA65FBF4F0E9454140E94A30D15
:107540000E94AC07A7E0B7E00981FF24A00FBF1D90
:107550006C920395098369F6CE5EDF4FF894CDBF38
:10756000DEBF7894DF91CF9108953F700000000056
:107570000000404F800000000000CF93DF93CDB7A4
:10758000DEB7C151D040F894CDBFDEBF7894AC2FA8
:10759000BD2FAF5FBF4F0E94A6140E9402180E9429
:1075A0001414E4E8FDE00E946814AC2FBD2FA75F1F
:1075B000BF4F0E94A6140E941414AC2FBD2FAF5FC2
:1075C000BF4F0E9454140E94070C0E9402180E9490
:1075D000141450900107609002070E9446080E9410
:1075E000070C0E941414ECE9FDE00E9468140E944C
:1075F000070C0E94150B0E941414AC2FBD2FA75F1F
:10760000BF4F0E9454140E941414ECE7FDE00E9446
:1076100068140E94150BAC2FBD2FA75FBF4F0E94AF
:10762000A6140E941414AC2FBD2FAF5FBF4F0E9451
:1076300054140E94070C0E9402180E9414145090C7
:107640000307609004070E9446080E94070C0E94EE
:107650001414ECE9FDE00E9468140E94070C0E94DB
:10766000150B0E941414AC2FBD2FA75FBF4F0E94B3
:1076700054140E941414ECE7FDE00E9468140E9468
:10768000150BAC2FBD2FA75FBF4F0E94A6140E9401
:107690001414AC2FBD2FAF5FBF4F0E9454140E9433
:1076A000070C0E9402180E94141450900507609065
:1076B00006070E9446080E94070C0E941414ECE979
:1076C000FDE00E9468140E94070C0E94150BCF5E1B
:1076D000DF4FF894CDBFDEBF7894DF91CF9108954E
:1076E0000F921F922F923F924F925F926F927F92D2
:1076F0008F929F92AF92BF92CF92DF92EF92FF92C2
:107700000F931F932F933F934F935F936F937F93A9
:107710008F939F93AF93BF93CF93DF93EF93FF9399
:107720000FB60F920E947906D6E0C3E828A839A8C0
:107730004AA85BA86CA87DA8E52C8CA49DA4AEA447
:10774000BFA47B0C6A1C591C481C381C281C28AA86
:1077500039AA4AAA5BAA6CAA7DAAD6E0CAEB28A8D5
:1077600039A84AA85BA86CA87DA8F52C8CA49DA478
:10777000AEA4BFA47B0C6A1C591C481C381C281CD6
:1077800028AA39AA4AAA5BAA6CAA7DAAFF2410E4F7
:107790001090B606A7E0B7E0A10DBF1D2C903324D2
:1077A00032180AF4322CA7E0B7E0110EA10DBF1D6C
:1077B0004C90552454180AF4542C1090B9061F10FC
:1077C00040941090ED06A7E0B7E0A10DBF1D6C90AE
:1077D000772476180AF4762CA7E0B7E0110EA10DF5
:1077E000BF1D8C90992498180AF4982C1090F006DC
:1077F0001F108094A7E0B7E0A10DBF1DAC90BB2483
:10780000BA180AF4BA2CA7E0B7E0110EA10DBF1DFB
:10781000CC90DD24DC180AF4DC2C04E808BB1091C1
:10782000FF062091000710FB03F920FB04F908BBB9
:10783000C59AE89403F904F908BBC59A1091FD06AE
:107840002091FE0611FB03F921FB04F908BBC59A40
:1078500010FB03F920FB04F908BBC59A47FA03F9AA
:1078600087FA04F908BBC59A27FA03F967FA04F9FD
:1078700008BBC59A55FA03F995FA04F908BBC59AED
:1078800054FA03F994FA04F908BBC59A53FA03F9B8
:1078900093FA04F908BBC59A52FA03F992FA04F96B
:1078A00008BBC59A51FA03F991FA04F908BBC59AC5
:1078B00050FA03F990FA04F908BBC59A35FA03F9AE
:1078C00075FA04F908BBC59A34FA03F974FA04F995
:1078D00008BBC59A33FA03F973FA04F908BBC59AD1
:1078E00032FA03F972FA04F908BBC59A31FA03F9BE
:1078F00071FA04F908BBC59A30FA03F970FA04F971
:1079000008BBC59AE89403F904F908BBC59AC59861
:10791000C69A0091F206002309F023D00F900FBE03
:10792000FF91EF91DF91CF91BF91AF919F918F9197
:107930007F916F915F914F913F912F911F910F9187
:10794000FF90EF90DF90CF90BF90AF909F908F907F
:107950007F906F905F904F903F902F901F900F906F
:10796000189504E808BB1091F5062091F60610FB67
:1079700003F920FB04F908BBC59A04E808BBC59AC3
:10798000C598C59A1091F7062091F80611FB03F9E6
:1079900021FB04F908BBC59A10FB03F920FB04F98D
:1079A00008BBC59A04E808BBC59AC598C59A10914A
:1079B000F9062091FA0613FB03F923FB04F908BB2F
:1079C000C59A12FB03F922FB04F908BBC59A11FB07
:1079D00003F921FB04F908BBC59A10FB03F920FB4E
:1079E00004F908BBC59A1091F3062091F40614FB24
:1079F00003F924FB04F908BBC59A13FB03F923FB25
:107A000004F908BBC59A12FB03F922FB04F908BB71
:107A1000C59A11FB03F921FB04F908BBC59A10FBB9
:107A200003F920FB04F908BBC59A1091FB062091CD
:107A3000FC0611FB03F921FB04F908BBC59A10FBF6
:107A400003F920FB04F908BBC59A0CE908BBC59AE9
:107A5000C598C69A0091F20602700093F206089546
:107A60006D6C206D6F7461706F7320313233342010
:107A70000000FE041454574954455354202020203C
:107A8000193F143F20202020202020202020193FB3
:107A90001448454C50202020202020201F3F144C0B
:107AA0004142454C5320202020204E3F1444412089
:107AB0002020202020202020C340144442202020C9
:107AC000202020202020DD4014445720202020208A
:107AD00020202020F14014444C2020202020202071
:107AE00020200B4114445120202020202020202041
:107AF0003141154446202020202020202020114004
:107B00001444424520202020202020202D401444D1
:107B100057452020202020202020464014444C455A
:107B200020202020202020206B401444514520207C
:107B30002020202020209840154446452020202049
:107B4000202020205F3F144442532020202020206A
:107B500020207B3F14445753202020202020202029
:107B6000943F14444C532020202020202020B93F53
:107B7000144451532020202020202020E63F15448B
:107B8000465320202020202020200342144D422054
:107B900020202020202020200E42144D572020207D
:107BA0002020202020201C42144D4C20202020206A
:107BB000202020204042154D46202020202020203B
:107BC00020202C42144D5120202020202020202035
:107BD0003C41144D424520202020202020204941B6
:107BE000144D574520202020202020205A41144D9C
:107BF0004C4520202020202020207341154D464553
:107C000020202020202020209C41144D4253202061
:107C1000202020202020A641144D57532020202032
:107C200020202020B841144D4C532020202020201B
:107C30002020D441154D46532020202020202020F4
:107C4000A14214504F5254532020202020200000E5
:107C5000145245534554202020202020473F144CE7
:107C60004F414450524F46202020403F145341562C
:107C70004550524F462020205508404D41494E4F17
:107C8000504D4F44452059004047494D534B20200B
:107C90002020202058004047494652202020202004
:107CA000202057004054494D534B202020202020B5
:107CB00056004054494652202020202020205500C4
:107CC000404D435543522020202020203B0040506F
:107CD0004F5254412020202020203A00404444525A
:107CE000412020202020202039004050494E4120B2
:107CF000202020202020380040504F525442202085
:107D000020202020370040444452422020202020C0
:107D1000202036004050494E4220202020202020A4
:107D2000350040504F525443202020202020340062
:107D30004044445243202020202020203300405043
:107D4000494E4320202020202020320040504F5216
:107D5000544420202020202031004044445244201C
:107D600020202020202030004050494E4420202058
:107D700020202020000000008E44393DB4330D48FF
:107D8000B64539193F2D392A06287C1D453650390C
:107D9000E7050000CF93DF93EF93FF93E8E7FDE75C
:107DA000E894C591D591C030CD0721F0CC0FDD1FEF
:107DB00074D5BEF7FF91EF91DF91CF91089580E0E8
:107DC00091E000914001112720914101E0E6FAE79E
:107DD000021759F00590DC01A00FB11F0C9203951A
:107DE0000F7300934001002099F700C0009107082D
:107DF00000231AF400E0009307080E940C03BEF46D
:107E00002AD43EF405E1C6DF26F4EA2FFB2F0995BC
:107E10002EF0EEE4F3E00E94F50200C004E60093C9
:107E20008C0101E000938D010FEF00930708089586
:107E30003E00E6E5F3E00E94F5026894089579D3E8
:107E4000F6F4E8E7FDE7E8940591159100300107A5
:107E5000B1F0BA94C9F7F801EE0FFF1F68940591CD
:107E600015910030010759F005911BE005910E9422
:107E700001031A95D9F70DE00E940103F0CF089590
:107E800058D326F40B2D0A950E94C903089551D3A7
:107E900026F40B2D0A950E94CE0308950FEF35D3DB
:107EA0006EF400E30E94010308E70E9401030B2F18
:107EB000F3D20A2FF1D20DE00E940103089500E2EF
:107EC00024D3C6F4CD010E9478050F9300E30E94ED
:107ED000010308E70E9401030F910F93DDD200E236
:107EE0000E94010302E60E9401030F91FDD20DE002
:107EF0000E940103089501E208D3AEF400E30E945A
:107F0000010308E70E940103CD010E947805102FAC
:107F100001960E947805202F012FBED2022FBCD2DD
:107F20000DE00E940103089502E2EFD20EF500E396
:107F30000E94010308E70E940103CD010E94780519
:107F4000102F01960E947805202F01960E94780537
:107F5000302F01960E947805402F012F9DD2022FCD
:107F60009BD2032F99D2042F97D20DE00E940103D8
:107F7000089503E2CAD24EF500E30E94010308E728
:107F80000E940103CD010E94780586D201960E94CD
:107F9000780582D201960E9478057ED201960E94D1
:107FA00078057AD201960E94780576D201960E94D1
:107FB000780572D201960E9478056ED201960E94D1
:107FC00078056AD20DE00E940103089503E29DD274
:107FD0003EF5CD010E947805402E01960E9478055D
:107FE000502E01960E947805602E01960E94780519
:107FF000702E01960E947805802E01960E947805C9
:10800000902E01960E947805A02E01960E94780578
:10801000B02E0E9470140E94AA090DE00E94010374
:10802000089500E272D2C6F4FD010E94C7040F93C6
:1080300000E30E94010308E70E9401030F910F93E0
:108040002BD200E20E94010302E60E9401030F917D
:108050004BD20DE00E940103089501E256D2AEF426
:1080600000E30E94010308E70E940103FD010E9452
:10807000C704102F31960E94C704202F012F0CD265
:10808000022F0AD20DE00E940103089502E23DD2C0
:108090000EF500E30E94010308E70E940103FD01C1
:1080A0000E94C704102F31960E94C704202F3196DA
:1080B0000E94C704302F31960E94C704402F012F21
:1080C000EBD1022FE9D1032FE7D1042FE5D10DE049
:1080D0000E940103089503E218D24EF500E30E94C6
:1080E000010308E70E940103FD010E94C704D4D1E7
:1080F00031960E94C704D0D131960E94C704CCD1DA
:1081000031960E94C704C8D131960E94C704C4D1D9
:1081100031960E94C704C0D131960E94C704BCD1D9
:1081200031960E94C704B8D10DE00E940103089562
:1081300003E2EBD13EF5FD010E94C704402E3196CB
:108140000E94C704502E31960E94C704602E3196BB
:108150000E94C704702E31960E94C704802E31966B
:108160000E94C704902E31960E94C704A02E31961B
:108170000E94C704B02E0E9470140E94AA090DE04C
:108180000E940103089500E4C0D1B6F40C910F934E
:1081900000E30E94010308E70E9401030F910F937F
:1081A0007BD100E20E94010302E60E9401030F91CD
:1081B0009BD10DE00E940103089501ECA6D186F445
:1081C00000E30E94010308E70E940103F8940D9167
:1081D0001C91789461D1012F5FD10DE00E940103C1
:1081E000089502E492D1B6F400E30E94010308E787
:1081F0000E940103F8940D911D912D913C9178946A
:108200004BD1012F49D1022F47D1032F45D10DE08A
:108210000E940103089503E478D116F500E30E945B
:10822000010308E70E940103F8940D911D912D911F
:108230003D914D915D916D917C9178942DD1012F5F
:108240002BD1022F29D1032F27D1042F25D1052F80
:1082500023D1062F21D1072F1FD10DE00E9401034A
:10826000089503E452D13EF40E9454140E94AA09D6
:108270000DE00E940103089500E247D14EF4AF9350
:10828000BF9357D1FF91EF911EF40B2D0E94BD04B7
:10829000089501E23AD16EF4AF93BF934AD1FF91B2
:1082A000EF913EF40A2D0E94BD0431960B2D0E94E1
:1082B000BD04089502E229D1AEF4AF93BF9339D142
:1082C000FF91EF917EF4082D0E94BD043196092D97
:1082D0000E94BD0431960A2D0E94BD0431960B2DDB
:1082E0000E94BD040895CF93DF93CDB7DEB7CB5086
:1082F000D040F894CDBFDEBF789403E206D19EF45F
:10830000B983AA8319D17EF4DE0113960E94A614C4
:10831000DE011396F981EA8118E00D910E94BD04F7
:1083200031961A95D1F7C55FDF4FF894CDBFDEBF08
:108330007894DF91CF91089500E2E7D036F4CD0133
:10834000F8D01EF40B2D0E942405089501E2DDD023
:1083500076F4CD01EED05EF4A02DB12D0A2D0E9451
:1083600024052EF401960B2D0E942405E6F70895AE
:1083700002E2CBD0C6F4CD01DCD0AEF4A02DB12DFD
:10838000082D0E9424057EF40196092D0E942405E3
:10839000E6F701960A2D0E942405E6F701960B2DBB
:1083A0000E942405E6F70895CF93DF93CDB7DEB79B
:1083B000CB50D040F894CDBFDEBF789403E2A5D077
:1083C000CEF4B983AA83B8D0AEF4DE0113960E942E
:1083D000A614DE01139699818A810D910E942405CD
:1083E0004EF4019617E00D910E942405EEF70196D8
:1083F0001A95C9F7C55FDF4FF894CDBFDEBF7894FB
:10840000DF91CF91089500E480D03EF40A2E1B2E18
:1084100090D01EF4A02DB12DBC92089501E475D02A
:1084200056F40A2E1B2E85D036F4A02DB12DF894CB
:10843000AD92BD927894089502E467D066F40A2E56
:108440001B2E77D0C6F7A02DB12DF8948D929D925A
:10845000AD92BD927894089503E457D086F40A2E25
:108460001B2E67D046F7A02DB12DF8944D925D924A
:108470006D927D928D929D92AD92BD927894089569
:1084800003E443D046F4AF93BF9356D0BF91AF916E
:1084900016F40E94A61408950F93EF93FF930F9282
:1084A000E8EDF4E80F9302950F70E00F0027F01F3E
:1084B000C895002D0E940103E8EDF4E80F910F70BC
:1084C000E00F0027F01FC895002D0E9401030F90B8
:1084D000FF91EF910F9108953031323334353637B3
:1084E00038394142434445460F930F921F93002E63
:1084F00018E0001C00E308F401E30E9401031A9550
:10850000C1F71F910F900F910895A5D08EF40F3FE2
:1085100051F408EF3FDC66F009EF3CDC4EF00AEF67
:1085200039DC36F00BEF36DC1EF000D1AB2DBA2D66
:10853000089591D02EF4FAC08ED016F40C94B4089D
:108540000895ECE3F6E80E94F50201E40E940103BD
:108550000AE30E94010300E20E9401030BB3C4DF9F
:1085600000E20E94010309B3BFDF00E20E940103A1
:108570000AB3BADF0DE00E94010302E40E94010386
:108580000AE30E94010300E20E94010308B3ACDF8A
:1085900000E20E94010306B3A7DF00E20E9401038C
:1085A00007B3A2DF0DE00E94010303E40E94010370
:1085B0000AE30E94010300E20E94010305B394DF75
:1085C00000E20E94010303B38FDF00E20E94010377
:1085D00004B38ADF0DE00E94010304E40E9401035A
:1085E0000AE30E94010300E20E94010302B37CDF60
:1085F00000E20E94010300B377DF00E20E94010362
:1086000001B372DF0DE00E94010305E40E94010343
:108610000AE30E94010300E20E94010303B164DF48
:1086200000E20E94010301B15FDF00E20E9401034A
:1086300002B15ADF0DE00E9401030895202020506E
:108640004F5254202020202050494E20202020200E
:10865000204444520D000F93CF93DF93E894A091F0
:108660008C01B0918D010C910023C9F0003211F4FE
:108670001196F9CF6894CA2FDB2F0881002329F4C3
:10868000C0938C01D0938D010AC0003211F0219665
:10869000F4CF00E00993C0938C01D0938D01DF915A
:1086A000CF910F9108953031323334353637383920
:1086B00041424344454601000A006400E803102794
:1086C00001001000000100100F931F932F933F93A0
:1086D000AF93BF93EF93FF932A95220FE894E6EBB5
:1086E000F6E8E20F0024F01D30E005901590339578
:1086F00000191109E0F73A95000D111D332309F413
:1087000046F46894E6EAF6E8E30F0024F01D34919D
:108710003D93225022F70EF03D93FF91EF91BF91D0
:10872000AF913F912F911F910F9108950F931F9338
:108730002F93AF93BF934424552466247724882431
:108740009924AA24BB24E89410E00C910D3211F472
:1087500011E011960C910033D1F411960D91023471
:1087600039F10835A9F1119768940D910053CAF1B8
:108770000830BCF523E0440C551C661C771C881C93
:10878000991CAA1CBB1C2A95B1F7B02AEDCF0D91FC
:1087900000533AF10A302CF568944DD0B00E002702
:1087A000A01E901E801E701E601E501E401EEFCF29
:1087B0000D910053B2F00230A4F46894BB0CAA1CD3
:1087C000991C881C771C661C551C441CB02AF0CFD1
:1087D0000D91003332F0073424F40A33DCF40053F3
:1087E0001CC0112389F0B094A0949094809470944C
:1087F0006094509440940FEFB01AA00A900A800A37
:10880000700A600A500A400ABF91AF912F911F91E0
:108810000F91089501342AF30753689424E0BB0CA8
:10882000AA1C991C881C771C661C551C441C2A9584
:10883000B1F7B02ACDCF0F924F925F926F927F9295
:108840008F929F92AF920B2CBB0CAA1C991C881C78
:10885000771C661C551C441CBB0CAA1C991C881C4C
:10886000771C661C551C441CB00C0F90A01C0F906C
:10887000901C0F90801C0F90701C0F90601C0F902C
:10888000501C0F90401CBB0CAA1C991C881C771C08
:10889000661C551C441C0F9008950F921F922F9236
:1088A0001F932F93EF93FF93202F302F27701A2EB3
:1088B0002B2E2E97E8942E96EC2FFD2F32961491A6
:1088C000112311F1187F1023B1F314911770243084
:1088D00018F0211780F302C0121769F7A12DB22DED
:1088E0003196C89510E2011629F01D91101519F75F
:1088F0001123B1F71D911123F1F66894EC2FFD2F90
:10890000A591B591049102C0A12DB22DFF91EF91D7
:108910002F911F912F901F900F900895CF44143ADC
:1089200047564420202020202020DB44143A47567C
:108930004620202020202020E344143A47564E2091
:10894000202020202020EB44143A4756502020209D
:1089500020202020F344143A475654202020202081
:108960002020FD44143A47442020202020202020AD
:108970000545143A47522020202020202020FD4485
:1089800014233A474420202020202020054514238A
:108990003A47522020202020202000000000E8EA52
:1089A000F9E80E94F50208954D41592031302032F6
:1089B000303035230000E0ECF9E80E94F50208951C
:1089C000585858230000E0EDF9E80E94F502089598
:1089D00030352E302300E0EEF9E80E94F5020895CC
:1089E0004D4334230000E0EFF9E80E94F5020895BA
:1089F00032333A30353A30302300EAEBF4E00E946B
:108A0000EC0203E20E9401030895E2EBF4E00E940D
:108A1000EC0203E20E940103089500E000930808BD
:108A200000E000930908CAE0D8E004E010E01883F1
:108A300019831A831B8324960A95C1F708950FB6EC
:108A40000F92AF93BF93CF93DF93CAE0D8E054E087
:108A5000459FC00DD10DA22FB32F1E930E9310E88A
:108A600000270E931E930E930E930E930E930E9368
:108A70000E930E930E930E930E930E930E930E93EE
:108A80000E930E930E930E930E930E930E930E93DE
:108A90000E930E930E930E930E930E930E930E93CE
:108AA0000E930E93F894AA83BB8301E0088300E041
:108AB0000983DF91CF91BF91AF910F900FBE1895B1
:108AC0000091080803950093080878940F911F916E
:108AD0002F933F934F935F936F937F938F939F93C6
:108AE000AF93BF93CF93DF93EF93FF930F921F92B8
:108AF0002F923F924F925F926F927F928F929F92AE
:108B0000AF92BF92CF92DF92EF92FF921F930F939B
:108B1000089500910808013001F4FF90EF90DF9074
:108B2000CF90BF90AF909F908F907F906F905F900D
:108B30004F903F902F901F900F90FF91EF91DF91FA
:108B4000CF91BF91AF919F918F917F916F915F91E5
:108B50004F913F912F911F91009108080A95F89429
:108B6000009308080F910FBF0F9118953608404CDD
:108B7000434449525141435420200000000008E082
:108B80000093220800932B0800E000932C08002794
:108B900000932D0801E000932E080FEF0093310899
:108BA00000932F080093300800270093350808959C
:108BB0007F00FF007F00FF007F00FF007F00FF00BD
:108BC0000000E0EBFBE800913508102F03950093BF
:108BD0003508110FE10F1127F11F15911093370878
:108BE0001591149100E001130895009135080A953C
:108BF0000093350808950090360800FE08950E94FD
:108C0000EA4800913708063321F4B9E4AEEA0E943D
:108C1000C24D00913208002349F00A9500933208B2
:108C200029F40E94F74D00270093C3040091220805
:108C30000830A9F00F3F39F402E00E94234900E018
:108C40000093220838C0039500932208A9E1B8E0F8
:108C5000A00F0027B01F0C910E9425492CC0009145
:108C60002B080830A1F00F3F39F400EC0E94234993
:108C700000E000932B081FC0039500932B08A2E28D
:108C8000B8E0A00F0027B01F0C910E942549009169
:108C90003208002381F400912C08003061F4009127
:108CA000C304002341F00E94F74D00270093C30442
:108CB0000FE10093320810912C08113091F4C3E8B1
:108CC000D6E00E945438CAEBD6E00E945438009196
:108CD0003708066330912F08689472D030932F08BC
:108CE00034C010912C08103081F500912D0800231C
:108CF00071F00091370806630F3F31F0009137089B
:108D0000096C0093370803C0002700932D08CAEBB5
:108D1000D6E0009137080E670E3F11F429D006C047
:108D20000F3711F439D002C00E945438C3E8D6E09E
:108D300000913708076B073F11F41AD006C00F3BAC
:108D400011F42AD002C00E94543800913708096FEC
:108D500030913108E89434D03093310800913708CD
:108D60000F6C30913008E8942BD030933008089580
:108D700000912E08053011F40C945938043011F488
:108D80000C946B38033011F40C947D38023011F4DC
:108D90000C948F380C94A13800912E08053011F4F2
:108DA0000C945E38043011F40C947038033011F4D4
:108DB0000C948238023011F40C9494380C94A63838
:108DC000031769F034E630933308330F30933408D7
:108DD000332730934B0831E030934A0841C0F6F511
:108DE000009134080A950093340869F5E09142082F
:108DF000F09143083A9605901590002D012919F13C
:108E0000E02DF12D3496E8940995EEF400904A088F
:108E100010904B082F923F921001000C111C3594BA
:108E20002794021813083F902F9000924A0810923E
:108E30004B080015110520F400934A0810934B08C5
:108E400001E400933408009133080A950093330835
:108E50002AF402E100933308032F02C0032F089580
:108E6000CAE9DEE810912C082CE0EC2FFD2F35919B
:108E7000311771F44591401759F4C591D5912C2FB4
:108E80002D2B49F0EC2FFD2F0F9309953F9108955D
:108E900024962A9551F73FEF089500FD654700FBA2
:108EA000774700EF814700DF894701F7C34E01BFD5
:108EB0000E4F01FE3F4E017F704E01FD654701FBE5
:108EC000774701EF814701DF894700912C08013086
:108ED00009F4089501E000932C08C3E8D6E00E944D
:108EE0005438CAEBD6E00E9454380C94F74D0F93D7
:108EF00000E000932C0801E000932D080F910C94E2
:108F0000F74D00912E08053059F0039500932E0877
:108F100007C000912E08013019F00A9500932E0821
:108F2000EAE3FFE800912E080A95000F000F000FFA
:108F3000000FE00F0027F01F28C053504545442084
:108F400020312D2D2D2D2D2D2D2D535045454420D7
:108F500020322D2D2D2D2D2D2D2D535045454420C6
:108F600020332D2D2D2D2D2D2D2D535045454420B5
:108F700020342D2D2D2D2D2D2D2D535045454420A4
:108F800020352D2D2D2D2D2D2D2D0F93EF93FF936E
:108F900008D013D00FE700933208FF91EF910F91A3
:108FA00008950F93AAE1B8E007E005900D920A95A5
:108FB000E2F7009322080F9108950F93AF93BF93A8
:108FC000A3E2B8E007E005900D920A95E2F700935E
:108FD0002B08BF91AF910F9108950F93EF93FF93DB
:108FE000EAE1F8E007E00D9001920A95E2F70093BC
:108FF0002208FF91EF910F9108950F93EF93FF9344
:10900000E3E2F8E007E00D9001920A95E2F70093A1
:109010002B08FF91EF910F9108954748144842584B
:10902000492020202020202049481448425856201A
:109030002020202020208948144842584420202005
:1090400020202020834814484258432020202020FC
:1090500020208F48144842585220202020202020D1
:109060005F49144842582020202020202020934986
:10907000144842585245414420202020A649144813
:10908000425854455354202020200000000069D04D
:1090900008950E949942B6F5082D0E944C42092D70
:1090A0000E944C420A2D0E944C420B2D0E944C42C1
:1090B0000B2DCCD014E600000000000000000000E2
:1090C0000000000000001A95B1F788D00B1589F058
:1090D0000F930B2D0E9474420DE00E9401030F912B
:1090E0000E9474420DE00E9401030DE00E94010302
:1090F00003C00EE20E9401030894B10AA10A910A7A
:10910000810AB0F608950E94994216F40B2D9BD067
:1091100008950E94994216F40B2D97D0089519D006
:109120005DD00F9300E30E94010308E70E94010352
:109130000F910F930E944C4200E20E94010302E64D
:109140000E9401030F910E9474420DE00E940103EE
:109150000895D09AD998D19ADA98D29AD49AD59873
:10916000089504E60E94940600E36DD004E60E9490
:10917000940600E368D004E60E94940600E363D0FE
:1091800004E60E94940601E30E94010308E35BD019
:1091900004E60E94940602E30E9401030CE053D00F
:1091A00004E60E94940603E30E94010301E04BD011
:1091B00004E60E94940604E30E94010306E043D003
:1091C00004E60E94940601E20E9401030DE00E9461
:1091D0000103089503D00093370808951F931FB625
:1091E000F894D49AD19AD5980000000000000000AD
:1091F0000000000000000000DC98D998000000008A
:1092000000000000000000000000000018E0D99AF3
:10921000000000000000000000000000000000004E
:10922000D9980000000000000000000000000000CD
:109230000000DC9A000FCD9901601A9541F717FCE8
:1092400078941F91089510E001C011E00F931F93CF
:109250002F931FB6F894DA98D898D998D29AD09AC2
:10926000D19A28E007FDD89A07FFD898000000009F
:10927000000000000000000000000000D99A00007B
:109280000000000000000000000000000000D9986D
:10929000000F2A9539F710FDD89A10FFD898DA9A5E
:1092A00000000000000000000000000000000000BE
:1092B000DA9817FC78942F911F910F9108954ED052
:1092C00008E40E94010302E0BEDF04E50E940103FE
:1092D00008E4BBDF01E6B9DF0CE6B7DF0CE6B5DF7B
:1092E0000FE6B3DF01E2B1DF0AEF0E94940603E468
:1092F0000E94010301E0A7DF00E30E94010308E7E9
:109300000E94010300913708C7D800E20E940103C0
:1093100002E60E94010300913708E6D80DE00E94A2
:109320000103689408950E94EE4800E30E9401033F
:1093300002E60E94010300913708D6D80DE00E9492
:1093400001030E9442037EF768940895F89406D0C2
:10935000009137084AD00E944203D6F708EC0E94D9
:10936000940600270BBB07E10ABB02E30E949406A8
:1093700000E310E03AD00AE00E94940600E310E017
:1093800034D00AE00E94940600E310E02ED00AE0F8
:109390000E94940601E30E94010308E310E025D037
:1093A0000AE00E94940602E30E9401030CE04BDFF6
:1093B0000AE00E94940603E30E94010301E043DFF8
:1093C0000AE00E94940604E30E94010306E03BDFEA
:1093D00001E20E9401030DE00E9401030895FEF3E3
:1093E00010E003C0FEF311E000C00F931F932F9312
:1093F0003F934F931FB6F89433273BBB30E144278C
:1094000028E007FDD89A0000000000000000D99A6B
:109410000000000000000000440FCD9941603BBBFC
:10942000000F2A9571F740933708113089F4D89AC4
:10943000000000000000000000000000000000002C
:10944000000000000000000000000000000000001C
:10945000DA9A000000000000000000000000000098
:1094600000000000000000000000000000000000FC
:109470000000DA9817FC78944F913F912F911F913B
:109480000F9108952F933F934F931FB6F89433276E
:109490003BBB30E1442728E0440FD99A000000008C
:1094A000000000000000000000000000CD994160B5
:1094B0003BBB2A9589F74093370817FC78944F9166
:1094C0003F912F9108950EE10093400805E9009324
:1094D00041080AE20093420805E900934308002787
:1094E00000934408009345080093460800934708FA
:1094F000009348080093490801E000934A080027B8
:1095000000934B08002700934C0800934D080093EC
:109510004E08002700934F080093500808954D45CA
:109520004E5520202020000000004F424A45435461
:1095300053208F4A000052412F44454320208F4A38
:10954000B84C53595354454D20208F4A00004F4288
:109550004A5F44495220954A214B4F424A5F444258
:109560002020A74A484B474F544F20202020AD4A87
:109570008F4C41444A5553542020AD4A8F4B414CA7
:1095800049474E203120AD4AE14B414C49474E20DE
:109590003220AD4A384C53455420524120209B4A3A
:1095A000C94C53455420444543209B4ACF4C50520C
:1095B0004F46494C4553A14A00005245534554205B
:1095C0002020A14A194B414E414C59534953A14ABD
:1095D00000005345542052412020CB4AD54C5345DE
:1095E000542044454320D14A164D2A2A2A2A2A2AA1
:1095F0002A2AD74A5F4D4143544956415445F54ABA
:109600008A4D44454641554C5420F54A994D4F4E9C
:10961000202020202020E34AA84D4F46462020202D
:109620002020E34AB24D3E2053544F50203CFFFFD0
:10963000000008950895089508950895F8940C94ED
:10964000000005C00EC017C0089508951BC000910A
:109650004608A8E3B8E00E94FA500E94ED476894DB
:10966000089500914808A8E3B8E00E94FA500E94CB
:10967000FD476894089500915F080A9511272227F5
:1096800068940895009148080E943451E894089520
:1096900005C00AC019C023C02EC00895AEE9B8E0C5
:1096A0000E94ED4768940895009146080E94345145
:1096B00000914808109149080E947C51AEE9B8E039
:1096C0000E94FD47689408950091800810918108D8
:1096D0000024089400091009222768940895009135
:1096E0004C08109146080113089500914D081091FF
:1096F0004E0868940895009180081091810816958D
:10970000079516950795169507951695079516953D
:109710000795169507950F5F1F4F68940895089554
:10972000089508950895089500C00FB7F894009023
:10973000B3061090B4062090B5063090B60640905F
:10974000EA065090EB066090EC067090ED06809073
:10975000560890905708A0905808B09059080FBF2D
:109760000092E3021092E4022092E5023092E602B7
:109770004092E7025092E8026092E9027092EA0297
:109780008092DF029092E002A092E102B092E202A7
:109790001090A6080090A7083090A8082090A9086B
:1097A0000092CB021092CC022092CD023092CE02D7
:1097B00001E000E0B6E2ABE6E5D161D20E94774776
:1097C000DBC10895089508950895089500C00FB766
:1097D000F8940090B3061090B4062090B50630902F
:1097E000B6064090EA065090EB066090EC0670904A
:1097F000ED068090560890905708A0905808B090B9
:1098000059080FBF009283021092840220928502B1
:1098100030928602409287025092880260928902BA
:1098200070928A0280927F0290928002A0928102BE
:10983000B09282020090A6081090A70810926B02C6
:1098400000926C020090A8081090A90810926D0276
:1098500000926E0201E00093FB0200E00093C80456
:1098600001E0B6E2ABE68ED10AD20E94774784C10E
:109870000895089508950895089500C00FB7F894C5
:109880000090B3061090B4062090B5063090B6064E
:109890004090EA065090EB066090EC067090ED0662
:1098A0008090560890905708A0905808B09059089A
:1098B0000FBF0092B3021092B4022092B502309210
:1098C000B6024092B7025092B8026092B90270920A
:1098D000BA028092AF029092B002A092B102B0920E
:1098E000B2020090A6081090A70810929B02009266
:1098F0009C020090A8081090A90810929D02009266
:109900009E0201E00093FC0200E00093C80402E024
:10991000B6E2ABE637D1B3D10E9477472DC10895A7
:10992000089508950895089500C000904408009295
:109930004C080090460800924D080090470800929D
:109940004E080090A6081090A7082090A808309014
:10995000A9081092D1040092D2043092D30420922C
:10996000D40401E00093C8048AD10E94774704C15F
:109970000895089508950895089500C0E894009109
:10998000C804003021F40E943F4E68940895E89482
:1099900008950895089508950895089508950895DF
:1099A00008950895089508950895089504C023C062
:1099B00027C038C0089560904808509049080E9418
:1099C00046080E941414E6E0F1E50E9468140E9423
:1099D000A30DA5EDB4E00E94A614109148080091D3
:1099E0004908B8E0A8E30E943729B8E0A8E30E943C
:1099F000FD476894089500E418E32FEF68940895F4
:109A0000A5EDB4E00E9454140E941414E6E0F1E5C0
:109A10000E9468140E94070C0E94AC07062D152DA9
:109A20006894089508E210E068940895089504C0C9
:109A300029C02DC040C00895609048085090490842
:109A400008E1601A05E1500A0E9446080E941414B9
:109A5000EEE0F1E50E9468140E94A30DADEDB4E0C4
:109A60000E94A61410914808009149081851054118
:109A7000B8E0A8E30E946829B8E0A8E30E94FD4787
:109A80006894089500E31AE2222768940895ADEDE2
:109A9000B4E00E9454140E941414EEE0F1E50E9418
:109AA00068140E94070C0E94AC07062D152D085E55
:109AB0001A4E689408950CE310E06894089505C068
:109AC00010C024C0089508950895E6E3F3E00E94CD
:109AD000D1471091460801E3010F009321086894D3
:109AE0000895EEE2F3E00E94DD471091480801E39B
:109AF000010F009323080091480810918F0101176E
:109B000019F40AE200932A086894089503E01127E3
:109B1000689408950895089508950895089500C0DB
:109B20000E9477470091460800938F01F8940C94A7
:109B30006B4F0895089508950895089500C0009109
:109B40004608F0E0E0E00E94BD040E943F4E14C0D1
:109B50000895089508950895089500C001E00093C0
:109B600047040AC00895089508950895089500C00F
:109B700000E00093470400C0EEE1F3E00E94C54717
:109B80006894089500904F0810905008012831F013
:109B9000EEE3F3E00E94C547E8940895B0934F08C0
:109BA000A093500800935108EEE1F3E00E94C547EE
:109BB00068940895F0914F08E09150080027F0173D
:109BC000E007A1F00091510809950FEF0E9494065B
:109BD0000FEF0E9494060FEF0E9494060FEF0E9471
:109BE0009406002700934F080093500808950F93A0
:109BF0001F93AF93BF93EF93FF9300270093320817
:109C000000912C08003071F1E0914008F09141087A
:109C10003A9605911591002311F4112331F0E02FAC
:109C2000F12F3096E89409952EF0E0914008F091DC
:109C30004108B7D9E0914208F09143083A9605915E
:109C40001591002311F4112339F0E02FF12F3196F3
:109C5000E89409950EF40CC0E0914208F091430895
:109C6000ACD906C0A1EBB4E0B8D9AAEBB4E0C5D931
:109C7000BF91AF91FF91EF911F910F910895E091E6
:109C80004008F0914108389605911591012B09F48F
:109C90000895E0914008F0914108E0934208F09364
:109CA0004308389605911591000F111F0093400845
:109CB0001093410800914608109147080093480806
:109CC00010934908009144081091450800934608F4
:109CD000109347080027009344080093450887CF56
:109CE000E0914208F09143083A9605911591002EB3
:109CF000012A31F0E02FF12F3596E89409957EF096
:109D00000091420810914308CEE1D5E9EC2FFD2FD8
:109D10003896259135912F3F19F43F3F09F4089566
:109D2000220F331F021711F4131711F02C96EECFE8
:109D30000093400810934108C0934208D093430811
:109D40000091460810914708009344081093450875
:109D5000009148081091490800934608109347085D
:109D6000FE013A9605911591002E012A39F0F8016D
:109D70003396E894099516F00027112700934808B8
:109D80001093490834CFE0914208F09143083A9685
:109D900005911591202F212B49F0E02FF12F3296BC
:109DA000E89409951EF00027112722278091480882
:109DB00090914908082E092A21F4222382F4C8012F
:109DC00009C000904A0810904B088019910910F4BE
:109DD00088279927809348089093490808CFE091F5
:109DE0004208F0914308349705911591000F111F17
:109DF00020914008309141080217130759F7E0916C
:109E00004208F09143083C97E0934208F0934308DE
:109E100000270093480800934908E9CEE0914208E2
:109E2000F09143083A9605911591202F212B49F086
:109E3000E02FF12F3296E89409951EF000271127A4
:109E4000222780914808909149088017910728F0AF
:109E500022239AF4882799270BC000904A08109073
:109E60004B08800D911D0817190710F4802F912FB2
:109E70008093480890934908BACEE0914208F09147
:109E80004308749605911591000F111F2091400809
:109E9000309141080217130759F7E0914208F091F9
:109EA00043083C96E0934208F09343080027009350
:109EB0004808009349089BCEB0E1AFEFBEBFADBFED
:109EC00000E00C931197B130E0F7F0E0E0E00E9481
:109ED000C70400938F01B0E1AFEFBEBFADBF0FEF7E
:109EE00000939501009396010E9477030E949003CE
:109EF000ECE9F0E00E94F502EEE8F0E00E94F502E5
:109F0000E0E1F1E00E94F50201E0009336080E94D2
:109F1000A9480090360800FE53C0E0E8F2E00E9435
:109F2000F5020E94BF450E94B1480E94EA480AE03B
:109F30000E94940602E087D90AE00E9494060DE48C
:109F400084D90AE00E94940603E47FD90AE00E94C3
:109F500094060DE27AD90AE00E94940604E375D9CA
:109F60000AE00E94940600EC6ED9EEE8F0E0339629
:109F70000AE00E949406059168D90AE00E949406BE
:109F8000059163D90AE00E94940605915ED90AE022
:109F90000E949406059159D90AE00E949406059101
:109FA00054D90AE00E94940605914FD90AE00E9414
:109FB000940605914AD90AE00E949406059145D974
:109FC000ECEAF2E00E94F5020E941D05E2E7F1E0F2
:109FD0000E94F50200918F010E94CE030E94233A55
:109FE000ECE8F1E00E94F5020CEF07BB04EC08BBC3
:109FF00001E00E9494060E94D7390E94123900277E
:10A000000093560800935708009358080093590886
:10A010000093C4040093C5040093C6040093C704CE
:10A0200001E000935A08E4EAF1E00E94F50202E040
:10A0300005BD00E004BD00EC06BFE0EEF1E00E94CB
:10A04000F50208E000BF09E003BF0FEF01BF00B752
:10A0500001FDFDCFE8E2F2E00E94F50202E407BF55
:10A0600002E406BF7894E6E4F2E00E94F5020E9462
:10A07000BF50E4E0F3E00E94F5020E941F34E0E6E6
:10A08000F2E00E94F5020E94A120E0E7F2E00E94C7
:10A09000F5020E944E28ECE9F2E00E94F5020E94CF
:10A0A0009D2AE6EFF2E00E94F5020E940E3FE2EEEA
:10A0B000F2E00E94F5020E94634AEAEFF1E00E949A
:10A0C000F5020E94DA4D0E94F63E009155080130DB
:10A0D00039F40E9434210E948B280E94A22AF1CFD9
:10A0E000023009F4EECF033019F40E94EA34E9CFCC
:10A0F000043001F4E6CF0F930FB70F931F93109125
:10A100005A0800915908010F00935908112700912E
:10A110005808011F0093580800915708011F009329
:10A12000570800915608011F009356080E94604589
:10A1300000E00093F106D6E0C7E90E94CF3819F09D
:10A1400001E00093F106D6E0C3EA0E94CF38D6E0E2
:10A15000C3E80E94BC38D6E0CEEC0E94CF3819F09C
:10A1600001E00093F106D6E0CAED0E94CF38D6E0B8
:10A17000CAEB0E94BC380E94FB450C94894519C06B
:10A180000EE618E024E0AEE9B8E00E94644311D086
:10A1900001E06AD00DE618E0AFD000E00E94345133
:10A1A0000BE310E00E947C51AEE9B8E00E94FD474D
:10A1B00008951F932F93CF93DF93EF93FF93E9EDD0
:10A1C000F1E0C0E6D8E0112722270E94C704003042
:10A1D00021F0E883F887219623953F961395183050
:10A1E000A1F720935F08FF91EF91DF91CF912F911D
:10A1F0001F9108950F931F93CF93DF93EF93FF93D6
:10A20000C0E6D8E0C00F0027D01FE881F88531965E
:10A2100018E00E94C70431960D931A95D1F718974C
:10A22000FF91EF91DF91CF911F910F9108950F93BF
:10A230001F93CF93DF93EF93FF93C0E6D8E0C00F57
:10A240000027D01FE881F885399614E00E94C704E2
:10A2500031960D931A95D1F71497FF91EF91DF91F5
:10A26000CF911F910F9108951F938F939F93CF9339
:10A27000DF93EF93FF9300937008A1E7B8E0BADF94
:10A28000A9E7B8E0D4DFC0E6D8E0C00F0027D01FB0
:10A29000E881F8853D9611240E94C704002E31966E
:10A2A0000E94C704000C001F111C00927D0800933F
:10A2B0007E0810927F0880E090E087D000938008AD
:10A2C00084D00093810881D000939B087ED00093B6
:10A2D0009C081CE0A2E8B8E078D00D9376D00D93EE
:10A2E0001A95D1F700E00C93FF91EF91DF91CF9198
:10A2F0009F918F911F9108952F938F939F93AF9369
:10A30000BF93CF93DF93EF93FF9300939C08109339
:10A310009D08C9E7D8E0AEE9B8E080E290E000240B
:10A320000A9419901D921812092E93959430C9F72A
:10A330008D939A95E9F7902D939519F0943009F043
:10A340009395AEE9B8E0A90F9927B91F24E00894C6
:10A35000091F191F0E94644300919C0810919D08D9
:10A360008CE190E020919B08029F800D911D129F2F
:10A37000900DC2E8D8E009911991003051F4FF9195
:10A38000EF91DF91CF91BF91AF919F918F912F91DD
:10A390000895013039F4AEE9B8E017D00D931850A4
:10A3A000E1F7E9CF023039F410D00093A7080DD0BF
:10A3B0000093A608E0CF033039F407D00093A90832
:10A3C00004D00093A808D7CFD6CFEF93FF930024F3
:10A3D000E0917D08F0917E0810907F08E80FF91F4A
:10A3E000101C1BBE06910196FF91EF910895180174
:10A3F0000C000140021003100000000000000000EB
:10A4000000000000000000000000416E6420416C6C
:10A410007020017928E9416E6420426574200C4265
:10A420003217416E642044656C2006EA2B66416E4B
:10A43000642047616D3115C83B8741716C20416CC8
:10A440007020D1510C7941716C2044656C20CCDFB7
:10A45000046141716C2047616D20D0860EED417121
:10A460006C204C616D20C97DF92341716C205468CA
:10A470006520D4EDFED941716C205A657420C9570E
:10A48000137F41717220416C7020E90CFF8E417185
:10A49000722042657420E308F82B417172204465F4
:10A4A0006C20F1A3E9C141726120416C7020B8E5D4
:10A4B000B9DE4172612042657420B7BFB1EA4172D2
:10A4C000612047616D20B7C3B0B9417261205A6500
:10A4D0007420B30EB14441726920416C7020165B48
:10A4E00020FF417269204265742014271D43417585
:10A4F0007220416C702037AB40AF417572204265CD
:10A5000074203F333F3541757220457073203515F7
:10A510003DA0417572204574612035E139FC4175DB
:10A520007220496F742034352EA44175722054680E
:10A5300065203F3B3455426F6F20416C7020966917
:10A540001AFA426F6F20426574209E8C38CD426F9C
:10A550006F2044656C20A0EE2ED9426F6F204570AD
:10A5600073209B902613426F6F204574612092B92F
:10A5700019DF426F6F2047616D20994C35DF4361D1
:10A58000702042657420D6A2EB3843617020446588
:10A590006C20E5C1E95343617220416C7020437E19
:10A5A000B5E64361722042657420613E9DF74361C8
:10A5B00072204368692053CFB57F43617220457094
:10A5C00073205855AC5143617220496F742061ED7E
:10A5D000ACA6436172204F6D65206BE29D834361A1
:10A5E0007220546865207105A5734361722055700F
:10A5F00073206734A47F43617320416C7020071F70
:10A600004F814361732042657420019D532E436145
:10A61000732044656C200F1654B543617320457058
:10A620007320141C5989436173204574612008A26A
:10A63000514E4361732047616D2009F855624365AF
:10A640006E20416C70319A9EAA7443656E20416CF5
:10A6500070329A9EAA7443656E20426574209454A9
:10A66000AB1B43656E2044656C208008B8AD436524
:10A670006E2045707320901FB4D143656E204574E1
:10A68000612099E6C4B843656E2047616D2085DC82
:10A69000BB2743656E20496F74208CBBCC6143653A
:10A6A0006E204B6170209E0EC4CB43656E204C61C2
:10A6B0006D207A4EA76243656E204D75202091D59E
:10A6C000C44643656E204E75202091D0C561436518
:10A6D0006E205468652094D5CCDC43656E205A65A5
:10A6E000742092DFBD8143657020416C7020E0C012
:10A6F00058034365702042657420E286633A4365DF
:10A70000702045746120DAE656F643657020476193
:10A710006D20F97F6D2C436570205A657420E9F037
:10A7200051D843657420416C7020200B05C04365EF
:10A7300074204265742007AAE6B643657420457408
:10A7400061200C0FF1AF4365742047616D201CB58B
:10A75000048D436574204F6D6920187FFBD14365DC
:10A76000742054617520124BE99743697220416C43
:10A7700070209B21A4A2434D6120416C702047387A
:10A78000E87F434D6120426574204346E6C1434D56
:10A79000612044656C204B4EDAE3434D61204570E7
:10A7A00073204996D743434D6120457461204E1074
:10A7B000D6CC434D61204F6D69324A5CDE7D434DFE
:10A7C0006120536967204A21D8B8434D61205A65FA
:10A7D000742042DAD5BA434D6920416C702050BDD7
:10A7E0000759434D6920426574204E9A0BA8436F68
:10A7F0006C20416C70203BB4D016436F6C204265D6
:10A8000074203DB1CDB443724220416C7020A44D00
:10A81000259143727520416C7031833DA745437289
:10A820007520416C7032833DA745437275204265A7
:10A83000742086F3AC114372752044656C20813A14
:10A84000AD634372752047616D20840AAFB04372D7
:10A85000762042657420849BDF1A4372762044651B
:10A860006C2083D0E8C743727620457073208058EF
:10A87000E0324372762047616D208157E756435698
:10A880006E20416C7032886935E343796720416CF2
:10A890007020DA383FAD4379672042657431CDCA04
:10A8A00027524379672044656C20D04C3F77437929
:10A8B000672045707320DB102FC5437967204761FF
:10A8C0006D20D6D8389C437967205A657420DFC242
:10A8D0002A82446F7220416C7020302AB2994472EF
:10A8E000612042657420B8A6498D44726120446598
:10A8F0006C20CA995F264472612045746120ACF8CF
:10A9000056814472612047616D20BD3F48684472A2
:10A910006120496F7420A29652EC447261205A65FE
:10A920007420B4D75C6945726920416C7020112D88
:10A93000AF844572692042657420361DF8DA45728D
:10A94000692047616D2029D7ED024572692054685E
:10A9500065311F56C75347656D20416C70204FE924
:10A960002CD847656D204265742051CB2769476517
:10A970006D20457073204701235747656D2045744E
:10A98000612041E51FA647656D2047616D2045E9BF
:10A99000171047656D204D75202043511FA947654D
:10A9A0006D2058692020473E122247727520416C65
:10A9B0007020E97BBDF74772752042657420EF88EF
:10A9C000BE124772752045707320F091B7D7477259
:10A9D000752047616D20E6F7CB7648657220416CA3
:10A9E0007031B5DF143D4865722042657420AE10A9
:10A9F0001E384865722044656C20B5F022EE48652B
:10AA000072204D752020BB7726FB48657220506967
:10AA10002020B5F133C3486572205A657420B00216
:10AA20002C7148796120416C702063C5F3D448795A
:10AA30006120457073205C9909074879612047615E
:10AA40006D208C6FDF6B487961204E75202072314C
:10AA5000E93B487961205069202094C7DA7B487926
:10AA600061205A6574205E1D085C48796920416C3C
:10AA7000702014E1A96C487969204265742004872C
:10AA8000935D4879692047616D2027F2979B496E55
:10AA90006420416C7020D98BBD804C656F20416C67
:10AAA00070206AF110D44C656F20426574207CA43C
:10AAB000147E4C656F2044656C20767F1CDD4C65F0
:10AAC0006F204570732066FB216F4C656F204761D6
:10AAD0006D316CFB1BE74C656F20546865207685F3
:10AAE00015B34C656F205A6574206C6720EE4C6579
:10AAF0007020416C70203A7DE6F14C657020426513
:10AB0000742039B3E2D04C6570204570732035B2A3
:10AB1000E08B4C6570204D7520203702E9374C6979
:10AB20006220416C70329C9AE9724C6962204265E5
:10AB30007420A131F2CF4C696220536967209EEBEB
:10AB4000DC734C757020416C70209B07BD5D4C75AB
:10AB50007020426574209DF2C3594C757020446585
:10AB60006C20A1F6C6D84C75702045707320A231B8
:10AB7000C1294C75702045746120A8C5CA024C7566
:10AB8000702047616D20A461C61D4C7570205A6508
:10AB90007420A05DB6BD4C796E20416C7020629F20
:10ABA000305D4C797220416C7020C456368A4C79E5
:10ABB000722042657420C6A62EEB4C797220476144
:10ABC0006D20C8342DF84D757320416C70208519A7
:10ABD0009EC84D7573204265742086B3A03A4F70AD
:10ABE0006820416C7020B97011AA4F7068204265CE
:10ABF0007420BAF0066C4F70682044656C20AB4638
:10AC0000FACF4F70682045707320ABF8F9684F7029
:10AC1000682045746120B51FE9E44F7068204B61DE
:10AC20007020B2E30D2F4F7068204E752020BDAC10
:10AC3000F2424F70682054686520B72ADCD94F7003
:10AC400068205A657420AF48F1254F726920416C25
:10AC500070203E6F0A6B4F72692042657420374A3C
:10AC6000F4784F72692044656C203A5CFF954F720E
:10AC70006920457073203B1AFE504F72692045745D
:10AC800061203909FCA24F72692047616D20392784
:10AC900008EE4F726920496F74203AF7F7B14F728E
:10ACA00069204B6170203D21F2684F726920506924
:10ACB000203332F309CA4F7269205A6574203BE68B
:10ACC000FD4650617620416C7020D772B0385061DB
:10ACD000762042657420DAD7A2E850656720416C7F
:10ACE0007020F36A15625065672042657420F33E58
:10ACF000277E5065672045707320E5400DE3506561
:10AD0000672045746120EF972A805065672047616E
:10AD10006D200254155A506567204D752020F0D2E1
:10AD20002299506567205A657420EF520F3B506599
:10AD30007220416C702023EB461E506572204265E4
:10AD40007420211439985065722044656C20273096
:10AD50004334506572204570732029CF38445065C4
:10AD6000722047616D20207C4B3E506572205268F6
:10AD70006F20208D369F506572205A6574202928D7
:10AD80002CD650686520416C7020049FC4835068A5
:10AD90006520426574200B9EBE4E50686520476159
:10ADA0006D200F88C31650696320416C702047C125
:10ADB000A8E650734120416C7020F22AD659507594
:10ADC00070204E75202045EBC342507570205069AD
:10ADD00020204CD7CBD65075702052686F2055B3C9
:10ADE000DDD350757020536967204EF7C31C507532
:10ADF000702054617520480FB8D450757020586980
:10AE00002020527EDD0B507570205A65742055014C
:10AE1000C7C052657420416C70202CB9A8265363BA
:10AE20006F20416C7020ADEBDAD553636F20426523
:10AE30007431A9B5E42753636F2044656C20A8CF13
:10AE4000E03153636F2045707320B191CFC75363D6
:10AE50006F2045746120B56FC33353636F20496F12
:10AE60007431BBA9C79353636F204B617020BAC480
:10AE7000C91E53636F204C616D20B934CBD453632A
:10AE80006F204D752031B1DECA8053636F20506949
:10AE90002020A88CDB4853636F2053696720AC796E
:10AEA000DC0453636F2054617520AF0FD853536394
:10AEB0006F2054686520B9DBC38A53636F205570D7
:10AEC0007320B8B4CB8E53657220416C7020A5FC02
:10AED00009095365722045746120C197FBED5367E2
:10AEE000652047616D20D2B81B69536772204465A5
:10AEF0006C20C189D60F5367722045707320C21829
:10AF0000CFA65367722045746120C0F1CC4F5367C0
:10AF1000722047616D32BEDDD538536772204C61B7
:10AF20006D20C2C3DC415367722050686920C5DFC1
:10AF3000DA0C5367722050692020CA1BE2705367F5
:10AF4000722053696720C78FDB06536772205461F4
:10AF50007520C99CD918536772205A657420C8DAC5
:10AF6000D5FC54617520416C7020308017375461D6
:10AF7000752042657420395B283B54617520457407
:10AF8000612027FD21E6546175204C616D202A4F18
:10AF9000119154617520546865322F3A16525461EC
:10AFA00075205A6574203B5A1DBB54724120416C78
:10AFB0007020B14E9EEF5472412042657420A7E587
:10AFC000A6CE5472412047616D20A1879F6C5472B8
:10AFD0006920416C702013E1299854726920426500
:10AFE000742016C5313354756320416C7020EB49D1
:10AFF000AB43554D6120416C702074AC56D6554D15
:10B0000061204265742074574F4A554D6120446554
:10B010006C2081465034554D612045707320880F57
:10B020004EB2554D61204574612091774559554D7B
:10B03000612047616D207D7A4B82554D6120496FBB
:10B0400074205EC8438F554D61204C616D206C7932
:10B050003C59554D61204D7520206D653A5C554D2C
:10B0600061204E75202077442E8A554D61204F6D0A
:10B07000692059B25563554D61205073692075B7E9
:10B080003E94554D61205468652064B348AC554DDD
:10B0900061205A6574208D514D3D554D6920416C9C
:10B0A00070201AB07D87554D6920426574209C92AE
:10B0B0006848554D692047616D20A1D965045665E2
:10B0C0006C2044656C205C3CB31256656C20476173
:10B0D0006D32560DBD7056656C204B61702062CF8D
:10B0E000B2A556656C204C616D206054C2ED56656A
:10B0F0006C204D75202071B1BA8256697220416C66
:10B1000070208D8AF04F5669722044656C208856F5
:10B1100004C75669722045707320897E0F6956698D
:10B1200072205A6574208F35FF2A6E0004000210C9
:10B1300003100000000000000000000000000000FC
:10B140000000000000003ACC1EF6E35FFEDA9087B4
:10B1500027EAACE6DAB0A17902EEBA58D2B2BCC5A1
:10B16000CF0ABE83DDB6B6ACE5F6B2C9FA3CC6D3AB
:10B17000F730B10CFD42B0143348B9E7FB6EE2C2C0
:10B18000111CC126EC9EC180E93EC157E7E8B3C15E
:10B19000DB10BE4CDF9CBEA6E05CC43ED5F4BD48CF
:10B1A000E542C0D0E602C366E4EEC5CAF2C8D2DE0C
:10B1B0001FF2C226DD08D7233630E496DF6607810A
:10B1C0003A080781397810812B1A1C7A3C2A40D81A
:10B1D00022383B1430003DF22DC639C73264E325D6
:10B1E000441C828051AE478BE2D83AF5F8563AFEBD
:10B1F000F8985B6C1C1A27E721EA512DEB2A504383
:10B20000EB9C56CDF7D883CD0B404A64F4488E5D55
:10B210004260F6D5569A8B60198CC787D522CF6CC1
:10B22000D474CB4F2A72C7442E748530109E85F299
:10B230001062863E103E82690648B382D5A68BE333
:10B240003B1C88871E7E77561266779112425D3CC2
:10B25000109E8581DA62C3E4D282C570D294D1D9BE
:10B260001A6ADC57EE60DD4AEE3C10FF1632D4025B
:10B27000E12E120048841C99FFFA3CF10012390AB1
:10B28000DD7AABBDDFAE68B2612068BB61FE8F9D29
:10B29000D60082F9121E83071992832B123683FA85
:10B2A00011708430144684D611A68508128484C98E
:10B2B0001464B64D3CA851ABDE70878239D271342C
:10B2C000107471B2109E769E4D5E80FD14F481DE86
:10B2D00014468296163E943C4C6E9F584E66106201
:10B2E000555C8598EFAA71DF11B281E74284AE7692
:10B2F000EDA676094E487E244B12071A3A9EA01EF0
:10B300000400021003100000000000000000000014
:10B3100000000000000000000000014926FA014979
:10B3200026EE01490BA6014D0BC4015F31B6017633
:10B330002DB4017AD5EE018C21840191217E018307
:10B34000D060018734A40187067E018C2F04018C14
:10B35000163E019A1E60019A270001EFEEFC01A73C
:10B3600026FA01A72E2C01AC2EDA01E22E6201B9D9
:10B37000272401BE247201BEDCE401BEAFC601D4A5
:10B38000245401D928C801D0AFD201E62EE601E647
:10B390001EDE01D9AFD801EB1A6A01EB052801F4D2
:10B3A000EEFC01F8EF20020108FA01FDAFE40218FB
:10B3B000F820022A2BAA0249660002401EFC024520
:10B3C0001F1402492B74024E2BFE027BDF66027BA8
:10B3D000086A028DF5E6027643D4028443D40296CD
:10B3E000F5B0029143DA02911A160296AB2802A830
:10B3F000F5F8029FC8E602B5117C02B51854028D1B
:10B40000F5EC02BAE1D602D0FF9402E7F73C030262
:10B41000ED10031D101A0314F65E035CDFCC03600D
:10B42000DFBA03332A4803382A4803382A3C033C4E
:10B430002A4E033C2A4803412A3C034EEA6A03533E
:10B440002A42036E090603722A180384E056039603
:10B45000012603B11FBC03BA1F6E03BA1F7403C3D6
:10B460001F8C03C31F8C03C81FC803C31FA403C8BA
:10B470001FB603BABB9C03BFBB9603BFBB8A03DAEC
:10B480001F8603D51F8603C8BB9C03DE1F8603E708
:10B490001F9803E70EC403EC1FB603F029D0040283
:10B4A000C058043816320438172E0434D234044AF3
:10B4B000EC6204735646043D9AA20473121E0458AB
:10B4C000F8BC0480F45A048E2916049B1EAE04D1E5
:10B4D000646204B2FC4C04B22C9A04BFFC7C04C429
:10B4E000FD7E04B6D0A204C8F52C04C801DA04CD50
:10B4F000FD7E04C4AFDE04D6FDDE04B69B6804DF27
:10B50000FDB404E3FDC004E8FD72051003FC051E54
:10B5100003F60522040805220402054254B4052757
:10B5200004080534D138054F02F4057C591C055830
:10B53000D13E0597ED34058A568805780E5205737D
:10B5400007440573072605812B4A0585074A0581AF
:10B55000E0320585E0440585E0260593F8C205D272
:10B56000590405D644340607D34E05ED2B320607A1
:10B57000D8E805FAF25C05C4992205FAF25C05FFE9
:10B58000EE36061AF0DC0615F442061EF4300623E9
:10B59000F44E0615B18E065921AE063EFC0406593E
:10B5A00021B40654F1C6066B03DE066BF1CC064BE4
:10B5B000ECDA0634DF240674E038067D21BA06741E
:10B5C000029A0693E3F8068FE038068A02B8067DF1
:10B5D000D68A0693E3F8064B99160698E04406E0EF
:10B5E000EC1406A5E6DA06AE0C2406B7297006B7F9
:10B5F00003D806BC297C06C5296406DB43F806C5CA
:10B60000046E06F6EB5A07BC780006F655E006D73E
:10B6100009E406DBF35806E9013206E904B006E95D
:10B62000044406F6F31006E9014406ED013E06ED7A
:10B6300003F006F6046206F6040E06FB013206FB72
:10B6400004F206FB04D406FF049E071A3A9E072361
:10B6500039480708EBE4071A03D806E0E5CC0723CE
:10B66000EC80073504D4070DB104073E1728074CBA
:10B6700023DC072CB0F20747E266074CF1E40759D8
:10B68000331E07700144071F98C8078239780723C3
:10B6900098C80782013207823A0807A156E2078656
:10B6A0002DCC077DFDD80786210C078F2106077456
:10B6B000DEC4073598D40782DEDC07A12B0207A180
:10B6C00014280786DEE207A6042007A6FFD607A1F6
:10B6D000B96E07D7FAAE07EE08A007A198BC07AA73
:10B6E00098B608122A18080DEA10081BFD900843A6
:10B6F000EF4A0848E2CC07FB98CE07FB993A08517D
:10B700000B2208671B84087026DC085EDC72085A6E
:10B71000D3D20867EFE0081298A408750BB2087935
:10B7200026DC0875FC16088B26F4082D992E089443
:10B730002CEE0899ED94087ECA3C085E98AA08C1D0
:10B740002D60087098F208D3F8B00887989808EA36
:10B75000F3D608EEFD5A0909326408EEF65208F7EE
:10B76000F61608FCF6100929E01A090EF3EE09296D
:10B7700042DE0932FCE8093B223809484F9E09485D
:10B780002B0E095FED76096CED820971ED7C096C79
:10B79000ED94096C2DAE0948DA9E0944D4200905C0
:10B7A0009922096CF3B209489994098CF5D40929B6
:10B7B00098DA09B42C5209BD2C8809ABF5AA09AB5B
:10B7C000F5AA097E9A8409A7CB0209E6F10009EAE5
:10B7D000F10609A2E89009DD21EA09D8110409A7B8
:10B7E0009A7209F3FD8409EAFD7E09F8F20E0A0156
:10B7F000FD840A202A9009E6B5C60A292AAE0A0164
:10B80000D30C0A292AAE0A292AAE0A203D920A3709
:10B810002AC60A05C25C0A56E2B40A17F8EC0A0EF8
:10B82000C28009F8B57E0A4DC70C0A2EF8C80A4432
:10B8300025C80A2EF8C80A05B5960A32F8E009E1CB
:10B840009A120A4DFC2E0A5609FC0A56E8D20A56EC
:10B85000CE980A6DE65C0A56E59C0A83F5560AA75F
:10B860002B1A0A2597420AA7F6520AB0F3160AB015
:10B87000F6760AB0DF540AD4DF480ACBF64C0A64E5
:10B880009A7E0ACBF66A0AB5B51E0AE2F66A0AE69D
:10B89000F66A0AEBFD4E0AEBFA060B01FD480B2196
:10B8A0001F680B1CF7180B21F6280B25F7180B76D1
:10B8B000573C0B52FEF20B0FA3BA0AEF9B620B1C14
:10B8C0009C5E0B9EE8B40B5BFECE0B44CE9E0BAC95
:10B8D00057840B69EEEA0B52C3280B71E70A0BB5CC
:10B8E0002D960B219AA20BBA2D9C0BC72D6C0BCB5E
:10B8F0002E140BCB2D7E0B3C999A0BA8E3CE0BA3F9
:10B90000D58E0BD52DBA0BD52DAE0C02569A0BD970
:10B910002D900BD92D960BD92D6C0BD92D720BDEDA
:10B920002D840BDE2D8A0BEB2D720C0B37D40BF80C
:10B930002DA20BDE01500C062E920C0F37C80C0600
:10B940002E980B7B9AC00BF406600C0B2E8C0C18F7
:10B950002DB40C212DDE0C212E080C252E140C2AC2
:10B960002E260C2A2E0E0C33323A0C02BE600BD956
:10B970009DBA0C692E920C772E8C0C38CDA80C7BBE
:10B980002E9E0BF09B140C5CE3DA0C38FC040C8943
:10B990002E8C0C57CE1A0BF89A420C7FE6740C6969
:10B9A000D5820C0299820CAC2D240CAC2D360C1DCA
:10B9B0009B140C8DD6EA0C92CA720CD536900CD121
:10B9C000FF9A0CBFD2EE0CD101620CD5FF880CDAC5
:10B9D000FFA60D0B2F700C9FA9780D3D54900CB154
:10B9E000AE160D0202E80D4A52B60D1408580CE7C7
:10B9F000CAA80CF9D35A0CD1AE0A0D02D34E0D1DB4
:10BA0000FE920D342EF20D582BB60D2B02B80D2BD5
:10BA100005E20D4A2E800D3DFDBA0D612E860D46C4
:10BA2000FEC80D652E800D6A2BA40D6A2E860D149E
:10BA3000B2180D5C074A0D1498F20DE852080D2B50
:10BA40009B620DB618AE0D269A540D97D06C0DBBA7
:10BA500005F40DDF16F20DE3312C0D4698E00D9242
:10BA6000AD260DEC04A40E072E1A0DF514EE0E03F0
:10BA700004CE0E0C14CA0E272E020E0C17460E15FD
:10BA800004CE0E1014E20E1916860E4B38EE0E1967
:10BA9000E08C0E4B05700E39F2200E3DF3100E1E99
:10BAA000C66A0E6A2F280DFEADB60E4F09DE0E6F68
:10BAB00007980E61E9020E6107620E610CF00E6FCD
:10BAC000078C0E4FD01E0E73079E0E7301560E97F5
:10BAD0002EAA0E932F100EA52F2E0E7CFEC20EA5A1
:10BAE0002F1C0EA02F100E8A07980EA92F0A0E8E5B
:10BAF0000CBA0EAE2EE60EAE2EB60E930D500EB252
:10BB00002EBC0EB72EC20EB72ECE0EA90D440EB708
:10BB10002F040EAE0FDE0EC42FB20EBB2F8E0EC939
:10BB2000122A0EDF2F160EC90D6E0EE42F0A0ED24A
:10BB30000D200EDBFDB40EDF05580EDF02700EE89F
:10BB40000E100EFF2FDC0EE80D680EE80DA40EC0DF
:10BB5000CEB60EC4CEA40F082F5E0F1130D80EE45F
:10BB6000FDC60F2C30DE0EFF0D080F08027C0EDF25
:10BB7000CA660F08FE020F3030D20F2C2FEE0F03D3
:10BB8000FDD20EFFE67A0F50E3D40F11FE0E0F35F3
:10BB900030C60F15FE2C0EF6CA720F1EFE200EF6D2
:10BBA000CA7E0F1EFE1A0F1EFE440F08CA300F3E3B
:10BBB00002D60F66344A0F6F2F100F6F2F100F54DD
:10BBC000E00E0F54E0020F54E0140F35FDB40F598E
:10BBD000FD3C0FBC59040F5DFD4E0F8130420F8AB2
:10BBE000440A0F50E5CC0F6FFD5A0F81FE2C0FA5B4
:10BBF0002D7E0F47F1960F74CDC60FAA0FAE0FA57D
:10BC0000FEAA0FCE2DBA0F93C8BC0FFB3A080FA5A2
:10BC1000CDF60FF61E240FA1B7700FF2FD360FE917
:10BC2000E020101F2F4C0FF2FD301062555C1028E1
:10BC30002F1C0FC5E63E100DF658101FFEB6101A49
:10BC4000F64C104331BC104C2B201047EF141074ED
:10BC50003F301070322E10622B1A103AEEA210599B
:10BC6000E8C010702B2C1055F61C1035D0EA10824D
:10BC70002B1A1050EEDE105EF5B61067EED80FC02E
:10BC8000989210982A72109D2B5010B83A0810AF55
:10BC90001E241094F59210C52F5E11165AC61094EA
:10BCA000E3AA1094E3B01086CCAC1094D6A210D7BF
:10BCB0002F6410B8F5B010E02F7C1082F23E10EE29
:10BCC0002EF810AACCB8110D3B88110031F810E005
:10BCD00000F010B3CCB210D3F1F010B8C5BC10BC5A
:10BCE000C8F811122F3A1100163211A2667E10CE3A
:10BCF000C8AA1104083A111B084610F2CB8C114354
:10BD000031C21148E3F8116CF56E12175A00118216
:10BD10000A2C1163D5EE1175F2CE115AC436116793
:10BD2000D5F410B895C21163C41E119D0810111FDF
:10BD3000A4B6118BF30A115AE6EC1194F30411FC2A
:10BD4000488411FC488A11B40B3A12003222124D79
:10BD5000570611EEEDA0120024C6123B4E9611F7C5
:10BD600011B21251555C121B132C1251285C125F38
:10BD700034FE12A25622123F05F4126C0EAC12A22F
:10BD8000305A127ADFC012B0334212D831FE12E1BB
:10BD9000273612CB126C12F82694130E1038133279
:10BDA0001F68132912541329084C132E1254133BE5
:10BDB0001EF013493252134D1EE41332F15413296D
:10BDC000EAEE1344106E135F26E212F3B5C6132990
:10BDD000DE881371331E137A31981352D96012F32F
:10BDE000E87E13761E9C131CBB96136D08A6138366
:10BDF0001EF0138C1FC2133BCEE613911F6E13442B
:10BE0000CF041371EF0E13B932B81388F25C13919B
:10BE1000FA4E13D432D613D032C413D432D013A76F
:10BE200008DC138CF40C13D432DC13D932EE13DD9E
:10BE300032AC13C7189C13E633C0143CF33A13F822
:10BE400032E813E6EDF413D911A0140A32EE13E62A
:10BE500005E813FD1BDE13DDECB0142E3762142E43
:10BE60001D161406DE941401DE7013CBE8C61452BE
:10BE7000F0CA13FDCD90143C05E8140ACDA2144578
:10BE800007E61433F352147B33C014762E80142E3D
:10BE9000E806147F301214842E7A14842E7A148DBE
:10BEA0002E7A14912EBC148D2E6E147607EC147B12
:10BEB00007EC14DE54A214D04E061413B04A14BA80
:10BEC0003F30146DF2B01476F9B81452D5E214A8CC
:10BED0002EB614AC2EB014B534FE14B13282141C3C
:10BEE000B02C1476F3401421E87E1476F3761464B3
:10BEF000FBA414B5331814B52EE614B52EF214961F
:10BF0000F85C14A3F35E149AE97414E222FE14DEC2
:10BF10000BB814E7F28614DE00BA15022B7414F481
:10BF20001AA615B165D614F91ABE14EBEFCE14FD9E
:10BF300013B614D5DB041514213C15212C34152619
:10BF40002BFE150BF79C152F27AE151D11C414B52C
:10BF5000AEC4154A2CD01553288C15692CBE155C1F
:10BF600015FC1545F358154AF66A15892D18155C08
:10BF7000F86E15650BEE15801614159B2D001589AE
:10BF800019D4150FB182148497A215B1359A15B141
:10BF90002D181580FFDC1580FFD015BF35CA14F0B1
:10BFA000A09015C3168C15C82B5615DE288015BA1F
:10BFB000F20815F028C215CCDF3615DEF3BE1607E1
:10BFC000129C15ECF1CC164A3EAC15609FC4159B33
:10BFD000EB6C159BEB541680292216921830169F95
:10BFE000368A1697291C1692142816920F78164135
:10BFF000C6221661DC36164ACCB8169708E216BF80
:10C000002B3816A40B3416E33720169FF50E16AD09
:10C01000F51416C4089416DF31F816BBF1C01707E3
:10C0200034F816BFF1C016F1E0F816ECE07416C84B
:10C03000F1BA16CCF1AE16E30B04171534BC16D1C9
:10C04000F51A170C2D2416E30882174234B6173D53
:10C050003EAC173D3EAC16E8F17E16E3E09E1710AD
:10C06000FDE41710055216A9B038172BF2EC172271
:10C07000CD96178E2736177CFEF8174FD312174B25
:10C08000E06E178AFEF817C02B4A17DF328217615D
:10C09000C4D817A9FEEC17D2087017ED283817A9D5
:10C0A000FEEC17E4017A17E8FEF8186F505E181ED0
:10C0B0001476181E147617CDE6F81803F01017ED55
:10C0C000DF66181A01BC183E146A18421476183933
:10C0D000DF24180CF3641854FA1E1861F6BE188E8B
:10C0E000163E186FF6821908505217A9FEEC193A3D
:10C0F00059B2188AE968182CABD01874C54A18F6DA
:10C100002EC819113B8E18BBDF7E189CC5CE18E4D3
:10C11000F84418E4F83E1974570C18CED09C193125
:10C120003AFE18F2E2C0193A254A193E255C190870
:10C13000E8901947267C195026761911F3BE198606
:10C140003B341923E2DE1928E224198F3B22198F90
:10C150003AD419A13B0A19A13AC219A13AC819AF98
:10C160003B46199D264C199D265219AF2D5419A6F0
:10C170001A0419B3264619FB40A419C5E9BC198253
:10C18000DD2619F23B0A19CE1CD419E52F3A19AF56
:10C19000FF8819C5111619F7264C19E5EF021A0088
:10C1A0001C981A122C0A1A001C921A3A409819F27A
:10C1B000FFAC1A0D1B9019F2FE621A483B701A1B55
:10C1C0001C8619BCC1841A432C821A1BFE621A3ABF
:10C1D000F0C41A3AF0C419CAEB9C1A1FF1301A7E47
:10C1E0003B6A1A1BE5301A28F1361A8234381A3A9B
:10C1F000F0821A28E0981A9930DE1A9429A01A2D94
:10C20000C5C21A79FE6E1ACA3ECA1B0050E81A7ED1
:10C21000FBDA1AC631EC1AA6F2F21A94F64C1ADCC2
:10C22000277E1A75FA0C1A90CD5A1ACFE5C61AAFA6
:10C23000E40A1AC1E7CA1B1730841B172E5C1B1BAC
:10C240002E681B1B2E621B1B293A1B202DBA1B2498
:10C250002E621AEE0D861B121D821AE5F0E81B36BF
:10C260002E381AA2C1661B5639841AE1F09A1B5166
:10C2700039961B3F2C521B3220F41B2DF3A61B00BA
:10C28000C91C1B902EDA1B51F2DA1B09E8CC1B7E6D
:10C2900010621B56F5F21BA21DAC1B8C02E21B8C1C
:10C2A00002E21BDD3A681BE63A921BA20A441BA27B
:10C2B0000A741BEA3A981BEF3A4A1BFC3A981BEFA8
:10C2C00030AE1C0139781BB402BE1C0A3A561BABB7
:10C2D000F07C1BBD03001BC202E81BD4033C1BB057
:10C2E000F07C1BB4F0821C012A661BBDEFCE1BBD87
:10C2F000F2981BCBFE261BD403001BBDF0821BC68D
:10C30000F28C1BD802B21BE6031E1BEA03181BDDCE
:10C31000F6A01C3236F01BFC0F421B7AB2D81C016F
:10C3200009301C9A568E1C0A0F3C1C0A0F2A1C1C32
:10C3300019561B87B2D81C05018C1C25F3A01BCFF6
:10C34000E9C21C0AF4901C371B241BC6FD661C2581
:10C35000021C1C7A3C2A1C833A5C1C2EF8501C32AE
:10C36000F4241C4001E01C520C481C32F01C1C56EA
:10C370000C421C37F48A1C3BF3FA1C13CFCA1C91E5
:10C3800030E41C52F6401C52F4661CB03A5C1C832C
:10C3900019981C71009C1CA328261CA72DAE1CBE3E
:10C3A00034861C9519561CB02D901CB02DA21CC7AC
:10C3B0002DB41C83F82C1C83F2D41C7FEAC41CCB44
:10C3C0002DA21CCB2DBA1C9AFFFA1C9EF4541CB54E
:10C3D00006FC1CA7F3AC1CBE006C1CC701F21CC7FA
:10C3E000E9141CC7E93E1CC7EB421D33385E1CDD57
:10C3F000F2BC1CC7D7381D0AF95E1D0AEA161D21BA
:10C40000F4721D25EA701D2EF5561D4005161D847B
:10C410003A021D40FF4C1D5B16C21D40EAD01D496B
:10C42000FFA61D13E7521D21E7581D9130661D72AE
:10C43000FF9A1D7606841CCBABBE1D3CD56A1CFD45
:10C44000E7341D0FE7161D1CE7221D96066C1D60C4
:10C45000E0BC1D88EC621DA3FFA01E4EE9EC1DFD93
:10C460003A9E1DC30B641DA3F4CC1DBA12A21DC3BA
:10C47000F4F61DD512781DE212961DEB12B41DBE06
:10C48000E8181DF912A21DFD12BA1E1D128A1DE226
:10C49000EEEA1D96E6AA1DBEEBAE1E06FD901E60DE
:10C4A0003B581E603B5E1E2ADBDC1E33E89C1E4EA2
:10C4B000FE2C1E6512A21E5708821EAD3A7A1EA8D7
:10C4C0003A861EB13A741E65FE381E5CF3A61E84C1
:10C4D00012481E06B2C01E0BB2901E9604261F07FD
:10C4E0003C8A1E65EB961EB1F1E41ECC00A81ECC62
:10C4F00000A81EC8FFC41ECCFFBE1EB1E5CC1F3471
:10C5000041521ED1F32E1F22F52C1F2FFF941F2204
:10C51000EAD61F22EAE81F38F50E1F4F04BC1F4F52
:10C52000F1721F53F1781F97237C1F53EABE1F2B14
:10C53000EBC61FC43CB41FDA3F3C1FDA3F2A1F730F
:10C54000EE901FB2E7E21FFA3BE81F6AD2D61FBF88
:10C5500010AA1FF131801FC810922046413A2015C1
:10C56000261020583D081FECEB2420613A2C209C1B
:10C570003C36206F3B88206F3A3220733B94207307
:10C580003A142019E56C1F22EAE81F1DEADC20425C
:10C59000F26820783A2C228F71A0202BF328209C5F
:10C5A0003C3C2019DFD8204BEA34203DEA0A2042E7
:10C5B000E9FE2046E9F8204BE9F820A93E6A204F21
:10C5C000FE7A203DEF142042EF0220BB3DF820BB55
:10C5D0003AE02046EA0A204FEF26205DDB58208112
:10C5E000F6E2208EEBCC2073EEA82010F26820B784
:10C5F000F394211535FA20BBF29820B2EA0A20D62E
:10C60000DBDC20DBFEE6212739722142365A20DBB3
:10C61000F29820E4F28620EDF28020BBC922211E90
:10C6200005CA2123030621B34B002111FA06213547
:10C63000FBD4211AFA2A21A13A2C2130FA3C219864
:10C6400031C8219C31B02115DFC62115DFB4211A74
:10C65000DFA82154EA16215DE30E21D7374A215481
:10C66000F4F621E436C021AE0F362186F3D0218FB7
:10C67000F0E22193FC7621E92AFC21A1F37621A1A5
:10C68000F37C21A5F36A20C9A216223A427220DF68
:10C69000A1E021C9F14221E4F8AA216BB4FA2259A0
:10C6A0003A26221F0210217DAE40221FFC0A222CB6
:10C6B00003CC2204DBD02216E11C22863A62221629
:10C6C000E16A22A13A2622B83A3821CEB25A22672C
:10C6D000E9B0226BEAC422CA3A4422DC3AE022746E
:10C6E000FCA022EE3A5022F23A5622AFC63422FB88
:10C6F0003A5023043A2623093A56230D3A68231B5D
:10C700003A6E231F3A6223243A6E231F3A7423247D
:10C710003A6E232D3A5022CEFFC4232D3A8C23317A
:10C720003A2C23363A3822BCF18422C5F5B022C512
:10C73000F53E22E9FC2222AAD22E22F7FD36230D55
:10C74000EC5622AFC62822D7D92A23703A3823754F
:10C750003A2C232DEC5022F7EDA02304E5242331BD
:10C76000FD0C232DF72A231BE4B2233FE5A223244B
:10C77000DB582348F5922355F98E2367FCBE2355D9
:10C78000DC1E238BF99A2399FC222387EA58235530
:10C79000CBC8232DB6A423CF01AA22DCA27C239DE3
:10C7A000FA1E23B4E1EE23A2CBB023A6CBD423A65A
:10C7B000CBCE23D8E1B82400FBC22405FBC8240952
:10C7C000FBEC2409FC0A2409F7EA23EEE1B223D8A2
:10C7D000CCB823FCDBE82424FA302432E73A24CB1B
:10C7E0003A2C244DE1FA2444E20024CB2C2E24EFF1
:10C7F0003AD424FC3A7A2451CDC02495F43624BD91
:10C80000EEE42495D29A249ED48C2490CBC2253277
:10C8100034802649660C249ED45024CFE6F824EFB9
:10C82000F83224DDE0B02595485425290624251C3E
:10C83000D0B42501CEF8252EE4E82549E2BA2556E4
:10C84000EA9A2583F8F8250AB94A257AECC8259191
:10C85000F8DA2595E49A257FDBA625A7F7362595F6
:10C86000E37A25C2F22C25CBF22C258CCD30259AEB
:10C87000D42025BEDCF025CBEA0425A3CCFA25D4B0
:10C88000E35C25CBDCF02625E9AA25D0CE8625D988
:10C89000CE7425D4CE68262AF8E62618E29C25F424
:10C8A000CE8025FDCE26260FCECE2613CE5C262AA0
:10C8B000CE802640E63826881644263CDD8C26218C
:10C8C000CD602625CE0E2660E9AA262ECDBA264EAC
:10C8D000E5482669E632261CCD00266DE61426843E
:10C8E000E64A2669DF9C2657CDD8269AF970267B22
:10C8F000DAF82669CE262696E5BA2691E008269132
:10C90000E5F6268DE086267BCDF626B5EA3426911F
:10C91000D3F626B5E5DE2691CE0E26E2FE3226E2DD
:10C92000FE322676C20226C7DB2226BAEA1626F097
:10C93000E18226D9E04426D9E00E2706F9642714BF
:10C94000F95826C7CB3E2726F7C6271DED0A26F045
:10C95000E1822721F70C273CF958270FD5F4272A25
:10C96000E0E62714CE322718CE8C2760F95E2745E3
:10C97000E65C277B040227B122442706BD9A277272
:10C98000F26227BF2172274ECD96274ECD90279F6A
:10C99000DFA22784E12E278DE65027ADFA3C278DB4
:10C9A000E65027ADFA5A28534A102789F22C27BAA5
:10C9B000FA4827B1F35E2777C13627BAFA3027A89D
:10C9C000F30A27BFFA48279FE5CC27CCFA6C27B695
:10C9D000E2EA279FE5CC281D1FBC2777C13C27E74B
:10C9E000E65627E7DC1E27BFCC6A282BE8F0287C18
:10C9F00009D227C3ABE828ADEA5229102DA8277722
:10CA00009B3228C4F38E28D1F7122A47607228D1AE
:10CA1000F35228FAEA582915F3EE27F9A018292B22
:10CA2000F15A2927F49628CDC1602922F3EE29274F
:10CA3000F3F42934F1A82939F1902934E34A294241
:10CA4000E32C28E8BD3A292BCBF82B1663D8298A8A
:10CA5000E1522973C46C29DB1A1C29C4E4F4290CA3
:10CA6000A3242AC9482A29DBCE2629C0BF0829C900
:10CA7000BB3C29E8C1782AF649FE2A8F20882A473C
:10CA8000EF1A2A50337E29DFB66E2B6B55AA2B8BFB
:10CA900057A82993A3242AA1F2E62AAAF2EC2A4253
:10CAA000B6142AFBFCEE2B3523B82AE4F0402ACE3C
:10CAB000C2F22A1AA0E42AE0C30A2BF245A22BCE26
:10CAC0002B4A2AE9B3EC2B9DF3822BD30C2A2B6241
:10CAD000E2362B9DE7D029C093F42BA6E2662B43C8
:10CAE000B5F02B47B3EC2C00F3A02C00F3A02B1ACD
:10CAF000A36C2BAABCAA2CE5480C2B74A78C2E4D3A
:10CB000069E42C4CD1CE2C51D1C82BEEB1162BBCE4
:10CB1000A7B62CAFEE182C1FB0922C99D37E2CC642
:10CB2000ED702D8725C22CDCD7F22D2D012C2D3652
:10CB300006C02C70AED03543793E2DDC46AA2CC100
:10CB4000B1282D36E6DA2DE133F02CF3B1D02DA249
:10CB5000036C2DA201FE2DC2FF102D09B18E2E05F2
:10CB60001B782E361B782D4DB9742C879CFA2D9589
:10CB7000C0AC2D48A7B62FF465162E3BE9B62E01A2
:10CB8000E9DA2E36E9E02E36E9E02E4DE9DA2DB469
:10CB9000B2C02DE6BC262E7AFEF22F9A5B322E13FF
:10CBA000C2A42E17C2A42E29C6E8305767022E0E43
:10CBB000AFE42ED0F1C62ECBFAEA2ED0F1C62E5F0E
:10CBC000B7762F7F31982F25F8B62E88B2C02FD098
:10CBD0003DAA2F2AE73A2F21E7582F06C4BA2F96ED
:10CBE000FF8E2F9600F02F9A00EA2F9A01322FAC79
:10CBF0000AB62F5BDA682F64DA142FCB00CC2F9A99
:10CC0000F7D82F2EBCC22F0AB29C2FACF0222F37A0
:10CC1000BCCE2FBEF98E2FC3F8DA2FC7F8D42F174A
:10CC2000B2962FC3F8D42FCBF87430573FA22FD52C
:10CC3000F8EC2FD0F9BE2FCB00D22FEBF9DC302F40
:10CC4000F9642FFDF9FA3002FA24300BFA06302A83
:10CC5000F3EE30841C0E2FF0C2862FC3B338308918
:10CC6000FB92308DF934309FFFCA3092F904309F27
:10CC7000FB863052ECFE314A46F230B6FB5C30BAED
:10CC8000F8F830C8F92E30C8F9642F579AFC30BF35
:10CC9000E56C30F0E2F030D9F29E31380A56313886
:10CCA0000A50313DFF3A3158F3E8317CFBFE3180C8
:10CCB000FD723160E818319BE3443089A38431BAB6
:10CCC00000DE31DAF89230DEA2E831ECF85C31FABD
:10CCD000F3FA32461AD03203F41230E39F3A321E8E
:10CCE000E9B630C89CBE30E39F70323DFC9A323DBD
:10CCF000FD0C324F1D70323DF8C8324FFD1831EC3B
:10CD0000C5B6325DF94631F5C5AA327CFD1E32B793
:10CD10000F6032BB1284332C3D7432A9F86232B7F3
:10CD2000F6C432BBF71E324BC11E31BFA37832F5B9
:10CD3000FC283308FEEC3239ACAE31A49DC6336614
:10CD4000219C3366219C31DF9F34331EF928334701
:10CD5000FC4C32FAD30632BBBCC23347F7D2336243
:10CD6000FBA43362FBC2336BFBA4336FFBDA337873
:10CD7000EA643335D04832B2ABE8339CF71833BCA1
:10CD8000024C33C9049233EDE314328A9E7A33E4C1
:10CD9000F976328E9E6832A0A00032BB9FA032DFAF
:10CDA0009EBC3435F9523431F92833FFD5FA32DBE1
:10CDB0009DC63378ABFA32ED9DEA33B7B4F4336BEA
:10CDC000A76E348B0B9435314A5E3486FF52344360
:10CDD000EA7C33119D9033359E50348BFF4C335990
:10CDE000A1E03359A1E63474E3503498FFA6335DD3
:10CDF000A1B034AAFFA0349DF4F03498F058335D0C
:10CE00009E6834A1F08E355A459C349DF05834AF5D
:10CE1000F51A335D9E7A34A1F05834C1FB4A34AA26
:10CE2000E9BC3393A1E0337D9F7033AAA23A338FDC
:10CE30009F4633AAA19E3386A04833BC9EB03509D5
:10CE4000E66E3509E6683512FB5C3504FA003509F3
:10CE5000FB5C33AE9EB034BCDB6A33BC9EB0355E47
:10CE6000217E33D7A18633C09EB033C9A018356C5C
:10CE7000214233B79DD2351BF46C3528FB4A33C0B1
:10CE80009CEE33DBA01E33C99E9E3531F9583582A6
:10CE9000216C34E0C98E341FA270341AA27C355E36
:10CEA0000234342CA2A03411A0D23474A8C433FFAD
:10CEB0009D3C34169E683428A0063455A28834352B
:10CEC0009FCA348BA6FC34289E2C3470A2B23459ED
:10CED000A16E342C9CF43474A29433FF978A3629C3
:10CEE000341A35ABF32235DCE49A3620E67434503C
:10CEF0009E6E348BA33035AFEF50347D9F28349431
:10CF0000A0BA3494A39035F3FB4A34599AE436B965
:10CF10004938348F9D5435A6CA9634A19E323620A6
:10CF2000E67434A69DD83536AA083617F4B436C64A
:10CF300043083617F4CC35DCD31234D39E1436872D
:10CF400021E435AFBA4C34E59EDA351FA30C351217
:10CF5000A066369E17403617CB3E35169E2C3548B8
:10CF6000A2AC3644D6D2364DD6D835319D1E356763
:10CF7000A16235249CB23567A16236DD177C357914
:10CF8000A2A036CB07503567A16236CBEABE359DED
:10CF9000A2E8355A9D1235F3AC0635759F1635AFAC
:10CFA000A2E23683CC0435759E6E3590A04E35874F
:10CFB0009E8035CFA4B636DDE9F2357E9C8E35AB4A
:10CFC0009EAA35A69E6835AB9F8235909C9435C647
:10CFD0009FBE35C69F8235DC9B02321989E035FC45
:10CFE000A1683737F10C3600A15635D89CE83612C7
:10CFF000A12035F39EFE36059BE6365AA2C4363B89
:10D000009F4C3737C7AE3651A0AE36E6AF483656DE
:10D010009F2E36639F2E36639EC838493756367129
:10D020009F1C36BDA44A36909F4C36839C7C36E1CB
:10D03000A30036BD9F4636EFA0E436E19F46371C7D
:10D04000A3F0371CA2CA3749A6123729A13E3705DB
:10D050009EC83725A12037059E803725A150370E61
:10D060009E6E38910966370E9E6E370E9E6E36F3B1
:10D070009CE83837D2CA37209E6E370E9E7A3768C2
:10D08000A306394A41763788A2F4375F9F04389166
:10D09000DE823783A2C438B1EFD438B1EFDA372E4D
:10D0A0009AA8387BCDC037BEA4AA38BA2EF8377FED
:10D0B0009E5637B5A15639331C5C37CBA12C37AC03
:10D0C0009E2037DDA08A3813A75C37DD9FC437EB7D
:10D0D000A25237C29E8C390BDD7A37EFA16E391818
:10D0E000E98C39A831AA394EFC70394AF49037EBF3
:10D0F0009EAA381CA21C39C8326437F89E3237D435
:10D100009BD4382EA21037D09E7438139EF838184E
:10D110009E0E3840A1E6385BA21038219DD83833E6
:10D120009E4A386DA3E439A4F8863891A37838571D
:10D130009E4439C8F43638649E4A3888A078394A03
:10D14000BE483A41302A38ACA2FA38A3A2FA389144
:10D15000A0783896A06C389FA06638A8A07E387F4B
:10D160009DAE387F9DA838B5A18038CCA2A63914D1
:10D17000A61838BA9D5438969A0C3933A2B239267B
:10D18000A29A3972A6543938A2D639269FB2390BE1
:10D190009DA2394AA2583ACD1EF639339F403A80B3
:10D1A000EC383953A11A383392AA3A85EC2639382B
:10D1B0009DCC39459DA83B1530003C2361923965D3
:10D1C0009F463A97CCCA3A9BE12239659F4639720D
:10D1D0009F3A39659EE03984A12C39659DD2396525
:10D1E0009F46396E9DC6396E9DD23AE8F95839A4EA
:10D1F000A1383AF5F96A3AF5F8563AFAF92839C3F6
:10D20000A2DC3AADDF363AF5F7B43AECF9C43AFEAF
:10D21000F89839929F0A39929ED43B5D2D0039923D
:10D220009D9C39849C7C3B541DDC3AC8D4B03B198E
:10D23000FE5039D5A12C3ACDD4803AFAE6F239B174
:10D240009ECE3A73BB843B73244E3A19A7203A977B
:10D25000BB8A3B27F694398D9ADE39DA9F583A0B10
:10D26000A1F83A22A28E3A1DA1623A029DF03A3804
:10D27000A1DA3AE3B8603AE8B84E3A269EC23A1DBF
:10D280009C6A3A61A10E38B58FB63C8A4E783A65F1
:10D29000A0D83A589EAA3A469DA83BA9E6E63A1D70
:10D2A0009C103A4F9D543A8EA0CC3A9BA12C3C2323
:10D2B0000CC63C0CFCDC3C1AFD663A8E9B203C50B4
:10D2C0001C4A3AE8A1E63AA99DA83AF5A1023AF526
:10D2D000A32A3AA99C2E3AF1A0FC3ACD9DF03B033B
:10D2E000A1E03AF1A0FC3AC89D783AD69DEA3ACD41
:10D2F0009CCA3C7D0C243B15A1023B22A1D43B07D8
:10D300009F1C3B199D723B0C9EB63CA5121E3AF128
:10D310009D3C3AFE9D4E3AEC9DE43C5DD5AC3B27EE
:10D320009E743B199C283B4B9DEA3B4BA1383CAE7D
:10D33000F1D23B3D9E683B279CA03B309D363B2B6A
:10D340009D603B309D6C3B589EBC3C74D0423BC4BE
:10D35000A1F23CF60C603CE000003B4B9D423B548C
:10D360009D543CE900243CF200123B819EDA3B854F
:10D370009EDA3D08006C3B6F9D3C3CCEE1163B9332
:10D380009E4A3B739CA03CF6E86C3BB29E083BB2C5
:10D390009DEA3BB29DDE3BB79E0E3BC99E683C15A5
:10D3A000A5943BC09DEA3BC09DEA3BCD9E0E3BD67B
:10D3B0009E0E3C86B1E83BE89E503D23E7403CFF93
:10D3C000CFDC3BED9E5C3C089EAA3C089F163C23AC
:10D3D0009FE23C3EA1563C279FB83C7DA7B63C351A
:10D3E000A0003DF22DC63C1E9EA43CE4B6C23C27E4
:10D3F0009E4A3C0C9BB03D04B7823C81A29A3DA65C
:10D40000E1A63C549CB23C6F9EB03C8A9FA03DE993
:10D41000F5863C989C3A3E3600903CBC9DEA3CC95F
:10D42000A04E3DC1B8DE3CFB9FA03D0DA1203D08B4
:10D430009EC23ED310CE3DA1A6723D2C9B803D4C9A
:10D440009D783DD3A4263EEAE3C83DA69E4A3FCF41
:10D45000462C3DB89E74401C51123F7520C43DE5DA
:10D46000A1503F0EDA8C3E70ABBE3DC59BE63D8BB6
:10D470009BFE3E12A12C3E049E443E169E4A3E5107
:10D48000A36C3F7ADEB83E3A9F883FD40EAC3F9EF5
:10D49000F1183FCF080A3BF18C863E519C464292E0
:10D4A0006E2E3E94A0183F0EACDE3FE6F2503E904A
:10D4B0009E2C3EA29EF23F71B8A83ED8A2A03ED8B4
:10D4C000A16E3F00A3F03EDC9FBE3ECF9EB6409AC9
:10D4D00021E43EEA9F7C3EEE9FFA3E8297723F5FD8
:10D4E000A65A40A71A403F0E9FA6413C48AE3F298E
:10D4F000A078407FF74840D9223840C2139E409A16
:10D50000F7003F099C9A3F449F7C3EF3995E40FDA3
:10D510001CD441011C923F87A1FE3F75A0C63FC6A7
:10D52000A65440B0E16A40F806A23FBDA43E40F4D4
:10D53000F718412EF7424133FB0E413CF742416D53
:10D5400007AA3FF89E2C410FD00C417201983F6C06
:10D5500096EE40C2B62641F4380A405FA47A41B53F
:10D56000120041D018D2416DE1584052A1AA41BAEF
:10D570000168401C98C841A3C29E41A3C292424187
:10D58000086A401C95EC420BE5C64125A8104218DC
:10D59000DA5C422AE1F4433D490240D09826414EEC
:10D5A0009EC84284E5E44289E5EA412A9B624188BB
:10D5B000A00042F9F5C24314E0F24319D9B443A0E4
:10D5C0001B304365F96A431DC10C42D5AF0642DAF0
:10D5D000AF18439BDFE4442211C443F5F26E43FAD3
:10D5E000F26E43D6E1164302A55E4307A4A4430BA3
:10D5F000A49842DEA10843F5F9524319A486446F6A
:10D6000017764334A4AA4481099C449C071A44A970
:10D61000070E44BB06F64511318043469F0A45423A
:10D620003EF44485D40244FA06D845080E4C44FA28
:10D630000732451E0E88455D250243D69F40450CA6
:10D64000F8EC45620BC4456F079246BC5D48459CAB
:10D650000AC84542CF164794686444A0A58E47AFD8
:10D6600068BE46110F4E45FBFDF0462C0C4846089F
:10D6700001AA4608DD1A46820DE6469410C846E027
:10D6800025EC4674D2524C4A76AA4700066C4700F5
:10D6900004D446CEDF0046CAD9664817559247944F
:10D6A0002F3447942F404E93789647AF2F0447C6A8
:10D6B0002EF847CA2EF84728D92447F339C04787A0
:10D6C00001DA475AE65C47EA2EB647F72EE647A648
:10D6D000FB8C478BE2D848322F0448322F0A483F50
:10D6E0002F04483F2F2847A6DA6247ABDA62484842
:10D6F0002F284799DA6847D3E8364716A66647E5E4
:10D70000CD604844F6284F74788A486300A848687A
:10D71000F61049293FFC48F3195647D3A5A048E124
:10D72000F5E647DCA58849953F964929F5E048C6C6
:10D73000C6884971F98E499E0E70497AF4D24BAD74
:10D7400069F04A45472849C7F514499EF51449BE72
:10D75000ECBC4A0604504AD047284ADE47644ADEF9
:10D76000470A4A64F4484A91017A4A4ED7A44B4E7C
:10D7700047584A96F01C4A45C4DE4B72445E4B80C3
:10D7800046984B1826764B8046924B4E317A4B92F8
:10D7900046984AFDF1D24E9870C24B9F3E824B2F65
:10D7A000F81A4B4A1A6A4BC3468C4B771CF24B7BD8
:10D7B0001D044B4AF1064C0742544B4AED7C4B7B0F
:10D7C000FEE04CA95B024A60A13E4B96F3E24C2678
:10D7D000113A4C34F1424C38DE1C4C65F1844C5803
:10D7E000DBD04CCD13624CD613A44CEC20DC4CC8DF
:10D7F000E8064D19ED704CF5EA0A4D10ED6A4D2220
:10D80000DCEA4EE061204D7CF55C4DC91F084EE915
:10D8100061564D5DE1284D85F1664CBFA8524E39E9
:10D8200021724E5429764E54297C4E7D2F884E0C01
:10D83000ED584E982F8E4E8120704E35F2684EA5D1
:10D840002F944EA52F8E4E08D94E4D58A7504E08F6
:10D85000D9484E30E2904E3EE26C4ED22F944EDBD1
:10D860002F7C4EED33D84EE42F8E4EF22F9A4EED94
:10D870002F944EF62F8E4EF61D6A4F1A2FD64EDB82
:10D8800009E44E98131A4EC5EF804D939EF84F2829
:10D89000226E4F16FFB24F1AFFB24EFFEC5C4F3EA6
:10D8A0000D9250515C40505A5C644F7D24724F7011
:10D8B00019BC4F7019CE50F364C24F62E7D64FFBCC
:10D8C0002E2C4FE919B64FE00C064FAFED944FAF39
:10D8D000EA4650513192501B10564F1FA876503FC8
:10D8E000192C508736AE50991E545036E3025043DF
:10D8F000EB9C505AEC8050FC372C5090EB18516C3C
:10D900004A46503FBD0450B8E8C65183499E50C1B5
:10D91000E90251CB4AA05105E52A51630D1A4FF790
:10D920009E9251992C7C51EF4938512DEB2A512D63
:10D93000EB485100D37E5132E662530166B4503A4F
:10D940009E3850369E38521336E4521336DE5264F7
:10D950004CC851ABDE7051ABDD4A522525DA522E50
:10D9600025F851CFCA9C5229D990523BD9B452B50F
:10D9700017045271E20C53574E0653724E185391CE
:10D980004FC252F80D6E53D554DE53AC4FB653CC44
:10D990004FAA53DE4FB053E24FB653F94FCE51C6A4
:10D9A0009B985313DAE654064F44540B4FB653601A
:10D9B000064254144FCE54214FBC54184FB6540253
:10D9C0004A5254064A5253CC38285306C9CA537295
:10D9D000EA525384E71653E2217253E7216C537BDA
:10D9E000DDD453A8D8B8541D352253CC0A8654022E
:10D9F000235E5414235854B14F8C53B5D5B8543CBE
:10DA0000261654180B3A5445260454723804543CD4
:10DA1000FF1C547B380454210B4C54C85016544EF0
:10DA2000231C542A0A8C54B647585421EBCC53A8D3
:10DA3000B674547B1F80545707E655144B545469F1
:10DA4000F0D654A8161A54BA0C0C5480E53054C3BE
:10DA50000D5654C80D3854EC20E854D10D3E54DE18
:10DA6000163E54F91C625414AA6854DEEEAE55A951
:10DA700047EE55C847E254D1D85E55EC513C55733A
:10DA800018EA5703677A55CD3714555CEFEC559774
:10DA90000B46554FD86455AD372655BF191455C49C
:10DAA000190E55C8190E562B2FBE559BD5F456A5E9
:10DAB0004E4856582370565D236A56B240B05661A0
:10DAC00005165642EDF456A0250E56F64500565D55
:10DAD000EDD056A932FA5831680A56DF1E06568E26
:10DAE000CB145642BAB856CDF7D857B7514858B3A9
:10DAF000681658BC673E57C54656577D1D64578605
:10DB00002100578A010857C01D6A57C01E2A57C9ED
:10DB10001CD45762D96057E01D8257D2068A57F647
:10DB20001DB857FF1DA057A5E15257DB1EFC57AA91
:10DB3000DC2A57A5D4EC578ACBD458281D5858282E
:10DB40001D6A57B3D63058231AE811EE8260580880
:10DB5000F36A5862222658672430585E1FB658234D
:10DB6000ED465816CD1E582CD55E58AF1A2258D304
:10DB70001C985874F8F25874F8F8587DF91058AA9F
:10DB8000F9105882D6845874D19E58AFF3AC58CA55
:10DB9000FF285AF36DBC592424845916186C592D4A
:10DBA0002460593F1E365931184E59A61E3C59A6BD
:10DBB0001E365A091FBC5A7E4A2858DCA0365A9095
:10DBC0004A4C5A9E4A3A5A3A298E5A994A525AA768
:10DBD0004A405A5625F25A9428085990AA145A3F96
:10DBE000E94A5A9E23345A51ED825A3FDFB45BE62C
:10DBF00066A25A75FC705AA2FD665AA7FA4E5ABD23
:10DC000000FC5AFC28625AF823165B0123285B1B90
:10DC1000230A5B2024365B131BC05B201BB45AA273
:10DC2000C6D05AEED5E25B7F211E5CAC66A25C5B7F
:10DC300066B45CA866A85B6D1C1A5CD568345CE2AF
:10DC400068045B25CF1C5CE267985B9A1BB45BD4CD
:10DC500034565C0A46985AF3B27E5CD566845B887B
:10DC6000FA365BB51BBA5BAC07025B37BF025D3CA3
:10DC700067505BDD1BA85BE214165C2130D25D2A85
:10DC800062DC5C1C10925BFCFAEA5E266E465D0666
:10DC900054AE5E266DFE5CC74BC05C5B0D985C01AC
:10DCA000D2165BDDC0CA5BCBBDB25C7611C45C69C9
:10DCB000EAB85C4ED0785CAC11B85C76E4E25D2AE0
:10DCC000422A5CDD1ABE5D0F33965C45B5845C600C
:10DCD000BB665C7FC51A5D0A1AD05D0F1AD05CD98D
:10DCE000EBEA5D804B605D6E42DE5D2A1AB85D3303
:10DCF0000FF05D6E2B685D6E2B685DC8482A5D3C39
:10DD0000109E5DA42EFE5E0245185E2652985E07A8
:10DD100045185E0B451E5E18450C5E14451E5DA43D
:10DD2000FC525E0237985E6549385E6548365E652E
:10DD300048305DF5FBAA5DF0F8FE5E10FBC85E267C
:10DD4000FB865E34FB925E2BF8D45EC44B9C5E3443
:10DD5000FBB65E34FB625E61375C5E38FBC85E45D5
:10DD6000FC5E5E41FBB05E3DFB445E45FB685EE3EE
:10DD70004E4E5E72184E5ED63F2A5E72041A5DC821
:10DD8000ACBA60596DCE5E8004565E65DD505EBBF8
:10DD900008DC5EF932405EC80FB45EBBF94C5EB67B
:10DDA000FAC65EF5047A5F19324C5F1E0F965FC9A2
:10DDB00054485F1EFB3E5F3D0F905F30053A5F5356
:10DDC00017AC5F4B0BAC61476F5A5F4BFAC05F7388
:10DDD00017AC5F6124785EFEBF745F9C1ECC5F9CB5
:10DDE0001EE45FFA48C65FFF48C05FAD19B06042ED
:10DDF000550E5FCD23285FC019F85FBB19AA5FFAE3
:10DE000031BC5FDA19EC61556B8E5FDF19C25FEDD3
:10DE100023C45FE419AA5FED19C8603023A05FCD69
:10DE2000E52A60503AAA60814BBA5FE4E53C5FDFC7
:10DE3000E536606F34E661AF6B6A603E19EC60A551
:10DE400046EC601EEA3460611E2A604204C26078BB
:10DE50002A0060B346E660F6546C60C046F2609CEF
:10DE60002E9260C546E06047DECA609C0A1A60C90F
:10DE70001A4C60BB09E461113F3660CE0A2061157F
:10DE8000313E6115314A6128311A60F2EB2A61672F
:10DE9000386A61502A2A6115DE046198398A616204
:10DEA0001116625061506081A078618F29D0618F16
:10DEB0001BBA618F18C0611AC45461E0306C61BC38
:10DEC00018C061C118CC61DC2B7A61CE18F061FBFF
:10DED0003B1062003B10623149DA61DC1C0861DCF6
:10DEE0001AAC61DC1AAC61E01C68627D5A2461E9FD
:10DEF0001C3261E91C2C6108A4C861EE1C3862CF99
:10DF0000650461C5E90E62041C0262091BFC62A67D
:10DF10005A5A61C9DEC462A2550261F6F95861BC61
:10DF2000CC82621F16CE62C15A6061E0DA4A616239
:10DF30009E1462502FD0624324F062552F706255B8
:10DF40002F46624C2FA0625A2FA6625A2F58626346
:10DF50002F7062632F7062672F70626C2FB86270CF
:10DF60002F6A6212E09261559E806228E8CC62902E
:10DF7000374A628B2F58629431C262CA47AC61AA99
:10DF8000A75062821AA662C138766231CA90626C6A
:10DF9000EB5A6275E8C66279E8C06250C706629DB6
:10DFA000F916628BE8D86300387C630438886324F0
:10DFB000453662B4EF3E632D4542633B456662F3EE
:10DFC000046E6331308A634D39C063120300634DC0
:10DFD00025A46312F160632D085E630EDF6C62CAD4
:10DFE000B82A62AFADFE6309F15A6312F15463CFF0
:10DFF00050B26371101A63711014637A101A63754A
:10E00000101463751014635AF68E6375031E6375DE
:10E0100002EE6363EF98642057E4637AEF2663951A
:10E020000B28635AD0126390EFC264202046639598
:10E03000E1646304A642638BD89463B4EFA463994C
:10E04000EB9063A2DD1A64B55F16643F29886417FC
:10E050000ADA649E50D6643F214264290318642979
:10E0600002E263ABB11C643F05D0649E2BC2645BCB
:10E07000EB4864951E3C643BD54664951E4264950E
:10E080000BE2647AE8786692700E66A85CCA644413
:10E09000B59C64DD0E4664D90E4664E60D5064E618
:10E0A0000E3A6387943C65131E8464FDFC7C6537DF
:10E0B0002C94650A0E7664F3E2AE6506E28A656426
:10E0C00034FE6540178E651CE8F064D9B4DC6584C5
:10E0D0002E2C6576212A657A17DC657F208E658473
:10E0E00020A0658820AC6520BDFA659A17EE659A78
:10E0F00017EE6560E248658D03D8658D03D865A786
:10E100006B52659F0D62659F0D8065AC17FA65CCFB
:10E110002FD065B517F465D42D726588E10465CC00
:10E1200017EE65ACEE8465C309C665F4179A666997
:10E1300052C265E7FFAC65D4F1BA660614DC660B23
:10E1400014FA662E327665D4E5246758669C660F0D
:10E1500010B666DA6078660F050466E76078661DBB
:10E1600007446753669C66772CCA668432F4665708
:10E1700006906653007866842CE86645F3E2669262
:10E180002CFA669B32DC6601B938659AD5A06669BF
:10E19000FACC662AE896673D5F82669F6948668981
:10E1A000F24A6680F1666684F27A66D52BBC6660B8
:10E1B000C1D8669BE33266960F9067C865A666B6BF
:10E1C000E21266F006F067261EF666E7E62667109E
:10E1D000080A67261EF666F5EBD866F9EBCC6738B9
:10E1E0001F1466ADB2F66719E1A066F0D426677C0D
:10E1F0003DFE66DEB914678E3E106710D534678920
:10E200003DF267772EFE67923E0A67923E1067974F
:10E210003DE6674AF6F467A43DFE67BF3E4C67D112
:10E220003E5867A92D4E67AD30CC67BB2F3467923F
:10E23000F958679B019867A911DC678EFC0467A9F0
:10E2400000DE67B611E867BB120667E32F2E67ADE5
:10E25000F8C267B200DE67CD11F467A0E16A67DF3C
:10E26000282668B7658867B2E50C677CF4AE67BF9F
:10E27000EECC68B261206815291C6780B0AA68BB23
:10E2800061FE6807F66A6797A7DA67F5D9FC67F158
:10E29000D1F268270306683D1B5468421776684F21
:10E2A00000FC68CD5364685D023A6846E5C6684B79
:10E2B000D9966885FE2C68971728688E0D086878AF
:10E2C000F16C6861D9A26881E5CC68B2171C6881DD
:10E2D000DBDC68A506006881D8346A7470E668548F
:10E2E000EE6C67BF980E68D617B268CD6AB068DF6B
:10E2F000020469C0657068B2F70C69CE657C69DBA1
:10E30000656A69302D846935289E691A0EB2691EC6
:10E310000E9469472C76690CE4CA69A14E36696B84
:10E3200031C8694B14466911E66E6A0D60A8693000
:10E33000DA2069D24E4E6974125A6962DFE4694785
:10E34000D5586974FBF8694BD9D86966E49A698134
:10E35000FBD46954CFE269AA1F806966D828699303
:10E36000FBDA6981E46469A1FBC869A5FBDA69BCD1
:10E370001632697DD3A26998E45E6A3A549069E0E6
:10E3800022C269F22DFC6998D37869C5FBCE6A4731
:10E39000548A6998D3786A28394E699CB2FC6A28F5
:10E3A0002BDA6A0D132C69EDD3726A04DB3A6A31F9
:10E3B000F6E86A8F42786A2CE2CC6A3ED7FE69F2B0
:10E3C000AB766A62F5266AA12BBC6A8F04146AC117
:10E3D0002E746AA114226A6BCFE26AAA143A6A9D6B
:10E3E000F6D06AB300186AA6E4FA6AA1D5E86AE929
:10E3F0002CD06A94E9566A82E9566AF219E66AE90B
:10E400000E0A6B0019AA6AB3C7246ABCEF326B24E8
:10E4100011586B6340A46A7DA13E6B16D7206B1226
:10E42000EF2C6B3FEF6E6B24E8A26B1BE89C6B3FFD
:10E43000F4126B3FEE4E6C32685E6B43EE846B7091
:10E44000E2A86C7167386BD346F86A238EEA6BD307
:10E4500036666BD8364E6BDC369C6BBD11D06BC606
:10E4600017FA6C90688E6BB404686B8BD3846BE581
:10E4700036846BEA365A6BEA36A86BEE365A6BD89E
:10E480001FF86BF3365A6C244FB66BD804C26BE599
:10E4900004D46C0929A06C5A54B46BF704E06C4D99
:10E4A00041886C36E2F67CCE7D526C05D9126D2027
:10E4B00069AE6C0ED7686C29E5426C631DB26C4D79
:10E4C000E9CE6CA239CC6CA73A3E6CAB3A386CE61C
:10E4D00051D86D4D684C6CB03A3E6C901E7E6C907D
:10E4E00009C66C991EC06CEF50BE6CAB1EB46CA715
:10E4F0001EB46CD441586CCF41526CB41ECC6D83A9
:10E50000692A6B248E486CC626E86C006D6E6CF828
:10E51000400E6C7AAE8E6CBDE6B66C90BEBA6D13D2
:10E520003C7E6CEADA746D05271E6D203C666D4DED
:10E5300050106D293C6C6CEFDBA66D1723D66E4036
:10E54000704A6C99A7E06E6970326D371BA26D88B6
:10E5500050346E91702C6D49219C6D3B0F4E6E2195
:10E5600068FA6D76363C6DA350346D641E546D713F
:10E570001BF66D44CFD06D44CF346DE251C66D951E
:10E580001BFC6D9A1BF06D4DB7466D9500186DA381
:10E5900011A66E2A5DF06DBE27666D56E0B06DD98E
:10E5A00025FE6DD927666E2E56286E0137C26E2A5B
:10E5B000507C6DE218246DC7E15E6DBED2526DD401
:10E5C000E5CC6E1CFC4C6DF4C7FC6E4528146E2A1D
:10E5D00005706E06AE886E5B201C6E18CED46E2160
:10E5E000C7D26E9F24AE6F8467BC6E7B11DC6E9FBA
:10E5F000297C6E21AAB06E5BC2446E88CDD86E8D28
:10E60000CDF06F335B7A6E96CDF06E91C1366E9A17
:10E61000C1E46E9FC1F06F2A4EDE6EF028806F530A
:10E620005B0E6EB5CE566EBECE506EBECE7A6F020B
:10E6300022F26ED5CE446F2128026ED5CDEA6F2628
:10E6400026E86EE7CC586EF0C7D26F41281A6F06E5
:10E65000C7D26F8D0FC06F33EE366F14CEFE6F26AC
:10E66000E0A46F41BF326FCC52506F60D9666FDA51
:10E67000526E6F961E726FDE52566F7BCE506FA435
:10E68000E7B86FD134626FBAF74E6FC3AE1C6FDA62
:10E6900034806F38EE3C6F38EE1E6FB1EE2470029E
:10E6A00046746FDE11DC6FE713EC6FF51EC66FC3A7
:10E6B000D27C6FFE1980701434AA6FDAD9CC700244
:10E6C00011CA6FDAD9486FDED96C6FE7D94E704640
:10E6D0004B3C6FECD9486FF9D93C7010DC66700286
:10E6E000D9127007D8F47014D930700BD95A70074A
:10E6F000C574705C3A9E706E42A8704AEF9E704A74
:10E70000EF9E7073239A7007AD8C7061FFB2706AD0
:10E71000072C708021DE70730CF671546C0670410A
:10E72000B3DA7053DE8270920CEA707CCD4E70BF0B
:10E730003474706EDE58708ED8F470D1070270DFBA
:10E74000135670E3FF7C70E8FF7670F5071470FADB
:10E750000D4471936726711E230A712210DA712706
:10E7600014E870FECCDC71C4666C712B097E7146B6
:10E770002B327134107471421F7471734EB4710C6A
:10E78000CCDC711EDF60713D097E714613CE7122B3
:10E79000CCD671A958E67142EFB07146EFAA715814
:10E7A0000948716F1F0871FF65D6719C028E6FA8B2
:10E7B000C29271A9135671B2109E71AEDC7E71C007
:10E7C000184871BB1368712BABD071C4133871E456
:10E7D0003CB471BBF20271CD088271DB13AA71A93E
:10E7E000C7BA71DF11B271F1283871FA30CC71FFFC
:10E7F00033A871C9DD9E71F611C471F106EA71F199
:10E80000070871F1070871F60C1871FF11A071ED7E
:10E81000D3A8721113FE726F5C7C71F6DC9C725D82
:10E820005C6A72392E62723E2E6272FF6CAE728624
:10E830004DE2722716CE726628087254082872427A
:10E84000EE3072F2679E7250EEF6723516D4729305
:10E8500047C472AA565272A5522C724BE80672989F
:10E8600047BE7250EDEE726B12DE727D2E14727D19
:10E87000275A728F3D7A728F3D8C726F0BEE727DCC
:10E88000278A727D139E7247E7BE7266EE7E7274AF
:10E89000EE907278083472932E4472810C0C728A56
:10E8A00019F872810BAC72810D0E726B0D0272A59C
:10E8B0002E567278E81272B3337E72A10E46729CA5
:10E8C0000558731A563470EC0B2872B7204072AE9C
:10E8D0000EDC72AE0C0C72F2505272B30A2C72CE75
:10E8E0002FB272C918B472C90E5E7311502272A190
:10E8F000C08272DB179473164C6272C5D1B071ED91
:10E90000E2AE7308264C72FBEFF872E9E15E730D1C
:10E910001866730D184E72FBE974731618C673509F
:10E9200050527316E800731A18C0731F18D273314F
:10E930000AD47328DB467316E26073E569C0735E20
:10E940000DB673700DBC738F39967379EBE473CA8F
:10E9500053B273DC5688738BE46473AA181273AFD6
:10E96000180673B8221473AF0D0E73B30CF673EE62
:10E9700040DA73D3EAF473D30D2673EEF56E73C5E4
:10E98000BE7E73D7D7F8748B6A9E740414DC741639
:10E9900028BC742418BA7443511E7412138C74006A
:10E9A0000D2C741F111C742D0EC474482700743A6A
:10E9B000053A743F051C73FBAB287443E4A0745AFA
:10E9C000143A74944F0E745169C67487194A74636B
:10E9D000EC20743FABD674942754747EEA3A749456
:10E9E0000F9674A219807487E91474CA06CC74ABAC
:10E9F000289E749DDF8A74B8276C74AFDF4E74B4A0
:10EA0000E58A74D327B47536660C75004F7A74C6E0
:10EA1000F6E874B8A9B474FCE6C87509FFF4752D5E
:10EA20001C38748269A8752910087524E4A6753FFE
:10EA30000A14754D2820754DE4A0754DE482758C3F
:10EA4000507C753B0A147524AD807548CBBC758C21
:10EA50002568758306CC7590280E7587F154760A63
:10EA60006A44759E285075A732A67590F0A075C6A9
:10EA700033F675EA564C760AE64A75CF33FC75BD17
:10EA8000ED2E75C20F1275D832AC75EF4B1275E1D1
:10EA9000287475B41E8A75E1285C75E1285C75E6FA
:10EAA000285075B91E90760A4E4875C6CB3875EF5A
:10EAB000282675E610E675E60FBA75FC28627649D9
:10EAC000667E760525EC75E1CB3275C2E3D475C25E
:10EAD000E3D47601083475EACB56762531DA76250B
:10EAE00026CA760AE64A75D8AB4C7601CC2E762932
:10EAF00026D676521FE07617A9AE767143E07644AB
:10EB0000E992761CA9E4765B05287625A9CC762EB9
:10EB1000A9D8768343F27632A9F0765BDA62763B47
:10EB2000A9BA769E4D5E767A1CB076B0555C764971
:10EB3000AA86767FEC38768C18487695120676D9B8
:10EB40004E5476B942BA76AC14CA7695DEA676B043
:10EB5000184876B9197A76CB3A8076BE073276CBEA
:10EB6000187E76ACA9DE76E2065A76F8195676DD7E
:10EB7000D07276FD19627701198677252574774062
:10EB800052AA771806667737257477495190773CF3
:10EB90004056772E20E8773714B87725DB4677453F
:10EBA0002106776D513C76D994D2773CD1DA7791B2
:10EBB0005E927757126677520A98779F5142778D07
:10EBC00019CE7791124277961320779F25EC77968E
:10EBD000042C77B54AC4779F1986779A050A77A3DC
:10EBE000F35277A3F352779AF18A77A8F190779648
:10EBF000F49C77CC19F877BA048C77BE048077F050
:10EC0000531677C7043E77CC03F677D0043277D516
:10EC10001C5C77D0041477FD381677EB1C6E77FDFB
:10EC20001D1C77F4222C77FD351C77F922207841C2
:10EC300061A4780B1752782A4BBA78384A6A783C24
:10EC4000363C7833190E782AF3D0782FEC98783345
:10EC5000FE74783CEEBA784E04B0785C3684784E18
:10EC60000FF6784AEC927880593A787B512A785C92
:10EC700021AE788D550E7869F2387872DA6878A806
:10EC8000503A789B3D4A7884F11278A4420C789FE0
:10EC90002736789FF8267889C32E78AD17B878E3A1
:10ECA0005DA278DA4FFE78CC17F4789F05D078E330
:10ECB000183678F0298278E7F31C78F92418790758
:10ECC000525678F917CA79020D3878F9ED7C79191E
:10ECD00031C87926320A7914F02E79101D40791D39
:10ECE000322878F0ABB2793431F2792F21DE7953C2
:10ECF000F3887938F3E2794AEFD4794F0D0E793DF4
:10ED0000CCCA794FEFC8796AFB7A796AFB6E79775A
:10ED10002004792FF070797C282C79922796799BA2
:10ED200027E4798EEC08799704EC798ED55E79BF6B
:10ED30004AA079AD012679B601207A10F2867A15BB
:10ED4000F26E79B6F1FC7A15F26279F1570679DF45
:10ED5000422479F1EC8079DA226279F54AB87A1E98
:10ED6000F27A7A0711A07A07F2267A2B4D227A1EC0
:10ED7000EC2C7A5863307A4667507A464D467A4F83
:10ED80004CAA7A4623407A61545A7A583FB47A3D65
:10ED9000CAA87A4F1E907A4F20587AA51EF67AA5F7
:10EDA0001EF07A9C69727AA91EFC7A4FCA967AAED6
:10EDB0001EE47AAE1ED87AA069DE7AAE1EEA7AAE7A
:10EDC0001EEA7A7333367A7C4C5C7A8A522C7A6AE1
:10EDD0001E607A814D166FF51EC67A7C20587A9C8B
:10EDE00056DC7A6AF22C7A81192C7A8A21EA7A5DC9
:10EDF000A95A7A9317BE7A8E191A7AA5435C7AB209
:10EE000053D67AC4F2E07AA91FEC7ABB110A7ACD04
:10EE1000F35E7AC0F1127AC0FB507A5DEE547AC488
:10EE2000B8AE7ADBF1127AF14F207ADF25147AED51
:10EE3000416A7ADFCAEA7AF125087AF625027AFF72
:10EE40002CE27AFF1CCE7AFF2CE87AB7F2807B03A3
:10EE500018EA7B03F2CE7B0307087AF12CD07AFA0A
:10EE60004D9A7B11526E7B2754CC7B112CDC7B1589
:10EE700022C27B1515907B1515967B1A18F07B1A0C
:10EE800018FC7B1A190E7B354F087B301CA47B3095
:10EE900019087B3019027B2C1F927B47543C7B392D
:10EEA00010207B4743147B3E22F27B4733667B5026
:10EEB00022E67B5922E67B5D1C4A7B620E827B66E2
:10EEC000F75A7B6B0E947B6B0EA07B6F1C987B6F4D
:10EED0000E767B6FEC867B8A4A3A7B780E767B785F
:10EEE00025447B811A827B8F17347BAA4A227B9C24
:10EEF00025627B9CEDE87BAA1FF87BAA0E4C7BAEBB
:10EF00001AD67BC5548A7BAAE8607BBC1BFC7BC9F4
:10EF1000517E7BBC0F307BBC1C3E7BC01C1A7BC06F
:10EF20001C0E7BBC0B287BC01C2C7BC51C207BD7FC
:10EF30004E487BC92EE67BB30E707BC904747C08F7
:10EF40004E967BCE1C1A7BD20E7C7BD2174C7BD785
:10EF5000F2D47BCE2EE07BD22EE07BE41B7E7BE9DD
:10EF6000F2F87BE91B607BDB1BDE7BE41C207BF281
:10EF70001B907BF20BEE7BF61B487BE9F3047BFBDB
:10EF8000F2E07BFF1B487BFF1B5A7C110F3C7C1679
:10EF900046987C232E867C11135C7C0D1BD27C1141
:10EFA0000C067C111BCC7BFF0CEA7C1F42CC7C2323
:10EFB0002EB07C4361987C282EA47C312E927C1F3D
:10EFC000B0BC7C3E1D1C7C231CB67C3ED8BE7C4C59
:10EFD0001BEA7C4CE84E7C624EB47C704ECC7CB319
:10EFE00068887C742ABA7C74F0947C8F44827C9804
:10EFF000538E7CA653947C9D44767CA1313E7CAAA2
:10F000004EDE7CAA25387CAA25FE7B936CD87CAF8B
:10F0100024BA7CA6CB447CAAD6D27CA6F2507CC172
:10F02000441C7CB8FE807CCA11227CBCBC267CCEF1
:10F030001E0C7CB323167CD3253E7CE94DD67CE99F
:10F0400009427CE9F8C87CF24D8E7CF248E47CDC15
:10F05000AF967CE91C267CD323167D004D767D047B
:10F0600046927CFBD7807D4346567D091ED27D1299
:10F070001F027D1627967D1F44767D1B1D8E7D1FEA
:10F0800035767D0449207D3F44287D2817A67D31B3
:10F0900017B87D3A2D967D36DA2C7D481D0A7D4CB9
:10F0A0003E0A7D5E69A27D481D8E7D5134027D0D34
:10F0B000EFF87D511CD47D5A24E47D5E55567D6762
:10F0C0001D9A7D671D2E7D671D827D7543507D7560
:10F0D00043687D7520E87D75FA607D7949987D7576
:10F0E0001D647D82DF6C7D82E3147D82E47C7D9DE6
:10F0F00052147D9DF5207CF7B1AC7DAF61807DA27F
:10F10000EC5C7DAF52447DA627C07DB4F0B87DCFC6
:10F110002D487DB8F4FC7DC610D47DB4E5607DBD7E
:10F12000EF147DCA2A307DD34DCA7DCA10E67DCF4B
:10F13000EF207DD855207DDC097E7DE14DE87DE521
:10F14000551A7DE1FC347DE14DE27DE1E4047DF37F
:10F150004D887DEE21967E2D28DA7DFC43F87DFCDE
:10F160002D067E1723707E1B27367E1B237C7E2474
:10F170004E007E202D787E244B127E2423827E2416
:10F180002D667E292D6C7E2D14227E2D23887E32C5
:10F190004DFA7E48235E7E36235E7E3B42907E366D
:10F1A00020A67E3620887E3B27367E3F23587E3F32
:10F1B000FD127E3F23587E4427A87E4823767E5149
:10F1C00042787E4823527E4D0E1C7E4D3DCE7E51B0
:10F1D00016C27E56233A7E4826B27E5626947E5626
:10F1E00023A07E5F13FE7E5F2AC67E63234C7E6370
:10F1F000237C7E6823287E4DE6327E6C35287E7522
:10F2000047AC7E7AE4E87E8C16D47E950B887EA28D
:10F21000FE747EA72CEE7EAB1C387EABE6E67ED479
:10F22000617A7EA7E9927ECF570C7ECF12D87EE618
:10F23000E5787EE6E5727EF319147EF357607EFC76
:10F240001C567EFC061E7F01FFBE7F0A02CA7F0E8F
:10F2500002767F1344647F1319567F171A647F1355
:10F26000E8FC7F203EA07EE6A7207F201BC07F20F9
:10F27000516C7F371DA07F441C927F7F1C927F3B87
:10F2800005047F401DFA7F491C9E7F491C6E7F4903
:10F290002CDC7F4902A07F4D19F27F4D1C6E7F4D03
:10F2A0001CA47F4D0F427F4449F27F4D1C987F4D37
:10F2B0001CBC7F4DA15C7F521C6E7F5B02AC7F5FEC
:10F2C0001C987F6402EE7F5F1C687F6402887F6801
:10F2D0000EE87F68FCA67F7125F87F5F5A9C7F7FD0
:10F2E0000F067F7F0EEE7F7F1DDC7F8346CE7F88FB
:10F2F0001C7A7F8CDAAA7F8C47167F8C1CEC7F8867
:10F300001C927F911CEC7F9A1CD47F9A1CE67F9AFA
:10F31000EB907F9E1CF27F9E42C67FA333D87FA3D3
:10F320001CFE7FA31D0A7FA745BA7FA723F47FB0E9
:10F330004A227FBEA9DE7FB9279C7FBED6247FC22A
:10F34000D6247FBE0EE87FC25E747FC73C787FD034
:10F350001A107FD03C907FD0C77E7FD42FD07FD42F
:10F36000EC0E7FD414467FE603CC7FEF3CA87FF4FD
:10F370003CA27FF40D6E800F61CE7FF45B927FD450
:10F380002E688001040E80010E9A7FFD5BAA801812
:10F3900016B6800A6C00800F60B48021F34C802187
:10F3A000FA60801829348025291C80136960802E1A
:10F3B000290A802E3DE080332A1880333E04803CA9
:10F3C0003D6E8040028E80450288804552C2803C5E
:10F3D0004AAC80403BD08052415280523816806007
:10F3E000252C80571A168057327080645202806D27
:10F3F0002AC080693768806D168C807619D4807237
:10F40000520E80761ACA80763780808446FE8088C5
:10F410001C6280726B16809A3D868091513080A864
:10F4200021EA80B532DC80B1129080B512A280B59D
:10F4300018FC80B5335A80BA129080B5290480BA7E
:10F44000291080BA291080B54F0280BA290A80BEDF
:10F4500028F880C328FE80CCF32880D0EC5080D0E0
:10F460000F4880D501D480DE09E480EB476480EB4F
:10F4700005B280E73D7480F4A7D480EB281A810B95
:10F4800014B880EB4758810FEE5A80FD12E480F9E2
:10F49000338481020A2080FD14F481021284810FDA
:10F4A0004CB0810F53D6811827F68121082881148A
:10F4B0004EC6812A543C812A11228126EFBC81C389
:10F4C000FE8081382EB0813C1D0A812F59B88141C0
:10F4D0001254814A0D7A8145138C814A281A814140
:10F4E0005CCA814E27A28153138C815321BA814E6D
:10F4F0003318815C0900815C127E8157423C815740
:10F5000043B08172C3108169435681605D2481726A
:10F5100012BA8177096C817B0A808180EEB4817296
:10F52000422481772F22817B331881802F34819B65
:10F53000B278818442BA818442B481920AB68196BB
:10F54000052E81960A1A818061B08196158A81897B
:10F55000592E819B1740819FF208819F096681A4E3
:10F56000402681A8F01681A4352E81A829A081BA51
:10F570000A1A81BA0A3881B142AE81BA07E0819F86
:10F58000639081BF279C81D107D481CC29EE81DE95
:10F59000144681E706C081DA5CAC81EC081081E793
:10F5A000428481F9079281F9089481F9082E81FE3D
:10F5B00014EE8207EEC68202083A8207EEC6820780
:10F5C00007C8820B1200820B076E820B0876820B33
:10F5D00007B082024FCE820B2AA882100786820BC8
:10F5E00029A6821026D6821D0AD48219078682197E
:10F5F000292E8226EF988226EF9282260792822673
:10F6000007DA8222293A821D51B48234EF9E823475
:10F610002946823807F2822F41168241053A823804
:10F6200051B4822269FC824F0678824A19DA824FED
:10F630001032824A2796825809608258096082589F
:10F6400014888261102C82610792825C06BA826102
:10F650001488826A06488277D0EA827311E882733E
:10F6600011FA82730CB4826A2A4282770A0E82806F
:10F67000291082802910828515D882891098828964
:10F680002A06828E0D1A82920D2682892BAA828EDC
:10F690000B88826169EA82A00ED68297163E829B11
:10F6A000165C8297165C82A0076282A40EF482A484
:10F6B000088882A4163282A9163882ADEE5482A937
:10F6C000100282806B2282925C9A82AD087C82ADAD
:10F6D0000A80829B523282B61B5A82C4AE4082A0FC
:10F6E00028AA82B6088E82B6178282C80A0282B61B
:10F6F00009EA82BB09C682B618A8828E69F082B276
:10F70000421882C4FB7482C4FB2682DFA8F482C83C
:10F71000177C82C8112882CD0FC682C80AF282CD1A
:10F72000112882D1FE9882D60C0682C8449482C8E1
:10F73000522082D12C5282D60D0E82DFE59082D1EA
:10F74000521482B2696682C8522082DF0A4A82F568
:10F750000A7A82E3112282E80EE882E3376282F1BC
:10F760000A7A82F11074831999D08303C81A82FA35
:10F77000121E82F52826830306F082FE14C483033A
:10F7800006EA82FE15F083070E1682FA44AC830760
:10F7900019928307172882FE4CA4831500CC82DFC0
:10F7A0006A3883151206831911D08310403E8319DD
:10F7B0000EB283035B5082FE4080831926BE831EF7
:10F7C000199E83192F2E83221608832219C283279C
:10F7D0000F0C831E2F34831E2F34831E2F2283276A
:10F7E00012728330F5328334F532832716C2832BAD
:10F7F0001236833011CA832B273683390384833929
:10F800000CAE83390C78833D0594833911BE833463
:10F810002BE6833D0BD683460B2883460D7A834B1C
:10F82000FECE834B152A834F0384834F15C0835D1F
:10F83000F7D28354084083580D3E835811E883580B
:10F84000272A8358272A8366F48483610FA2836161
:10F8500008CA8366114C836A08C4836AF45A8366B3
:10F860000B76836F1266836F11528454002A837360
:10F87000124E838EAB7C8378114C835D5B20838139
:10F880000DC8838112788397C328838A0D448385AA
:10F890001392838A138C8385283E83853E04839349
:10F8A0001806839C0D08839C1086839C092483A0E2
:10F8B000FD48839C20168373D5A683A9050483A9DC
:10F8C00012A283A913AA83A03F1883A9128A83B71F
:10F8D000DF6C83D6A4E083BB0B7C83BB0B4C83C063
:10F8E0000AD483C00B4083C013C283C00C4E83C4B0
:10F8F0000AFE83C90B2283CD0B4083CD12E483D251
:10F9000013C883CD265283D6115E83D6132C83E48D
:10F91000115883E4131A83E805FA83CD5A1283DF62
:10F920000F2A83F60CAE83A5EF9E83ED3AA483FAEB
:10F9300011708408F4AE83FF0BC483FA178E83F131
:10F940003A8C8403102684030B5E840C00DE84153D
:10F950002442841128FE841E0588841A10568423AC
:10F9600017B28435C7CC841551848430144684354D
:10F97000177C84350FBA843EF55C843E059A843941
:10F9800012DE84D2C7DE8442083484622D248423AC
:10F990005A5A84394F6E844B59DC842C5D48844715
:10F9A00029D0845D16DA8462147C8454002A84662B
:10F9B0000B0A84740C2A8481F59E845459EE847D4C
:10F9C0000CE4848115548481EF1A84812A96848AF8
:10F9D0000AD4848F03BA848F0FEA84271CD48481CD
:10F9E0003A268498126684980918849C0348848F68
:10F9F00031F284980B8884A1031284C0477C84AAC6
:10FA000004B084A5199884AE15DE84C0FFB284AE1C
:10FA1000477C84C9089A84D2044484A5595284CE70
:10FA2000FAA884AE52E084C9146484AE52E084CE55
:10FA3000112E84D2114084D711A684E9C88684D7B8
:10FA40000FBA84D7254A84DB25D484E925E684DBF4
:10FA500025FE84E4275484E90ACE84E91B3084D24D
:10FA6000245A84E025F284F6101484F2248A84E077
:10FA70004C3E84FB0FD284FF0FCC85081284850D89
:10FA80000A32850D13FE84E0686A8531C2AA853189
:10FA9000CE14853AC700852C062485280888852839
:10FAA0000D6E8531109E8535078C85470210854780
:10FAB0000042853E2F10854C1272854328B685552D
:10FAC0000612855903C0856209848523685885829A
:10FAD000DA62857908768579FF40858BF87A859892
:10FAE000EFAA8594158485940E5285A1F7D885A632
:10FAF0000BCA85AF01AA85AA046885BCC67C85B3FC
:10FB0000F8C885C1C65E85B8F8C2859856A685C571
:10FB100010C285CE10B685CE0E468600A77485D756
:10FB20000ADA85DC135085DC0A4A85D724AE85D7EE
:10FB3000249C85DC24A88600C6D685CA46EC85DCD4
:10FB400039DE85E5315085F2123685F21062860D78
:10FB5000C6B285FB0ACE8600045085EE3A088604BC
:10FB6000F61C85F22DCC8604F63A860DFE1A86091F
:10FB7000059485F72DC08609FFE2860D142E8612A6
:10FB8000141C860D1C0E861603C6861B10148616C2
:10FB90001014861B12A28624114C86280F8A862DEB
:10FBA000FF16862D02CA86124D8E8655C54A861BC3
:10FBB0004D228636104A85E968A6863F103E865A51
:10FBC000C6B8863F1710862D52EC8648FF34864C07
:10FBD0001278863A39B4864C2D3C86552D48866776
:10FBE000F1D28663130286630FBA8682C69A866351
:10FBF00034328670F1A8867E044A867E044A867E68
:10FC0000FF58868710148690FF4086704D2E868799
:10FC10002628869DF61086B4C5568694261086AB97
:10FC2000F3D686944CF886AB2B3886D3C58686C629
:10FC3000F98E86EAC85C86CFEFAA86EAC31086E111
:10FC4000F1D886F3C59886E1FC2E86D81B6086C65F
:10FC50004CB686E531B686F7061886F7135C86FC47
:10FC6000FDB48709FB5086FC264686D864208709A8
:10FC70000F7286EA4C7A8724C5E6871BF7D887126D
:10FC80000BEE872DF3D08732EFF2873604C2872D33
:10FC9000263A873BF32E87243AF2873FF8B08756FF
:10FCA000C5F2871247F4874DF064875FC5CE874859
:10FCB0001554872931B6874823D0875A077A876831
:10FCC000ED4C8751271E8771F2BC8775F2BC877196
:10FCD000F892875F2E9E877AFA3687632670879E12
:10FCE000ED46878CED5E8783EBD8876C23DC879E9F
:10FCF000EC028787EBD88771269487ABC62887B438
:10FD0000C6228787F700875F4A58878C0F5A8790EB
:10FD100006D8878728B0878339D287833006878CB7
:10FD2000288087A2F42A879EEC028783430887AB4A
:10FD3000F14E87C2C5C887C6C6408795269487B04E
:10FD400010FE87AB244287BDED28879064BC875F97
:10FD5000667887DDC40087C212F687C6FE5087C268
:10FD60000FEA87FCAB2887DDEA5287D8F17E87D47B
:10FD7000164A87E6F31687E6F13C87E6F31687DD39
:10FD80000FCC87F3E81887EAF31687EA064887E678
:10FD9000F166880AC82687EFF29887EFF29887F80D
:10FDA000F29E87F301C887F8030C87FCF3DC87EA2F
:10FDB00033C68805F6B28813F30A880EF3A68813B3
:10FDC000F31088050DB08813F3E28820F1308829FC
:10FDD000EE548829EE5A8829F11287F8BB6C8825E1
:10FDE000F658881326108817266A881C261088372C
:10FDF000F19688320B528840EE6C882928B08844EE
:10FE0000EE42883B0B5888400B5888372676883B53
:10FE1000268E884904148829417088294AAC885F55
:10FE2000EF0E885B0B948864EDAC884D274E88718B
:10FE3000D684885226B2885F060C883203BA88328C
:10FE400003B48891C5388891C5328883F670884D8F
:10FE5000520E88C2A4AA8871270688712760888CF0
:10FE6000F406887F25F28895ECBC887F25E6889586
:10FE7000F0E288A7ECB0888326B2889EECC8888818
:10FE80001E7E8888263A8888276688A3ECB088A7D3
:10FE9000E44C88B0D99C88B9C820890A9C52887AD9
:10FEA000498C88C7BEF688ACEE12889143EC88BEB8
:10FEB000EDA688A726AC88AC26D688AC280E88B0DC
:10FEC00026A688C2FAEA88C7EDA088C2023A88BE90
:10FED000332488D9ED8888C727BA88CB252088D4D1
:10FEE000275488D027968921AC3088DD26D088E633
:10FEF00026E888FDED6A88FDEADC889E62B888EF16
:10FF0000278A88EF25B688F4278A88EF3108890187
:10FF1000EC26890AEC4A88F8275A88FD277E89064C
:10FF200013EC88FD275488F4347A8901274288FD30
:10FF300034088906274E890A274E890A275A890AD2
:10FF40002754890A273C890F2742892EEA82892A69
:10FF5000F7728933F77E8925118E891C27BA891C8F
:10FF6000275A8918276C891C275A8933F664891CFB
:10FF7000275A8937EB60894EF778892127548937CA
:10FF8000F9948940ED1C891C25D48921344A892A99
:10FF90002754892A27A8893327DE8945ED16892A1F
:10FFA000274E8945EC628937038489184260894964
:10FFB000EB96895BD4808949FFF48960D498893CA9
:10FFC0002742894027968945276C8976C3DC895B5F
:10FFD0000258894527128940349289403486893CE9
:10FFE000347A8960F99A893C348C8945426C896DF0
:10FFF000F9AC895727188972F004895B2736895B29
:020000021000EC
:10000000293A8960272A897FEAF4897BF52C89724D
:1000100026D68976276089A3F4A28996277289D586
:10002000C5C289A3276C899146F289CCEFDA89B1E0
:10003000276689B1143A89DED51089F0BD9A89A363
:10004000483089D9F17889F9BD8889D9F83289DEB3
:10005000F53E89C7277E89C727A28A0FBA708A0F03
:10006000C2B08A0FCE5089F9F4D289D928D48A1423
:10007000C2CE8A02F6DC89FD28F88A2FCB2C897F34
:100080006A088A2FD62A8A02317A8A0626C48A21E9
:10009000F4BA8A1D2EAA8A2126BE8A2127008A2622
:1000A00028E08A213AAA8A0F4F2C8A60D84C8A38D5
:1000B00028E08A1D4B548A5CDEB28A5713328A6E5E
:1000C000DE348A53282089D969E48A144B7E8A2633
:1000D0004B788A84F8F28A9FBA648A334E428A7BCC
:1000E00019E68A7222E68ABAD7BC8AA8F6768AA866
:1000F000F11E8A9627D28AB1EA2E8A893A9E8A967A
:1001000031808A8449088AD5C3648AC3F8628AC365
:10011000F8988ABF034E8AB1105C8AD1DF188AD55D
:10012000DF1E8AD1F4FC8ACC013E8ADEE8CC8A8DBF
:1001300047408ACC02588AD528A48ACC4B368AFEFE
:10014000337E8A9F3D808B1029AC8B07341A8B2F0E
:10015000E4F48ABF576C8B1923B28B02466E8B4F27
:10016000E9CE8B61C3648B26203A8B4104808B22BD
:1001700033068B4AF9EE8B3D21E48B61E86C8B658D
:10018000E48E8B5C06A88B5311B88B3D40F88B7CBA
:10019000E4828B413DEC8B61198C8B5C2CB88B9B82
:1001A000C3948B7708888B89EDA68B5342308B8E56
:1001B000E8CC8B97E95C8B7727188B7733788B416A
:1001C000635A8BB6E8CC8BB2FA1E8BBFE8AE8BC4F9
:1001D000E9988BBBFA248B8048188BAD2B2C8BD6DF
:1001E000DE468C0CAB888BD1E8F68C19A6D28BE35B
:1001F000E9088BE3E8C68BF1D8168BECE8F08BE3CB
:1002000004088BFAD83A8BDA29B28BFE18E48C19E1
:10021000E89C8BE33B1C8BF52B808C032B9E8C1076
:1002200011A68C190B048C27087C8C4BDA448C5853
:10023000CE2C8C58CE508C73BC9E8C342BB08C58EA
:10024000F19C8C58F1C08C6FE26C8C66F1A88C7CB0
:10025000EE728C660B288C78EE608C85EB188C58CF
:100260002C408C7C0AFE8C85EE128C8AEE368C97A4
:10027000D9788C8EEE248C850BD68C7C28148CC976
:10028000C28C8C7337B08CAEE14C8CAEDDA48CD6B6
:10029000C2748CB2E3028CAEEE548C8E2A8A8CD25D
:1002A000C2808CD6C2808C9C20588C8E38CA8CC060
:1002B000EC328CBBFCCA8CA92E868CC9EE728CA940
:1002C0002E9E8CDBEDA08CD20C9C8CF1D96C8CFA20
:1002D000CC7C8CB73C908CDF00788CF1ED6A8CED97
:1002E0000BEE8CDF36308D30D2888CC951128D11D7
:1002F000ED9A8D1EEDC48CF636788CDF51248D542A
:10030000D2828D23139E8D2325F28D2727D28D3EF9
:1003100008FA8D50EEBA8DB3A6D28D78CB028D59E6
:10032000F1068D303C908D78D55E8D500DA48D7D7D
:10033000D5588D4B2C648D98C3828D5913AA8D622C
:10034000F1A28D542B928D6613CE8D7DFA548D8F34
:10035000E2488DA1D60C8D7813508D7813C88DE9A5
:10036000AD028DD2BD3A8DBCD05A8D7D332A8D81A0
:1003700033308D81333C8D23632A8D8A3CD28DC5E9
:10038000EEAE8DBC02F48DC903428DB332888DF67A
:10039000D66C8DC917B88E04D65A8E08D65A8DC021
:1003A00032A08E50A6D28E28BB368DED2D068DFB49
:1003B00018FC8E1604328E16086A8E3ED15C8E3A78
:1003C0000FD88DD74A2E8DE44E068E2310028E163E
:1003D0002D068E2311DC8E98AA508E1141A08E59C5
:1003E000E6BC8E4310808E4317FA8E1A41888E43E6
:1003F0000F788E430F788E4310928E4310988E475D
:1004000010568E4710868E4717A68E5012B48E82D5
:10041000D8708E67FD908E6BFDA28E6212DE8E62AA
:10042000111C8E5E2BC28E9DCF168F00A3368E7D43
:1004300019808E820FC08E8BFD7E8EB8D1448E5E69
:1004400042608E6242788EA1FDBA8EA6FD9C8E6BB4
:1004500041A08E7D30F68EAFFFF48E3E4AA08EC155
:10046000FD9C8EC5F3A08E5052268E5E57EA8F09F2
:10047000BC4A8EC5138C8ED30A4A8EDC0A508EE598
:100480000A148EF2FE8C8ED70A448F3605CA8EE08F
:100490003AE08F43D0E48EC1582C8F1B191A8EC5B9
:1004A00058448FEABF868F6CD0F08F3F136E8F3F1A
:1004B00013508F2830CC8F4C09188EF7486C8F431F
:1004C000138C8F5101FE8F2D30E48F1B43628F5AA6
:1004D00013388F6704328F70F40C8F4830C08FB49C
:1004E000B9EC8F75093C8F9DD6008FB8C3B88F3695
:1004F00048968F870A5C8F6C32048F8BF4308FA202
:1005000003E48F7935EE8FE5BF7A8FB405768FB42B
:1005100005BE8FCFE6DA8FB40C7E8FB816748F705D
:10052000480C8FB4268E8FD8065A9020D37E901216
:10053000EFD48FAB504C8FD843E69020012C902401
:10054000012C90052B929036DE769032071A8F554B
:100550006984902427F0906CD5EE902933D290AB2B
:10056000BC3E903F36849083EC8090FCA786908CB4
:1005700005F4906C2A5A908727EA90833222908C57
:1005800029F4908C29EE9090321C90992A1E906C40
:100590004E4890714E4890A229FA914DA78C90B97F
:1005A0002A4890565F28914DACC690EF02EE9144D8
:1005B000B7C4910129E891ACA50A910A3A5C91135C
:1005C0003AAA9171D53A917FD47A915B16E0910E57
:1005D0004DBE8FE56FBA91403DAA91443DB09195D3
:1005E000D52E91F8ABB8919A058E914440D491B034
:1005F000D516918335DC91E6D4FE9188353491BED1
:10060000F5E09218B800915F55BC91E6E9DA91DD0A
:10061000001891B9384091DD2F4C91D9383A913B6F
:1006200062EE9296A2769296A900921C070891FD1E
:100630002F6A91FD2F6A91F43A2C92062F5291C79E
:1006400054A8911C6C129245F77E921335D6920AEB
:1006500037A49245FCE89269D7F292490348926D1B
:10066000D7F8925202F4924517E292B1BBC6926952
:10067000FE6E926D03FC92453CD2925737D4928421
:1006800007569291F4D891BE662A925B3534922532
:100690005436929AF55C91E6680492A8FE0292762E
:1006A00037AA927B2F1692A3075C9276354C927FE5
:1006B00038C492843552928832D6928438A6928475
:1006C00038AC929138BE92C7078092F4D558929F69
:1006D00038A6939F9D0092E7070292BA361292C302
:1006E0003A1A92F9076292FD070E934AC2329306B4
:1006F000FFAC9341C7C692B14C689318F84A929FD9
:10070000555692E738E892BA5286932A076893388A
:1007100008949318290492D553AC9302426C931811
:10072000352892E25406931D34E693C3AC3C9357AC
:1007300008D093263ADA9353093092526B2293579A
:1007400008EE936008889377EC1A92F95400932F7F
:1007500038DC93214116938DFB8093BFD774936946
:1007600034AA9369349E937B28F293DED04293E7B8
:10077000D180939230EA93C3FBFE939B32FA935756
:10078000541E93A435B293DA001E93DA0ADA93B6B4
:1007900036BA93D1370E943DC5CE93F50D5C93C810
:1007A00039A893FE0C9693336780934A5B5094026A
:1007B0000DFE9321638494070D4A94070B52940B0A
:1007C0000AD4944FD036942FEB7293F52F9493C89C
:1007D0004D9494220D26942B0D4493CC44229441A5
:1007E000F7789441F7849441F7849441F78493CC4B
:1007F0005370942F0D32944AF7A294192DBA943D58
:100800000D4A9453F7B4944A0D7A944F0D62944F65
:100810000D8694024122942F30E4943830C694859A
:10082000F256940B4E7E9441316894463144948E36
:100830000D8694194C569426452494194C629419AB
:100840004C4494224C7492B16DFE942F4C5C947C79
:10085000143A942F4C38948510B694384C6E9438D2
:100860004C509497127894FEBC0E944F4C6294585E
:100870004C7494BB0D2C94E8D5CA94C8F83894A055
:10088000282094CDF84A94D1F85694260D2094C887
:10089000087C94774C8094DFF850947C4D34948994
:1008A0004B7894924E669519F77294A44C989519CA
:1008B000FD9C94B25C5E94C8475294D647529522F0
:1008C0000C90957CC31694DA4D6494EC4D5894F5D5
:1008D0004D7C955D0B5E9510D12C95C4BF32956A09
:1008E00018AE959308F495811B9695AEF8E695D6CB
:1008F000D4E695D6D9DE95B2FE62957C36AE959754
:1009000024249593327C9573444695D601C8955816
:1009100054FC954F54F695D2164495DB12B495FAD3
:10092000FB7A95FFFB9295D622AA95D222AA960C25
:10093000E6B695F60C1E95DF2B6295FA1CBC960C5C
:100940000AC895DB3744966FBC5695F13234961A37
:100950001D5296300A7495D246D49662063096425D
:10096000154E9642239A9635333096661416961A8B
:10097000513C965D32E296810BA6966632EE96E980
:10098000C2F896980F4E96A10F30967D31B696C557
:10099000F59296C00B829686378C96BC09EA96C073
:1009A0000A8696C00B8296425460968A37AA96C9E8
:1009B0000A9E96D20AC296A5336C96AA337296D72F
:1009C0000AA495616E8896D2235896E90A5C96E44B
:1009D000121896FB07A496FB09E496E424F6970800
:1009E00009DE96FFE5189747D6DE96E43354971F45
:1009F00009E4970422E0973105A096B75298973101
:100A00000E6A973109EA973509DE973509D8973A82
:100A10000588970D3168971131569743059A9711BC
:100A20000A74971A316E971632D0974709B49755C2
:100A3000048C975508B8975E0498976204D497621F
:100A400008B89743317A974C3186975E2106974CC8
:100A500037D4977912969798FF7697234FC8978B3C
:100A60001284978F139297703162977031929779B1
:100A7000317A97A1134A97DCD7AA9831B2EA97BC8A
:100A800024EA97E9E87E979D343297F7E86C979DC2
:100A900038B297D3093C97D7149497AF38AC979452
:100AA000470A97B838C49800FB7A9812ED7C988B67
:100AB000AC24971164AA97C13ABC97DC30FC97EE3E
:100AC000229897E92E6E99A791C097E5311497E582
:100AD000310897E9310897E9333C98E5AA9E987068
:100AE000FCD0987506C0979D61D4988B0B9A98435B
:100AF000444698702EBC985548909867382E98E1D7
:100B0000D62498AB0FFC98A6193298A22454988248
:100B10003A0898554F9298A2FFB8987E40E698DC24
:100B2000F79698AB268E98E1049898BD209A98E1A4
:100B3000048C98B82AC0975070A498CF288698CA79
:100B40002A369968C1E4990010C2990E0A3E98D8D5
:100B500031D4990910B0990913B0990913B09912B9
:100B600008709929FEB09917086498F72BE698EA5F
:100B7000331E991B13AA990031AA990E2904995A78
:100B80000060992023A698E545C6994408C499D8E1
:100B9000B07A999EE8B49995EB7E995A0B5E997A52
:100BA0000EBE990053A69987064299680DE699EF03
:100BB000BF62988761EC99632C8899324644999971
:100BC00007A499633306996C459099AB23CA994D54
:100BD000517299CF078099F3FFEE99EF0BAC99C64C
:100BE000447099CB447099F333609A052A0C99FCB0
:100BF000334E99CB4C9E9A9AC0AC99E6448E9A4952
:100C000003369A52FF709A6404C89A0544529A9E19
:100C1000DAB09A37336C9A293ACE9A173A9E9A32BA
:100C200036189A64297C9A2E44469A8C078C9A7AB4
:100C30001CDA9A6D297C9A5238FA9AA7FEFE9A71AC
:100C40002ADE9A4048849A6438E89A7A2AD29A919D
:100C50001C329A951C2098E16EE29AB9FF9A9A5F2D
:100C600041949B49AF129AE2E76A9A7141A69AD4DD
:100C700004E09AD9FF8E9A6847889A7F41A69A83A2
:100C800041A09A7F41A69A8841B89AE2030C9B330F
:100C9000E6149AC72FCA9B1CE7BE9B0AF3469ABE6E
:100CA0003C1E9AB03C249ACB365A9B2EFF829B96D0
:100CB000E2A89B1C28689B4E0FC69B401A8E9B6423
:100CC00002469B213AD49B76025E9BC3EF449BB5C0
:100CD000EF689B96E29C9B60E6029B96EC689B8D7E
:100CE00002BE9B7611169B911ED29C41B3569BC7A8
:100CF000FFB29B604B1E9B9F36729BA336729BA3D9
:100D0000368A9BA836849C06EB1E9C0FE52A9BF036
:100D100013389BF912F09C0B1A0A9C4AE35C9C382E
:100D200011889C45118E9D14B5EA9C9607329D0250
:100D3000E1F49C6542A29CD1FC709CE70B289D0BC2
:100D4000058E9CD529FA9CBF39189CE329E89D198A
:100D5000050A9D2604FE9D41042C9CAD52EC9D3D50
:100D60001A349CD54E9C9D3828B69D9BE7BE9D7C31
:100D700010B69D10493E9D2F3BD69D2249569E0799
:100D8000C4EA9D613BC49D0249329D9B2A7E9DC45D
:100D90000BA69DFEE4E89DECFE7A9E19E8849D7307
:100DA00045F09D8E45729E19E8A29D8E45E49DCD2D
:100DB0002A249F2C9A249E8EB6FE9E46EC749E4B4F
:100DC000EC6E9E61EC749D7345D29D7C45EA9E3429
:100DD00002AC9D7359E29D1D66AE9E5DEC149EA90A
:100DE000E6DA9E4B02469E61F5869E6A02649E7319
:100DF00002469E4BE8549E93E9509E22E93E9DFE9A
:100E0000460E9D2666D89DFA4BC69E034BD29F1E6A
:100E1000B3929F35B1D09EE8D1809E8E1A4C9E2B06
:100E20004E129E8524849E4F464A9EAE20D09E81BF
:100E300043509EED01B69DD164CEA04799889EE8AF
:100E4000D1809E9C44B89E1E67E69F0811C49F27D0
:100E500002F49F2C024C9EF6297C9F3002CA9F0C04
:100E60001DA09F86CCE8A016A50A9F42024C9F5465
:100E700002409F5008FA9F6202D09F6BEB789F74EC
:100E8000022E9F6B12189F6F12129F3937929F93F9
:100E9000039C9F9805949F7D19F29F861B909FC08D
:100EA000F03A9F8A1B8A9F5D3BF49FD7F0169F42C2
:100EB0004E24A01AE60E9FE4044A9FF200BA9F59FE
:100EC0004E6C9F544E609FF200BA9FF200A89F5D47
:100ED0004E009FFB00BAA023EFD4A074CA609F9875
:100EE0004CFE9FD249E09FE04CA4A074F910A0A151
:100EF000EBF09FED5028A0DCEB849FCE5886A12814
:100F0000BFCEA0E0EB72A0862CD0A0DCF1D2A07006
:100F100039F6A0CE0198A0823A08A08B3A20A15AB7
:100F2000E746A112EFCEA09DEA34A0983B04A0436F
:100F3000541EA0A13B0AA0A13B0AA143E272A167F3
:100F4000DE1CA0D73B22A0DC3B5EA0DC3B58A0BC53
:100F500046CEA179DE28A17902EEA0E94E12A0FBCF
:100F60004F38A1004F32A1244DEEA03A69FCA1995F
:100F70001D6AA1CA04F8A04369FCA1E1FC5EA17E40
:100F80003AE0A200ED94A200ED7CA1F7F5A4A199AE
:100F9000408CA1FC0AE0A2090AD4A20E0720A1EE0F
:100FA0003A98A1EE3AAAA20E2BECA313B356A25183
:100FB00011DCA320B8C0A2C2196EA2CB3A98A2CB72
:100FC0003A9EA3640AAAA2EA445EA2F3445EA3295D
:100FD0003C5AA32E3C60A37A1242A39EFC0AA49A18
:100FE000A1F8A29060AEA3B00A80A3BE0A50A3C22B
:100FF0000A44A3713C2AA3C70A4AA3713C5AA472AB
:10100000B8C0A39A3C12A3FD059AA3205B14A3BE0B
:1010100038DCA4211518A45206F6A4451560A4498D
:101020001560A4600720A45B1086A46D10F2A44E86
:101030002850A4C7E8A2A49107F8A4642B62A49F37
:10104000175EA4184F92A4D0086AA42E4FBCA47FA8
:1010500037F2A6A99598A538D50AA4574F68A4F9E0
:101060001122A4764F6EA50617F4A545F3E2A50F4D
:101070002CA6A53C1E30A4AC5382A54E1812A5A8E0
:10108000ED64A697A9EAA57B1632A4DE5382A502D9
:101090005376A5B60B94A5BF1404A52A5370A64F8A
:1010A000CADEA53851AEA60B0E76A5805406A65C06
:1010B0000360A62B229EA60239C6A60739D2A66EC9
:1010C000191AA6B6EC9EA6731920A6890BB2A6E340
:1010D000D7C8A761B098A6FAD6A8A6972844A6971D
:1010E000283EA6DF1ABEA70C1AA0A803AF3CA7850E
:1010F00010ECA79710CEA7811DB8A79C10FEA7C41F
:1011000000C0A6656576A7BB1482A781392AA8030B
:10111000085EA73D57A2A80825F2A8420870A8506B
:10112000164AA7665B32A8421F80A8501668A85DC1
:1011300016E0A85D16ECA78E5B50A967AAECA8FF85
:10114000CF70A89C1D2EA8FF1B36A91A11ACA9119F
:101150001944AA16B3F8A9471D7CA986FD00A95910
:101160001830A9591D64A9860570A9860558A935A6
:101170003486A98618E4A98618F6A98F18EAA98FDB
:1011800018E4A99D1902A9A11920A9A618F6A99DDC
:101190001B36A9A618EAA854636CA9C10B64A9B3AD
:1011A00018FCA99D21A8A9AA1CE0A9B31980A9B37C
:1011B0001902A9B8198CA9B81944A9BC198CA98617
:1011C0003936AA0DF6FAA9CA1E3CA9DC19AAA9DC6F
:1011D0001BD2AA040B34A9FB1CE6AA121380AA1B7B
:1011E0001398AB12B3C2A7F16F18AA1B36BAAA8222
:1011F0000102A8F2634EAB09CD0CAA87177CAAC1E5
:10120000140AAAC121AEAAB425C8AAB425E0AAE14D
:1012100013F8A98B61ECAB0E030CAB090DE0AB7EB0
:10122000CFD6AB1713ECAB3F18F6AAF3294CAAF7AD
:101230002976AC13AE94AAA250D0AAFC2E74AACFE1
:1012400049C2AA1F6252AAFC2754ABBDDFAEA9E96E
:1012500065F4AAB45628AB56255CAB44315CAB7E32
:101260001B5AAB7E1B5AABBD0120AD499A78AB7EB1
:101270002796AB832CEEABA73234ABBD3108AC0E56
:101280000A6EABC6310EABCB3162ABDD3138ABD8B9
:101290003156AB7A5838ABE6315CAC2013DAABF898
:1012A0003174AD13B6ECAC0E316EAC253426AC9572
:1012B000FCCAAC373528AC3B3522ACE6DAB0AC4DD5
:1012C0003528ABC65718AD40C6D0AC135100AC831F
:1012D000332AAC205184AC1C518AAC95356AAC2EB3
:1012E0005106AC9E36C0ACEB1098AC494FB0AD9FE8
:1012F000BAE2AC175B44AC684EAEACD03552ACC76A
:101300003990AD9FC95EAC6D5BF2ACD03960ACDD9D
:101310003468AC914D76AD8DDB64AD253990AD2E42
:10132000397EAD2A398AAD8421DEAD911B90AD495D
:1013300038F4AF7C98FEAE80B602AE4AC766AD40C8
:101340004614AD574404AEDEAAC8AD454DDCAD9F92
:101350003762AD913C06AD9F398AADBA2E26ADBE3F
:101360002E38ADBE2E38AEBABC5CAEBABC5CADC7D2
:10137000379EAECCBA40AE451C68AEBFC20EAD7F44
:1013800053CAAE77EDA6AE65FDEAADFD3966ADF99F
:101390003972AE02392AAD9653CAAE213150AF0729
:1013A000BFD4AE263162AE1D390CAE6E1BE4ADF07B
:1013B0004E12B0109E6EAE4A3912AE9631B0AECC1F
:1013C0001E4EAE4E512AAFDFBB66AE4E53E2AE604C
:1013D0005232AE6052B0AFD6C304B003BB6CAF2F75
:1013E00032E2AF2B36E4AF5332C4AF5832ACAEFE6C
:1013F00050E2AF9B32C4B085BD3AAFD12166AF1D7C
:10140000571EAFDA216CB0EDBDE2B0153348AFCD59
:101410005274B05433CCB174B452B2709A00B093D9
:10142000217EB00C5142B05D37F8B00C5154AFB2D0
:101430005CD6B1BCAD0EB16FC118AE7B6DF8B10C0E
:10144000FD42B0E40CB4B10CFF9AB208ACBAB1AA38
:10145000C112B0545694B13908DCB13E08BEB06632
:101460005724B1D2C60AB13024D8B10342D8B1A5AD
:101470000672B23EC538B05D6354B18F2124B1E02D
:10148000062AB223E0CEB0936390B0ED62FAB10CBD
:101490005760B18F3C18B2110360B18F3FD8B2864C
:1014A000C874B1F620D6B1355772B0C06390B1861A
:1014B0004E1EB139588CB0E862F4B2E0C106B2F207
:1014C000BF98AE7B7416AE777428B324B5DEB2CA6B
:1014D000FA3CB2623354B336CBCEB29837C2B1F2D3
:1014E0005526B36CC130B1DB599AB2AF2760B22C2C
:1014F0005010B2B82724B2D32730B2DC272AB382E7
:10150000D5A6B2FB2052B3B8C820B2F22730B3122E
:1015100026DCB316275AB31B2748B3C1DB10B331FF
:101520002A1EB28658F2B35A2082B370206AB3756D
:10153000205EB31F426CB3A20960B424CAB4B37076
:1015400029F4B3314638B417DD2CB30452F2B30D8D
:1015500052ECB436E014B2DC6042B2E9605AB375C2
:1015600052F8B37552ECB3D355DAB517DA9EB51C01
:10157000DAA4B3D854D8B4D4057CB3EE573CB3E561
:10158000573CB42D57D2B649A7AAB4CF3B88B5B5BE
:10159000CBD4B431601EB5D9D690B67AACD2B4A251
:1015A0005568B4A7556EB56820E2B5C6EDD6B4B49B
:1015B00055C8B5293A92B5323B76B52043F2B5838A
:1015C00020B8B58C20A6B637D870B4EF586EB66D7B
:1015D000C886B4FC5892B59138A0B5D91C8CB68D8C
:1015E000C39AB5A33D8CB43F6A0EB676DE94B6F4CA
:1015F000B73AB5C23D5CB777A49EB5D03D6EB61381
:101600002952B3EA6E94B5EF3D62B6ACE5F6B6E7A3
:10161000CDC6B6E7D5A0B62A3D98B738C9E2B5FD24
:1016200050BEB64D3972B52065ACB64D3CA8B70674
:10163000E476B65739BAB6523BB2B5FD50A6B5FD01
:10164000509AB6CC1770B6883A92B6A732B2B69610
:101650003A9EB6AC32ACB7C8BBEAB7061614B79F11
:10166000C9D0B784DAF2B772E6F2B79FCFF4B6A367
:1016700049FEB67256E2B7C3D5D0B691553EB8E82A
:10168000A1B6B74A39D8B79B2958B74A5772B82B71
:10169000F8DAB7BA351CB80F103EB873DE94B765E8
:1016A0005028B8142544B8222538B79252FEB8FA0B
:1016B000D228B87316C8B7C352BCB7C352BCB8ADB2
:1016C00008D6B8AD16E6B985C910B8195466B82F52
:1016D0004FF8B96AD234B8FE09F0B83850EEB861A4
:1016E0004A28B84A50F4B9AEC118B90C1710B84F0F
:1016F0005484B86152C8BAF29DDEB8A053E2B896DD
:1017000053B8B7F063FCB9FECEC8BA74B488BACE89
:10171000A942B8E353DCBA78CC0ABA15DE5EB9E860
:10172000FB6EBAE4A942BA42D13EBA58D2B2BA0864
:101730001A7CBB35AA98BA1E1A88B9BB4764B97C13
:101740005586B98E5580B8806A74BA7411BEB8AD2A
:10175000689ABB1ACEC2BB1AD282BAA12148B9FE7E
:101760005292B99C5FD0B9A45FA6BB59D09CB9AEC8
:101770005FACB9C05FD6B9A9626ABB8BD3A8BB31D5
:101780000438BAF623D6BB0423E8BB0823A6BB2340
:101790001986BB1623DCBBA1DD02BB0833B4B9C478
:1017A000655EBA58580EBA8A5502BBEDCE2CC26A95
:1017B00087E2BBCAE8D2BBE5E35CBC1FCBE6BB8BD0
:1017C0001D2EBB23439EBC00CF0ABBF2E3DABB66EF
:1017D00031FEBB7031FEBB164B48BAFB4FDABBA6DD
:1017E0001A22BC36D582BBBC1D52BC3FCF58BB3180
:1017F0004E54BC70CE3EBAC05F04BAD25D78BBF224
:101800001D46BB5E4E66BC041D34BA1A675CBB281D
:101810005706BAF25F0ABB59559EBC99DC48BBC556
:101820004854BC3618A8BC3618A8BC99E092BB0C2A
:101830005F04BB0C5F04BB115F10BB8F50A0BB8B60
:1018400050A0BCC6CF0ABCC1D708BB045F16BBD72B
:1018500047EEBBCA4C2CBCE5D534BC9405DCBC6758
:101860002070BDC2A678BC632274BC672C40BC8BC0
:1018700029F4BC9029FABBF75784BC165484BCE108
:1018800019DABC1A5688BE56A29ABC28568EBD4894
:10189000E542BCEE19C8BDABC1C0BC4C53ACBC43A7
:1018A00053A6BD0519DABD2419C8BD2819D4BE95A3
:1018B000A402BBFB62A6BD242EB0BC515C2EBDCFE2
:1018C000DD56BDC6E788BC12654CBDBD08D6BCCA96
:1018D0005580BCEA5580BCEE581ABDC22304BE40F8
:1018E000DF9CBD634758BD005820BE29F364BDCBC3
:1018F0002898BE71D618BE71D8C4BD1B580EBE7ACA
:10190000D5C4BE83DDB6BDB44092BE360F8ABE4D8F
:10191000DED6BE291BC0BEB0D5BEBED0CCF4BEB094
:10192000DDC8BEA7E05CBDAF4F0EBEBDDD02BD246D
:101930005A72BE83FF94BD5F5B50BEC2E416BCD337
:10194000673EBEB0F556BEF4D8E2BF40C28CBDCBF8
:10195000564CBD995DB4BF21DCD8C002A654BF1C53
:10196000DF30BEBD2376BEE61A22BEDD1A10BEE60B
:101970001A22BF6DD672BDDC5DA8BF7BDB94BF7140
:10198000E614BF3718C0BF9AD94EC19B9454BFA864
:10199000D354BF9ADE1CBEC741E8BFB1E860BEB5F4
:1019A0004F1ABFF4D060BF711878BFF0D85EBF1374
:1019B0004980C041E52AC018E1A0C03CD33CBFCB60
:1019C00013D4BFC31DDCBFF809A2C045E0D4BFF0EB
:1019D0001512BFBE2BB6BFEB1E1EBFF81E30C0B621
:1019E000E33EC0021E24C0061E24C00F23BEBFC794
:1019F0004626C09FE0E0C11DB692C00637B6C04182
:101A00001DA6C04A1A7CC1A0A648C0D1E434C0D5E6
:101A1000E40AC04E1D94BF96565EC0571F56BFA322
:101A200055F2C0D5E40AC0ECE890BFD55604BF64B7
:101A30006120C0962310C09B2334BFF05664C0C3FE
:101A40002334C114E61AC106EECCC0D9EAF4C06E44
:101A50003CD8C002563AC00F563AC00F563AC0DEC4
:101A60001518C126EC9EC0B132BEC158E7E8C24687
:101A7000A714C11D12A8C0F91F4AC052563AC1800E
:101A8000E93EC1262148C1DFDA4AC01D6024C021D9
:101A90006018C146215AC203D54CC1ECEF0EC227D3
:101AA000DD08C1D61614C1BF2106C25DDF60C39335
:101AB000A702C2A0EF14C23D26B8C2B7093CC31AA0
:101AC000D102C2B214D6C1B65DB4C35DD282C347DF
:101AD000DC24C322ED70C2C8303CC2E82034C37499
:101AE000DEFAC15368DCC393DCA8C393E83CC30CA3
:101AF0003810C362E79AC2585B62C3BCF160C24F40
:101B00005FA0C21E64B0C423D19EC5AF98F8C214B2
:101B100066EAC3F6F796C43EDE64C3A52FDCC3CEE7
:101B2000202EC3CE2124C3ED203AC3ED203AC3D2E8
:101B30002D12C3BC3852C44CF472C3E92B2CC40D13
:101B40002F3AC33E5F9AC3B35E68C4861F08C3BC06
:101B50005436C46B2520C3C93C30C5C5A86AC4A18E
:101B600023B2C46B3858C3AE5E26C3C05E68C3AE32
:101B70005F6AC3C05E68C4D71F5CC570D294C528B5
:101B8000F94CC543F72AC675A456C4DC383AC4E4F8
:101B90003870C46253D6C5003300C3FB6330C3F64C
:101BA0006330C4C14E3CC52D30F6C52833EAC5CAE2
:101BB000F2C8C55A38D0C4E0536AC5CA23E2C65138
:101BC000DB8EC700AF66C5EE2D66C5705550C61BCF
:101BD0004044C629400EC6CBF8B0C6D3F730C7D9AB
:101BE000A72CC795B452C79EB476C6E60E8EC6BD66
:101BF00025BCC6754302C72DF3C4C6C22FBEC5EAB5
